:020000040000FA
:100000000848040001000000F82F0000F82F00004D
:10001000F82F0000F82F0000F82F0000F82F000044
:10002000F82F0000F82F0000F82F0000F82F000034
:10003000F82F00009E090000F82F0000F82F0000A4
:10004000F82F0000C4090000EA090000F82F0000A2
:10005000F82F0000F82F0000F82F00004AA1000040
:10006000F82F0000F82F0000F82F00008610000085
:10007000F82F0000BA07000026090000F82F000042
:10008000F82F0000E0070000F82F0000F82F000014
:10009000F82F00001E0A0000440A00006609000054
:1000A000F82F0000F82F0000F82F0000F82F0000B4
:1000B000F82F0000F82F0000F82F0000F82F0000A4
:1000C000F82F0000F82F0000F82F0000F82F000094
:1000D000F82F0000F82F0000F82F0000F82F000084
:1000E000F82F0000F82F0000F82F0000F82F000074
:1000F00020110000F82F0000F82F000094070000E6
:1001000054120000F82F0000F82F0000F82F000014
:10011000F82F0000F82F0000F82F0000F82F000043
:10012000F82F0000F82F0000F82F0000F82F000033
:10013000F82F0000F82F0000F82F0000F82F000023
:10014000F82F0000F82F000080070000F82F0000B3
:10015000F82F0000F82F0000F82F0000F82F000003
:10016000F82F0000F82F0000F82F0000F82F0000F3
:10017000F82F0000F82F0000F82F0000BA1100003F
:10018000780A0000F82F0000F82F0000F82F000078
:10019000F82F0000F82F0000F82F0000580800008A
:1001A000F82F0000F82F0000F82F0000F82F0000B3
:1001B000F82F0000F82F0000F82F0000F82F0000A3
:1001C000F82F0000F82F0000F82F0000F82F000093
:1001D000F82F0000F82F0000F82F0000F82F000083
:1001E000F82F0000F82F0000F82F0000F82F000073
:1001F000F82F0000F82F0000F82F0000F82F000063
:100200000000000000000000F82F0000F82F0000A0
:10021000F82F0000F82F0000F82F0000F82F000042
:10022000F82F0000F82F0000F82F0000F82F000032
:10023000F82F00009E090000F82F0000F82F0000A2
:10024000F82F0000C4090000EA090000F82F0000A0
:10025000F82F0000F82F0000F82F00004AA100003E
:10026000F82F0000F82F0000F82F00008610000083
:10027000F82F0000BA07000026090000F82F000040
:10028000F82F0000E0070000F82F0000F82F000012
:10029000F82F00001E0A0000440A00006609000052
:1002A000F82F0000F82F0000F82F0000F82F0000B2
:1002B000F82F0000F82F0000F82F0000F82F0000A2
:1002C000F82F0000F82F0000F82F0000F82F000092
:1002D000F82F0000F82F0000F82F0000F82F000082
:1002E000F82F0000F82F0000F82F0000F82F000072
:1002F00020110000F82F0000F82F000094070000E4
:1003000054120000F82F0000F82F0000F82F000012
:10031000F82F0000F82F0000F82F0000F82F000041
:10032000F82F0000F82F0000F82F0000F82F000031
:10033000F82F0000F82F0000F82F0000F82F000021
:10034000F82F0000F82F000080070000F82F0000B1
:10035000F82F0000F82F0000F82F0000F82F000001
:10036000F82F0000F82F0000F82F0000F82F0000F1
:10037000F82F0000F82F0000F82F0000BA1100003D
:100380009E480100F82F0000F82F0000F82F000011
:10039000F82F0000F82F0000F82F00005808000088
:1003A000F82F0000F82F0000F82F0000F82F0000B1
:1003B000F82F0000F82F0000F82F0000F82F0000A1
:1003C000F82F0000F82F0000F82F0000F82F000091
:1003D000F82F0000F82F0000F82F0000F82F000081
:1003E000F82F0000F82F0000F82F0000F82F000071
:1003F000F82F0000F82F0000F82F0000F82F000061
:1004000000480400010000004F0E2300807D2400FE
:1004100000018800000000000B000700A078290000
:100420000100200010000700000020000000E00094
:10043000020032000000020000000000ECB40200E4
:10044000000000000000FE004440A900E050210030
:100450000000E0000300320000002000A00188003E
:100460004440A80000000600F8FF2000591C2100AD
:1004700091018800800078000000EB001A0037002E
:100480008180E80032A0B4009101BA00E28040000F
:1004900032A0B4009102BA00E280400032A0B40061
:1004A0000002EB00472BDE00F507B200602CE100F4
:1004B00009003A00330007000700E00002003200A4
:1004C0000059EB00010037000201E8008301E90058
:1004D000F8FF3E00040037006128E100010032000F
:1004E0000082EB00040007001101BA000200E000E6
:1004F000E3FF3A0000000600220007000700E000CA
:10050000020032003159BA00020037008100E800D1
:100510000201E8008301E90017003200190007001A
:100520000700E000020032002159BA000200370043
:100530008100E9000201E8008301E9000D003200BA
:100540000400E00003003A00E280400032A0B40062
:10055000E9FF37000B0007000700E000020032004F
:1005600011D9BA00010037000201E8008301E90057
:10057000F5FF3A008100E800E180400032A0B400BD
:10058000000006000810E600020037000910E6002F
:10059000020037008083EB00000006008003EB00C0
:1005A0000000060091018800800078000000EB0048
:1005B00015003700E280400032A0B4009101BA007B
:1005C000E280400032A0B4009102BA00E280400014
:1005D00032A0B4000002EB00472BDE00F507B200AA
:1005E000602CE10004003A000059EB008301E900AF
:1005F000FDFF3E00040037006128E10001003200E9
:100600000082EB00040007001101BA000200E000C4
:10061000E8FF3A00000006003159BA008301E90002
:100620000C0032002159BA008301E90008003200B1
:100630000400E00003003A00E280400032A0B40071
:10064000F5FF370011D9BA008301E900FAFF3A003B
:100650008100E800E180400032A0B4000000060004
:100660006A9D0400000000005A9B04000000000086
:100670005E9B0400000000008E9B04000000000050
:10068000B69C040000000000C874040000000000D4
:10069000FA740400000000002A7504000000000045
:1006A0006C75040000000000AE750400000000003E
:1006B000F075040000000000367604000000000021
:1006C0009A76040000000000DE76040000000000BE
:1006D0002277040000000000907704000000000072
:1006E00008780400000000005A78040000000000B0
:1006F0007478040000000000FE7804000000000090
:100700004879040000000000827904000000000025
:10071000BC79040000000000507A040000000000D2
:100720008A7A040000000000847B040000000000BE
:100730006893040000000000129404000000000010
:10074000E093040000000000449404000000000056
:100750007694040000000000AA9404000000000049
:100760002A950400000000008695040000000000A7
:1007700058950400000000003097040000000000BD
:10078000B49504000000000006960400000000007C
:10079000A496040000000000D296040000000000AF
:1007A000EA96040000000000029704000000000028
:1007B0005A97040000000000CEB4040000000000BE
:1007C00050A1040000000000FAB304000000000083
:1007D000E0B304000000000008B4040000000000C2
:1007E00014B404000000000076BF04000000000004
:1007F000D8B70400000000002AC604000000000072
:1008000038A9040000000000027C04000000000081
:100810001A7E04000000000008CC04000000000064
:1008200034AC040000000000020AB900001BB9004B
:100830000200B80081004200810043000000060071
:1008400080017800110009008280D8008001FD003D
:10085000110009004288D8008300780000000600DB
:100860006022B800060220000000D0008180D20083
:100870000482D2008582D2000000A0000202520051
:1008800083825A00030031000202420083824A0040
:100890000000A1000603E900F3FF3A000000060093
:1008A000839F68000100E00002003D00600010002E
:1008B000E08018000300E00002003D00600111002C
:1008C000E0811900E6FF07004F00E00002003B0056
:1008D00060001000E080180000000600889FBE0045
:1008E0008A9FBE008C1F78000205BE000004BE0077
:1008F0000006EB00E00F5000E08F5800E00F5900B9
:10090000E08F590007003D006000B8006011B8009A
:1009100008045000898458000A0559008B85590045
:100920001C002000E00F5200E08F5A00E00F5B0037
:10093000E08F5B0002003D000F0007000C00A200EA
:100940000800BE000A01BE001D0107000203BE0030
:100950000002BE000C00E0000100320006000700AB
:100960000400BE000601BE004F0678004F05BE0021
:100970004F04BE00000006006000B8006011B8001F
:1009800004025000858258000603590087835900ED
:1009900000000600881F7800000478005001BE00A7
:1009A0004000BE0004004000858048000601490068
:1009B00087814900009CBE000294BE000400E10053
:1009C0000588E1000690E1000798E100020031008F
:1009D000680044001008E8004F047800000006009A
:1009E000F4874700889FBE008A9FBE008C9FBE0090
:1009F0008E1F78000205BE000004BE00D4B79F0021
:100A0000E5B79F00F6B79F0087BF9F000000EB008F
:100A1000C0B79F00B0B79F00A0B79F0090B79F00DE
:100A200080B79F000D042000BFB097004FB0970023
:100A3000000140000000E0000F003D004F08DE0014
:100A400000007100C0B79F009E00070001003D003C
:100A500012002000A100070001003D00120020004C
:100A6000A6000700B1000700B60007000F00400015
:100A7000C8FF0700220037004F08DE0000067100A3
:100A8000CCB79F008F00070001003D00120020003E
:100A90009200070001003D001200200097000700AF
:100AA000A20007000FB297009FB297002FB39700E4
:100AB000BFB39700A90007000000520081805A00D0
:100AC00002015B0083815B0080B79F0091B79F00AC
:100AD000A2B79F00B3B79F000007EB009F0007007D
:100AE0000020E10001A8E10002B0E10003B8E1004C
:100AF000010031001E0020000E005600C0B79F000C
:100B00004FB297000400E0000700350010002000FD
:100B1000010020006011B800080470008984700092
:100B20000A0571008B8571008D06E900BEFF3A0051
:100B30000400E00003003D00820007000F004000B9
:100B400094FF07004FA897000000E00004003A005F
:100B50000FB497009FB497002FB59700BFB59700CB
:100B6000940007004F0778004F06BE004F05BE00F7
:100B70004F04BE004F01B10000000600881F78003E
:100B800018002000881F780095FF07008F87E90074
:100B90004F04780000000600801FEB0090FF070064
:100BA0008F87E90000000600889FBE008A9FBE0074
:100BB0008C1F78006E00070007003D0073000700DF
:100BC000E00F5B00E08F5B0007003D003200070094
:100BD0000006EB00040037003400070002003D006F
:100BE0002A0007001C00200072000700E3FF070036
:100BF0000203BE000002BE000C00E0000100320053
:100C0000220007000400BE000601BE004F06780067
:100C10004F05BE004F04BE0000000600889FBE00C6
:100C20008A9FBE008C1F78005100070005003D0020
:100C300056000700E00F5B00E08F5B0006003D0000
:100C4000040037001900070003003D006000B800F1
:100C50006011B8001000070056000700CEFF070023
:100C60000203BE000002BE000C00E00001003200E2
:100C7000060007000400BE000601BE004F06780013
:100C80004F05BE004F04BE00000006006000B80023
:100C90006011B8000000370004025000858258003F
:100CA0000603590087835900000006000006EB0088
:100CB000E00F5200E08F5A00E00F5B00E08F5B0016
:100CC000000006000180400090B79F000001EB008B
:100CD0008FB097000100E0000000060002007000E5
:100CE00090B79F000180400080B79F000001EB009B
:100CF000FFA897000100E00000000600020070005D
:100D000080B79F00018040006FAA9700CF20DE00CF
:100D100001007000F0AF9F000402420025000700B0
:100D20004F18DE000002720000000600E4AF9F00D2
:100D30000804440089844C000A054D008B854D0051
:100D4000000006003FB29700CFB297005FB3970054
:100D5000EFB3970000FE2F00000006003FB09700A1
:100D6000CFB097005FB19700EFB197000000060089
:100D70000205BE000004BE00E00F5000E08F5800E6
:100D8000E00F5900E08F5900000006006000B80035
:100D90006011B80008045000898458000A05590001
:100DA0008B8559001C002000E00F5200E08F5A0094
:100DB000000006000800BE000A01BE000000060098
:100DC000889FBE008A9FBE008C9FBE000404B800AE
:100DD0000506B8008904460060854E000606B80086
:100DE0000A054600E0854E000706B8008B05460060
:100DF000040EB800890446000A854E00E0854D00C7
:100E0000050EB8000A0546008B854E00060EB80098
:100E10008B0546000416B8000A0546008B854E0077
:100E20000516B8008B054600041EB8008B05460069
:100E30000800BE000A01BE004F06BE004F05BE00FE
:100E40004F04BE00000006000400FA00E0BF9F004F
:100E5000E4815700812978000002EB000F00370081
:100E60006FB89700904078007FB8970010407800E6
:100E70000402E80080CF5000040032008180FB00B3
:100E80000080FB0000805000070037006FB897001B
:100E90000000E800E0BF9F009309E800820F5200C5
:100EA000EFFF3A000000EB000080FA0000000600AF
:100EB0008001EB0002003700817178008301E800B7
:100EC000828F5100FCFF3A0000000600800078008D
:100ED0003004E000FEFF3A00010050000000E9008D
:100EE000000006008001EB000200370061F079008D
:100EF0008301E800828F5100FCFF3A0000000600E9
:100F00003400F800881F780008002000A80188003D
:100F10004F0478008D00A9009D00A9008AA0A800B8
:100F20003400F900004006003600F800809FBE0043
:100F3000829FBE00849FBE00869FBE003400F800E2
:100F400000002000A00188008AA0A9009AA0A900A2
:100F50000000EB00915607003400F9004F03BE007B
:100F60004F02BE004F01BE004F00BE003600F90028
:100F7000004006003600F800809FBE00829FBE0041
:100F8000849FBE00869FBE003400F8000000200051
:100F9000A00188008660A900DA42E20001003D005D
:100FA000C45B07003400F9004F03BE004F02BE00CF
:100FB0004F01BE004F00BE003600F90000400600A1
:100FC0003600F800809FBE00829FBE00849FBE0056
:100FD000869FBE003400F80000002000A0018800B9
:100FE00086E0A900E30B800078C1BF0081CFB30089
:100FF0000140600078E1B700F0E2A80035C6A90022
:1010000042FA8000C9C2BF000058A3000B003A009A
:10101000007122000018B80009FE070022C5210057
:101020000001510093002000110009000301D800C5
:1010300080017800CDA2A9000E0037000200E00078
:101040000B0032006F10B80003004000E080480041
:1010500068004000E08048004C09DD004400DE00EC
:1010600000007100C408DE0040FA8800010037006B
:1010700043FA8800EC62A90051FA80000100E00008
:10108000020032000300780001000100F0C2A90054
:10109000C9A2A9003400F9004F03BE004F02BE00F0
:1010A0004F01BE004F00BE003600F90000400600B0
:1010B0003600F800809FBE00829FBE00849FBE0065
:1010C000869FBE003400F80000002000A0018800C8
:1010D0008FA0A90031F68000C41EE2000E003A0085
:1010E0001000200020F68800200C800010F68800F8
:1010F0000000280000F68800E0002000F0F58800DD
:101100006011B80001007800A331070030F68000BC
:1011100076340700460037006011B80001007800FF
:101120009D31070080C1BF000048A3003D00320090
:1011300037003700210C800010F68000008150003D
:1011400011F68800F0232A000000410021D222007D
:10115000810F50000C003E0001F68000F2F5800087
:101160008201E800100020000300DD000080600024
:101170000000D1008080700001F688000201E900C3
:10118000F2F5880024003700B0512700000041002C
:10119000C1782300810F50000C003E0002F6800051
:1011A000F1F580000100E800130020000018DD00C8
:1011B0000000610013003A000118DD00000071001A
:1011C00000F688000100E9000F00370020272C00FE
:1011D000800F51000E00360002F68000F1F580000D
:1011E0000100E800130020000018DD00000061008D
:1011F000070032000100E9000018DD000000710066
:1012000000F688000180E900F0F588000200370050
:10121000635E070006003700BE1EE20001003C00CE
:101220005F5E070080C1BF000038A300C1FF3A0025
:101230003400F9004F03BE004F02BE004F01BE0054
:101240004F00BE003600F900004006003600F800EE
:10125000809FBE00829FBE00849FBE00869FBE000E
:101260003400F80000002000A00188008680A9005A
:1012700082B48000A1B48000F0072000808F50006D
:1012800004003600606921000200E00004003A001A
:10129000060037000200E000040032006071210007
:1012A000020001000000E00001003A00E65B0700D8
:1012B0003400F9004F03BE004F02BE004F01BE00D4
:1012C0004F00BE003600F900004006003600F8006E
:1012D000809FBE00829FBE00849FBE00869FBE008E
:1012E0003400F80000002000A001880087A0A900B9
:1012F00091B48000F0072000808F50000400360079
:1013000060792100E15B070060792100030037006C
:1013100060812100DD5B07006081210038500700FB
:101320003400F9004F03BE004F02BE004F01BE0063
:101330004F00BE003600F900004006003600F800FD
:10134000809FBE00829FBE00849FBE00869FBE001D
:101350003400F80000002000A00188000000EB002D
:1013600051F18000010001008460A9003400F900FF
:101370004F03BE004F02BE004F01BE004F00BE0033
:101380003600F900004006003600F800809FBE00DD
:10139000829FBE00849FBE00869FBE003400F8007E
:1013A00000002000A001880084E0A90010002000B7
:1013B00071F18000010001003400F9004F03BE000C
:1013C0004F02BE004F01BE004F00BE003600F900C4
:1013D000004006003600F800809FBE00829FBE00DD
:1013E000849FBE00869FBE003400F80000002000ED
:1013F000A00188008500A90080F1800066006000DF
:10140000E60F500003003A009000200071F18000C8
:10141000020037002000200091F18000010001004F
:101420003400F9004F03BE004F02BE004F01BE0062
:101430004F00BE003600F900004006003600F800FC
:10144000809FBE00829FBE00849FBE00869FBE001C
:101450003400F80000002000A00188008760A90087
:1014600030002000B1F18000010001003400F900DB
:101470004F03BE004F02BE004F01BE004F00BE0032
:101480003600F900004006003600F800809FBE00DC
:10149000829FBE00849FBE00869FBE003400F8007D
:1014A00000002000A00188008780A900C0F1800012
:1014B00066006000E60F500003003A00A000200024
:1014C000B1F180000200370040002000D1F180001F
:1014D000010001003400F9004F03BE004F02BE00BE
:1014E0004F01BE004F00BE003600F900004006006C
:1014F0003600F800809FBE00829FBE00849FBE0021
:10150000869FBE00889FBE008A1F78003400F800C6
:1015100000002000A00188000200FA000082800084
:10152000E10F500008003A0094C4BF000068A30017
:1015300005003A008AA4EF008C04A8008C84A8005F
:1015400020002000008288008AC4BF000028A30079
:101550000C00320082C4BF000048A3000900320022
:1015600008012000082488008430EF000001EB000F
:101570008000EB0040072000CE5E07008284A900B7
:101580000824880088C4BF000018A300D4023A00D1
:101590008AC4BF000008A300090032008CC4BF0049
:1015A0000008A30006003200051107009EC0A80035
:1015B0004000200000828800100020005024880095
:1015C0008AC4BF000048A3000D0032008CC4BF00D5
:1015D0000048A3000A0032008284A800080120000D
:1015E0005824880010002000208488000001EB00AF
:1015F0008000EB0050072000AE5E070058248800F2
:101600008AC4BF000028A3000F0032008CC4BF00B2
:101610000028A30004003200120020008000EB002C
:1016200030072000A35E07004000200050248800FF
:101630008650E200010032008670ED008650E20024
:1016400001003A00251107008A44E20014003D0021
:101650008C44E20012003D00AAC4BF000018A300A1
:101660000D003200328280009240900000C8B3002A
:1016700080CF500007003A008082800090409000A8
:1016800040C8B30080CF500002003A0068404000DC
:1016900010419800AA24A9000008200050248800C6
:1016A0008AC4BF000018A3000A0032008CC4BF0027
:1016B0000018A30007003200120020008000EB0099
:1016C000F0FF27007B5E07008EA4EF0020002000C3
:1016D0005024880000828000E30F50008002360012
:1016E0008CC4BF000038A3007D0232000045EB002F
:1016F0008AC4BF000038A300790232009024800021
:101700006CF0B7006CD0BF000080FB004400DE002E
:101710006AF0B70080002000502488006CD0BF0021
:101720000038A30004003A006AD0BF000080FB002C
:1017300021072100030037006AD0BF000080FB00B2
:10174000E10621000100400010417800E140610005
:101750000104A2001004A10010C870006A50E20049
:1017600058023A00D0C2B30086F0B7006CD0BF0078
:1017700080017800B30FB20015023A006CD0BF00B0
:10178000C00FB20001002100010140003282880038
:10179000428288004850AA0012409000C043B20024
:1017A00041C3B300814F50009A013A008200780093
:1017B000020321001100900010F179001100900047
:1017C0000000E800900098008301E800E88F5100D5
:1017D000F8FF3A00920098005670EF007630EF0064
:1017E0007C30EF007E30EF008030EF005870EF006B
:1017F00081828000114090000074A1009040980008
:101800005050AA0081828000114090000074A10015
:10181000904098005050AA004182800011409000F2
:101820000074A100904098005C70EF005E30EF0003
:101830006270EF0063D0BF006370EF0064D0BF0040
:101840006470EF0030D0BF000046B20040013A00A3
:1018500031D0BF000080FB0001002000EB0F5000E2
:10186000E08F58003A013E00006001005D00370043
:101870008900370036013700870037003401370010
:1018800006003700080037002D01370053003700ED
:101890003300370018013700210137005CF0A80041
:1018A00080002000450037000103210091407800AE
:1018B00000C8B30080CF500025013A0000CCB3002F
:1018C0005CF0B70033D0BF00E24F50000800320098
:1018D000E34F500013003200E14F50001E003A0069
:1018E00000122100D082880020012000180037005B
:1018F00032D0BF000080FB0000004000E11B21004F
:1019000060807800D0828800D082800020409000E3
:101910005EF0B700D0828000304090005FF0B700EA
:101920000B01370032D0BF00E24F50000A003E00EA
:1019300032D0BF000080FB0000004000011C2100ED
:1019400060807800D0828800D08280001080FB0008
:10195000F0828800FE0037005C70EF00FC0037006A
:101960005CF0A800AC24EF00AE24EF000000EB0018
:1019700001002100010178000019EB000019EB00C3
:101980000000E800EC0F5000FBFF3A009424A80090
:101990004470EF009424A900800021008082880018
:1019A000318288004182880032D0BF0042F0B70007
:1019B0004250E20003003A0000012000008288004B
:1019C000E300370012002000210421001000200055
:1019D000B85D070000022000F8FF37002004210056
:1019E000C90037003870EF003970EF0030D0BF0009
:1019F0007F006000E10F50000B003200E20F50004A
:101A00000B0032000000E0001B003A005CF0A80070
:101A10003810A80010848000E10F500016003A0032
:101A20003830A800140037005CF0A800120037001E
:101A30005CF0A8003450E2000500350034D0BF004F
:101A40006F00600000004000A10421000400370086
:101A500034D0BF006F00600000004000010521008D
:101A600060807800104090000028A300020032003F
:101A700010C0B30038F0B7005C50E200B4003D0085
:101A800080032100D08288005C10A80020C0B30031
:101A90005EF0B700AE00370032D0BF00E14F50001B
:101AA0000B003A0030D0BF007F40600008003A00D1
:101AB0005CF0A80031D0BF00E34F500003003A00B3
:101AC0001000200010848800010037008230EF00F1
:101AD0003250E2009E003A0030D0BF007F406000EC
:101AE000E24F50009A003A0034D0BF006F406000CF
:101AF0009700320034D0BF006F006000E20F50004A
:101B000093003C000182800000022000808F500082
:101B10008F003A005CF0A8003450E2000A00350063
:101B200034D0BF006F00600000004000A10421001D
:101B300060807800F0BF9F0034D0BF006F0060006D
:101B4000210721000900370034D0BF006F0060007A
:101B5000000040000105210060807800F0BF9F0078
:101B600034D0BF006F006000E106210060C478003F
:101B70000808A30004003A006FF997000224A100AE
:101B8000E2FF9F00030037006FF897000024A000D9
:101B9000E0FF9F003450E2000500350034D0BF0064
:101BA0006F00600000004000A10421000400370025
:101BB00034D0BF006F00600000004000010521002C
:101BC0007FB9970002B0780031D0BF00E34F5000DA
:101BD00014003A007FB897001000E0000B003D00B1
:101BE0003450E2000400350034D0BF006F006000C4
:101BF000210721000300370034D0BF006F006000D0
:101C0000E1062100010040001014A0007FB89700F9
:101C10009040900042C8B30082C07000114098000C
:101C20004B0037008F84E9006FF897000024A20072
:101C3000E0FF9F00FFB89700114090001100E00006
:101C40000B003D000074A10090409800FFB8970081
:101C5000114090000064A0009040980022002000F5
:101C6000FFB8970050002000125D07000200370007
:101C70000064A000904098001924A2000818A30056
:101C800006003A007FB9970000402800120060006B
:101C900001002800810F500013003A003450E20088
:101CA0000400350034D0BF006F0060002107210020
:101CB0000300370034D0BF006F006000E106210050
:101CC000010040001014A100FFB8970011409000DF
:101CD000B043B2009040980022002000FFB8970067
:101CE000500020001900370012409000B043B200AD
:101CF000104198001600370034D0BF000080FB0070
:101D00004104210001004000D08288005C10A8003E
:101D100010C0B3005EF0B7005CF0A8000C00370004
:101D20005CF0A80034D0BF000080FB00410421001B
:101D3000220321001241780002F0780004003700ED
:101D40000001EB008000EB0020002000D95C0700C0
:101D50000001EB008000EB0030002000D55C0700A4
:101D600094A4A9005C50E200130035006250E20028
:101D700008003D0020C0B30058F0B7007E10E2001C
:101D800001003A00A80F07007A30EF007830EF002A
:101D9000D000370081C0B300408280000148780045
:101DA000418280000003210090009800C0C8B30069
:101DB00090409800A40037003050E20006003D003B
:101DC00010C0B30058F0B7007C10E2000C003A00DD
:101DD000950F07000A00370020C0B30058F0B70085
:101DE00081C0B300408280000148780041828000B9
:101DF000000321009000980040C8B3009040980074
:101E00007A30EF007830EF007610E200B1003A004F
:101E10005E00370058D0BF00E24F50005D003A002E
:101E20001242780063D0BF000080FB004106210011
:101E300091407800C808DD00808070000480FB00BD
:101E4000810F50000400360063D0BF00410621001E
:101E500091407800004278003106210091407800DE
:101E60008180FB0064D0BF004800DD0001007000ED
:101E70008480FB0001005000310621009140780071
:101E800063F0B7004800DE00410621009140780071
:101E900064F0B7008503210010003700010621001F
:101EA000914078008180FB0061D0BF004800DD00D8
:101EB000010070008280FB0061D87A0001062100D9
:101EC0009140780060F0B7004800DE001106210064
:101ED0009140780061F0B7008301E8000341780089
:101EE00084CF5100EDFF390042828000310621008D
:101EF000914078008180FB0064D0BF004800DD0085
:101F0000010070000A00320080C0B3000049780070
:101F10004182800080032100900098003082800080
:101F2000104090000068A3004E0032004F003700C0
:101F300080C0B30000497800418280000003210086
:101F40009000980040C8B3009040980051062100CE
:101F5000914078008180FB0066D0BF004800DD0022
:101F60000100700007003200510621009140780006
:101F70008180FB0066D0BF004800DD0001007000DA
:101F80000000010062F0A9009FFF3700D30E070098
:101F9000500037008001FD0058F0B7008001FD00BF
:101FA0008010E20008003A0081C0B3004082800047
:101FB00001487800418280000003210090009800D1
:101FC000C0C8B3002A0037000384880041003700EE
:101FD0006CD0BF00B00FB200E80F50003D003A00D7
:101FE00080828000104090004600DE0061046000A6
:101FF0005050AA0000828000E80F500008003A000C
:1020000032D0BF000080FB00B02488000001200017
:102010009604E20001003A0040002000008288009F
:1020200058D0BF00E14F500013003A008003210058
:102030008182800090009800CD0E070056D0BF002E
:10204000E24F500004003A0041C8B3008082800093
:10205000114098001F003700818280000804E000D2
:1020600002003A0080CCB3000100370080C8B30002
:1020700090409800170037006250E2000F003D00CA
:1020800051062100914078008180FB0066D0BF009E
:102090004800DD00010070000700320051062100F9
:1020A000914078008180FB0066D0BF004800DD00D1
:1020B000010070000000010062F0A9005870EF00FC
:1020C000040037000001EB00C106210020072000BA
:1020D000F85B07000A45E800E44F550084FD3A002C
:1020E0008EC0A9000080FA003400F9004F05780086
:1020F0004F04BE004F03BE004F02BE004F01BE00A2
:102100004F00BE003600F900004006003600F8001F
:10211000809FBE00829FBE00849FBE00869FBE003F
:102120003400F80000002000A00188000400FA003C
:102130008620A90050F38000E10F500003003A0010
:102140000110800060F38000014878009320200097
:10215000934178008381FB0042F38000C719DE00C1
:102160008F80E9000000EB0034F3800004000100E0
:1021700080007800E0BF9F00E40F5000190032009B
:1021800006003C00E20F50001000320013003C003B
:10219000E10F50001C003A0008003700E60F500025
:1021A0001500320011003500E70F50001400320016
:1021B000E80F500014003A00190037007FB897006C
:1021C00060F388000662A800140037007FB897000B
:1021D0001080FB0010108800100037000622A800B5
:1021E0000E00370006A2A9000100370006A2A800D1
:1021F0000682A800090037000642A8000700370041
:10220000663EEF0005003700E481570042A0200041
:10221000F10F200060BF2A007F5D070051F38800A6
:102220000080FA003400F9004F03BE004F02BE00E8
:102230004F01BE004F00BE003600F900004006000E
:102240003600F800809FBE00829FBE00849FBE00C3
:10225000869FBE003400F80000002000A001880026
:102260000400FA008A40A90090F38000E10F5000BA
:1022700003003A0081108000A0F38000014878003C
:1022800093212000934178008381FB0082F380003A
:10229000C719DE008F80E9001000200074F3800071
:1022A0000400010080007800E0BF9F00E40F5000B0
:1022B0001900320006003C00E20F5000100032000E
:1022C00013003C00E10F50001C003A0008003700EA
:1022D000E60F50001500320011003500E70F5000E6
:1022E00014003200E80F500014003A0019003700C3
:1022F0007FB89700A0F388001662A800140037008A
:102300007FB897001080FB00901088001000370005
:102310001622A8000E00370016A2A90001003700FF
:1023200016A2A8001682A800090037001642A800CD
:10233000070037006E3EEF0005003700E4815700CC
:1023400042A02000E113200060BF2A00325D070098
:1023500091F388000080FA003400F9004F03BE00BA
:102360004F02BE004F01BE004F00BE003600F90014
:10237000004006003600F800809FBE00829FBE002D
:10238000849FBE00869FBE003400F800000020003D
:10239000A00188000400FA008EA0A900D0F38000FC
:1023A000E10F500003003A0081138000E0F3800049
:1023B0000148780093272000934178008381FB0037
:1023C000C2F38000C719DE008F80E90020002000E2
:1023D000B4F380000400010080007800E0BF9F009B
:1023E000E40F50001900320006003C00E20F5000DC
:1023F0001000320013003C00E10F50001C003A00B6
:1024000008003700E60F50001500320011003500BB
:10241000E70F500014003200E80F500014003A009B
:10242000190037007FB89700E0F388007662A800B3
:10243000140037007FB897001080FB0090138800CD
:10244000100037007622A8000E00370076A2A900FF
:102450000100370076A2A8007682A80009003700A4
:102460007642A80007003700763EEF0005003700EF
:10247000E481570042A02000D117200060BF2A004D
:10248000E55C0700D1F388000080FA003400F90011
:102490004F03BE004F02BE004F01BE004F00BE0002
:1024A0003600F900004006003600F800809FBE00AC
:1024B000829FBE00849FBE00869FBE00889FBE0094
:1024C0008A1F78003400F80000002000A001880076
:1024D0008AC0A900D87EAB001F003200D75EE200A0
:1024E0000D003200D6DEEC00D6FEB700FF4F5000E4
:1024F0000200340000CEB300D6FEB700D6DEBF0027
:102500000000FB0001003B000000EA008040780072
:10251000E0C0B300614607008040EB00D75EE200F8
:1025200004003A0011C0B30010002000E85EE20091
:10253000010032000000EB008000FD00E8FEB70063
:102540008000FD000004E000030032008040EB004A
:10255000E0C0B30051460700D8BEAB00D80032003F
:1025600084C4BF00684460003B003200D45EE200D7
:102570000B003A008040EB0050C0B3004746070014
:102580008040EB0060C0B300444607008040EB0091
:1025900070C0B3004146070010C0B300D4FEB700BE
:1025A00051ED210091407800100020000104E0006E
:1025B000040032000100FB0072C0B300EA0F5000BB
:1025C00007003C0022002000811F78001100090054
:1025D0000200D80000017800CF0078000241E80036
:1025E00082C0400001007800D5FEB70040C6B300AD
:1025F00080CF500012003400D35EEC0080407800A1
:10260000D3FEB70010C0B300D5FEB700E3CF500033
:1026100001003A00D37EEF0038ED21001844780025
:102620000804E00006003A008840780070C0B3005B
:102630001A4607008840780060C0B30017460700BC
:1026400051ED210091407800D3DEBF00654040008D
:10265000124607009A003700209380006212B400EF
:10266000823E20000280B900A2F82000809FBE00B8
:10267000110009004288D800800478004F00BE0095
:10268000D45EE2002100320008007800D4FEB700DA
:1026900050182000808F54000800360001C2B3009B
:1026A00050C0B300FD45070001C2B30060C0B300D5
:1026B000FA45070001C2B30012003700801620005F
:1026C000808F54000500360001C2B30050C0B30033
:1026D000F245070001C2B300070037004015200093
:1026E000808F54000900360001C2B30050C0B3000F
:1026F000EA4507008840780060C0B300E74507005E
:102700008840780070C0B300E44507008040EB00CB
:1027100050182000808F54000400360011C0B30010
:1027200010002000E75EE200010032000000EB0034
:102730008000FD00E7FEB7008000FD000004E0001F
:102740000900320001C2B30050C0B300D3450700F6
:1027500001C2B30060C0B300D045070001C2B3009E
:1027600070C0B300CD4507008040EB0070E92F003A
:1027700000804400F70F500004003E0011C0B30079
:1027800010002000E65EE200010032000000EB00D5
:102790008000FD00E6FEB7008000FD000004E000C0
:1027A0000900320001C2B30050C0B300BB450700AE
:1027B00001C2B30060C0B300B84507008040EB0021
:1027C00070C0B300B54507008040EB00B0EA2F00B1
:1027D00000804400EE0F500004003E0011C0B30022
:1027E00010002000E55EE200010032000000EB0076
:1027F0008000FD00E5FEB7008000FD000004E00061
:102800000900320001C2B30050C0B300A345070065
:102810008040EB0060C0B300A04507008040EB00A3
:1028200070C0B3009D4507008040EB0040152000BC
:10283000808F540004003E0011C0B300100020003F
:10284000E45EE200010032000000EB008000FD00C9
:10285000E4FEB7008000FD000004E0000600320046
:102860008040EB0060C0B3008C4507008040EB0067
:1028700070C0B3008945070040152000808F5400C8
:102880000F003E00D55EEC00D5FEB700E34F5000D0
:1028900003003A0001C2B30050C0B3007F450700F7
:1028A00050ED210051C0B30090CF1000040034005F
:1028B0008040EB0050C0B30078450700D57EEF00A4
:1028C000D83EAB008A003200F3FA2000E1EC210090
:1028D00044FB20001304E00008003200114178009E
:1028E000634041008048780002C2B300824F50002C
:1028F0000300360082487800010037008048EB0072
:102900008301E8008100E800848F5100F1FF3A0064
:10291000D05EE2000A0032000802200001ED210032
:1029200091407800084078005C4507000804E80002
:1029300040022000800F540019003200F7FF3700DA
:10294000E1EC2100914078000104E0000200320037
:1029500010C2B30051450700F1EC2100914078000E
:102960000104E0000200320020C2B3004B45070022
:1029700011ED2100914078000104E00002003200D6
:1029800000C2B3004545070021ED210091407800C9
:102990000104E0000200320030C2B3003F450700EE
:1029A000CE5EE20003003A0010002000D05EE2009C
:1029B000010032000000EB00804078000004E000DD
:1029C0000300320010002000E35EE200010032004C
:1029D0000000EB008000FD00E3FEB7008000FD007A
:1029E0000004E000030032008040EB0010C2B3009E
:1029F0002A450700CF5EE20003003A0010002000E5
:102A0000D05EE200010032000000EB008040780060
:102A10000004E0000300320010002000E25EE2004B
:102A2000010032000000EB008000FD00E2FEB70074
:102A30008000FD000004E000030032008040EB0055
:102A400020C2B30015450700D15EE20003003A0042
:102A500010002000D05EE200010032000000EB0018
:102A6000804078000004E0000300320010002000E5
:102A7000E15EE200010032000000EB008000FD009A
:102A8000E1FEB7008000FD000004E000030032001A
:102A90008040EB0000C2B30000450700D25EE200B8
:102AA00003003A0010002000D05EE2000100320076
:102AB0000000EB00804078000004E00003003200DA
:102AC00010002000E05EE200010032000000EB0098
:102AD0008000FD00E0FEB7008000FD000004E00083
:102AE000030032008040EB0030C2B300EB4407002B
:102AF000D81EAB003C003200AFCFBF000400320054
:102B000010C0B30011002000DF5EE20001003200BF
:102B10008000EB00DFFEB7000104E000020032009D
:102B200020002000CD510700B0CFBF0004003200CC
:102B300010C0B30011002000DE5EE2000100320090
:102B40008000EB00DEFEB7000104E000020032006E
:102B500020002000C1510700B1CFBF0004003200A7
:102B600010C0B30011002000DD5EE2000100320061
:102B70008000EB00DDFEB7000104E000020032003F
:102B800030002000B5510700B2CFBF000400320072
:102B900010C0B30011002000DC5EE2000100320032
:102BA0008000EB00DCFEB7000104E0000200320010
:102BB00020002000A9510700B3CFBF00040032005D
:102BC00010C0B30011002000DB5EE2000100320003
:102BD0008000EB00DBFEB7000104E00002003200E1
:102BE000200020009D510700D85EAB00530032004A
:102BF00081E121004324210062E0210064E2210000
:102C000013007800910F100001003D00800878004B
:102C10000000E00003003200920F100001003400B9
:102C2000000978008180E8008381E8000281E800E3
:102C3000848F5000F2FF3A00A2252100A3E2210078
:102C400012007800910F100001003D00800878000C
:102C50008180E8000281E800838F5000F8FF3A008D
:102C60008004EB000905780060E02100EA007800AC
:102C7000402421006A0078000101500080E1210019
:102C80006A007800810150000200E00001003D0070
:102C90000001EB00000220000090B900809FBE0000
:102CA000110009004308D800000478004F00BE005E
:102CB000C0DF210069407800884078007744070031
:102CC000E28F540003003A00FE5DEC00884078007B
:102CD000724407008904E8000A85E800E78F540081
:102CE000E1FF3A00A825210069E221003AE0210035
:102CF00019017800180078000000E00001003D0094
:102D00000000EB00010220000180B900811F780063
:102D1000110009004208D800CF00780080407800F8
:102D20003A4078005D4407000884E8008984E800A0
:102D3000E0252100800F5400EDFF3A00D8DEAB0003
:102D4000160032008040EB00BC5EE20004003A0056
:102D500011C0B30010002000DA5EE2000100320072
:102D60000000EB008000FD00DAFEB7008000FD00EF
:102D70000004E000030032008040EB00D0C1B3004B
:102D800046440700BC5EE20004003200BC7EEF0057
:102D900001C2B300D0C1B30040440700D91EAB004C
:102DA0004B003200B0938000F40F500042003C0012
:102DB000A1938000909380001D2E07002200200028
:102DC000110009000200D8008000FD00067D2000EF
:102DD00006804000F3F92000C9012000830F500055
:102DE000200036000577210005804000B901200051
:102DF000830F50001B003600047122000480400045
:102E0000A9012000830F500016003600006B23003C
:102E10000081400099012000830F5100110036000D
:102E200089012000F0D52600800F51000D003E00E2
:102E300006805000EC844400830F500009003600E7
:102E4000058050008904E800830F5000050036001B
:102E500004805000F9012000830F5000010036006B
:102E60008084EB00B09380000000E00001003D0092
:102E70000000EA00800040008002200001045000B1
:102E800001003B000004EB000900E00008003500F1
:102E900060F680000000E000020035008040EB009A
:102EA000FE4307008840780009407800FB43070094
:102EB00069F688000600370060F680000000E00038
:102EC000020035008040EB00F4430700CCBEEF0069
:102ED000D93EAB0024003200CB5EEC00CBFEB70045
:102EE000EA4F500020003A00CB7EEF00C1938000F3
:102EF00050092000808F500005003C008040EB000E
:102F000060C2B300E543070001C2B30014003700FC
:102F100080112000808F50000500340001C2B300F2
:102F20006E404000DD4307008040EB000C0037009E
:102F3000A8F62F00088440004544DD002208200048
:102F4000110009000204D8000004780088407800CD
:102F500060C2B300D143070001C2B30088C0500073
:102F600070C2B300CD430700D95EAB000100320050
:102F700065230700D97EAB0001003200E23C070068
:102F80003400F9004F0578004F04BE004F03BE0027
:102F90004F02BE004F01BE004F00BE003600F900D8
:102FA000004006006D610000746800002E72000091
:102FB000616E000064000000666900006C6C000037
:102FC000206100007272000061790000207700002B
:102FD0006974000068200000726100006E640000E7
:102FE0006F6D000020760000616C000075650000C8
:102FF00073000000646500007374000000000000AE
:10300000D2970000DC970000FFFF0000FA97000055
:1030100000000000000000006D6100007468000006
:103020002E6E00007A7300006571000000770000CA
:103030007269000074650000207400006F200000B9
:10304000646500007374000020740000686500006F
:10305000206D000069640000646C000065200000C1
:10306000696E000064650000782000006F66000053
:103070002074000068650000206C00006172000090
:103080006765000073740000207300006571000024
:10309000756500006E630000652000006F6600002B
:1030A000206E00006F6E00002D7A00006572000037
:1030B0006F200000656C0000656D0000656E00000B
:1030C0007473000020660000726F00006D20000025
:1030D00073720000632C0000202D000031200000DE
:1030E00069660000206E00006F740000206600001A
:1030F0006F7500006E640000206F000072200000F9
:1031000069660000207300006D6100006C6C0000B7
:103110006572000020740000686100006E200000ED
:103120006D6900006E4C0000656E00006774000061
:103130006800000073720000630000006D69000009
:103140006E4C0000656E00006774000068000000AF
:103150000C9800001798000001000000FA9700008A
:10316000FFFF00009A980000010000009E980000F8
:1031700000000000000000006D61000074680000A5
:103180002E73000071720000740000007065000072
:10319000726600006F7200006D7300002064000012
:1031A00065730000742000003D2000007371000072
:1031B000727400002878000029200000656C00006F
:1031C000656D0000656E00007420000062790000EB
:1031D000206500006C6500006D6500006E740000E5
:1031E0000078000000000000BC980000C6980000B5
:1031F000FFFF0000FA970000FFFF0000F1980000B9
:1032000000000000000000006D6100007468000014
:103210002E7200006F74000032000000726F000018
:1032200074610000746500007320000076200000C7
:103230006F660000206100006E6700006C65000092
:1032400020610000207400006F2000006465000011
:1032500073740000007600000061000000000000B0
:10326000049900000E99000002000000FA97000087
:10327000020000002B990000010000002D990000C1
:1032800000000000000000006D6100007468000094
:103290002E6300006F730000007000006572000074
:1032A000666F0000726D000073200000646500000E
:1032B00073740000203D0000206300006F73000065
:1032C0002878000029200000656C0000656D000072
:1032D000656E000074200000627900002065000027
:1032E0006C6500006D6500006E7400000000000059
:1032F000449900004D990000FFFF0000FA9700007C
:10330000FFFF0000F1980000000000000000000036
:103310006D610000746800002E730000696E00008B
:103320000070000065720000666F0000726D0000A2
:10333000732000006465000073740000203D0000ED
:1033400020730000696E000028780000292000002A
:10335000656C0000656D0000656E00007420000063
:1033600062790000206500006C6500006D6500005A
:103370006E74000000000000889900009199000020
:10338000FFFF0000FA970000FFFF0000F198000027
:1033900000000000000000006D6100007468000083
:1033A0002E610000746100006E32000000700000A9
:1033B00065720000666F0000726D000073200000EF
:1033C0006465000073740000203D0000206100006F
:1033D000746100006E320000287900002C78000033
:1033E00029200000656C0000656D0000656E00001E
:1033F0007420000062790000206500006C65000008
:103400006D6500006E74000000790000000000008F
:10341000CC990000D7990000FFFF0000FA97000048
:10342000FFFF0000059A0000FFFF0000F198000078
:1034300000000000000000006D61000074680000E2
:103440002E6D0000756C00006469000076000000BD
:1034500070650000726600006F7200006D730000FE
:103460002064000065730000742000003D2000000F
:10347000286100002A620000292F0000632000005C
:10348000696E0000203300003220000062690000F5
:1034900074730000206500006C6500006D6500001D
:1034A0006E7400002062000079200000656C00004E
:1034B000656D0000656E0000740000006200000091
:1034C000630000001C9A0000289A0000FFFF000023
:1034D000FA970000FFFF00002D990000FFFF000099
:1034E0005E9A0000FFFF0000609A000000000000EC
:1034F000000000006D610000746800002E73000081
:103500006F72000074000000736F0000727400009E
:1035100020610000727200006179000020690000E3
:103520006E200000706C0000616300006500000008
:103530006172000072610000790000007A9A000058
:10354000849A0000FFFF0000989A0000000000002D
:10355000000000006D610000746800002E61000032
:1035600072670000626F0000756E000064730000F7
:1035700000670000657400002074000068650000AA
:10358000206900006E64000069630000657300003C
:103590002028000061720000676D0000696E000065
:1035A0002C20000061720000676D0000617800004F
:1035B000292000006F66000020740000686500008C
:1035C000202800006D6900006E6900006D75000024
:1035D0006D2C0000206D000061780000696D000016
:1035E000756D000029200000766100006C750000F8
:1035F00065730000206F00006620000073720000F9
:103600006300000061720000676D0000696E0000D9
:1036100000610000726700006D610000780000002A
:10362000AA9A0000B99A0000FFFF00009A980000D3
:1036300001000000029B000001000000099B000047
:1036400000000000000000006D61000074680000D0
:103650002E730000746100007400000070650000AB
:10366000726600006F7200006D730000207300002E
:1036700074610000746900007374000069630000E5
:10368000732000006F6E0000207300007263000062
:10369000006D0000696E0000006D000061780000A0
:1036A000006D0000656100006E000000249B0000BA
:1036B0002E9B0000FFFF00009A9800000100000010
:1036C000499B0000010000004D9B0000010000002C
:1036D000519B000000000000000000006D61000030
:1036E000746800002E6400006F7400000077000012
:1036F00072690000746500007320000074680000A7
:1037000065200000646F00007420000070720000EB
:103710006F64000075630000742000006F66000095
:10372000207300007263000031200000616E000011
:1037300064200000737200006332000020740000F7
:103740006F20000064650000737400002C200000EE
:1037500061660000746500007220000061200000B6
:103760007368000069660000740000007372000056
:10377000633100000073000072630000320000003B
:103780007368000069660000740000006E9B000012
:10379000779B000001000000FA970000FFFF000087
:1037A000B69B0000FFFF0000BB9B00000100000073
:1037B000C09B000000000000000000006D610000E0
:1037C000746800002E6D0000617800000077000032
:1037D00072690000746500007320000074680000C6
:1037E000652000006D610000786900006D750000C3
:1037F0006D2000006F6600002073000072630000FF
:1038000031200000616E000064200000737200002F
:1038100063320000207400006F2000006465000027
:10382000737400002C200000656C0000656D0000C2
:10383000656E0000742000006279000020650000C1
:103840006C6500006D6500006E74000000000000F3
:10385000DE9B0000E79B0000FFFF0000FA970000DE
:10386000FFFF0000B69B0000FFFF0000BB9B0000B5
:1038700000000000000000006D610000746800009E
:103880002E6D0000696E0000007700007269000074
:10389000746500007320000074680000652000005B
:1038A0006D6900006E6900006D7500006D200000FC
:1038B0006F6600002073000072630000312000007A
:1038C000616E00006420000073720000633200002B
:1038D000207400006F200000646500007374000015
:1038E0002C200000656C0000656D0000656E000016
:1038F0007420000062790000206500006C65000003
:103900006D6500006E740000000000003C9C00002B
:10391000459C0000FFFF0000FA970000FFFF000039
:10392000B69B0000FFFF0000BB9B000000000000F2
:10393000000000006D610000746800002E6400004B
:103940006976000000640000697600006964000088
:1039500065730000207300007263000031200000D6
:1039600062790000207300007263000032200000C2
:10397000746F00002064000065730000742C000068
:10398000206500006C6500006D6500006E7400002D
:103990002062000079200000656C0000656D000069
:1039A000656E0000740000009A9C0000A39C00005B
:1039B000FFFF0000FA970000FFFF0000B69B000029
:1039C000FFFF0000BB9B00000000000000000000A3
:1039D0006D610000746800002E6D0000756C0000C1
:1039E000006D0000756C000074690000706C0000D0
:1039F00069650000732000007372000063310000ED
:103A0000206100006E6400002073000072630000FB
:103A100032200000746F0000206400006573000015
:103A2000742C0000206500006C6500006D650000CE
:103A30006E7400002062000079200000656C0000B8
:103A4000656D0000656E000074000000E89C0000D9
:103A5000F19C0000FFFF0000FA970000FFFF00004C
:103A6000B69B0000FFFF0000BB9B000000000000B1
:103A7000000000006D610000746800002E730000FB
:103A8000756200000073000075620000737400002E
:103A90007261000063740000732000007372000004
:103AA0006332000020660000726F00006D2000008D
:103AB0007372000063310000207400006F2000006A
:103AC00064650000737400002C200000656C000029
:103AD000656D0000656E00007420000062790000D2
:103AE000206500006C6500006D6500006E740000CC
:103AF000000000003A9D0000439D0000FFFF000011
:103B0000FA970000FFFF0000B69B0000FFFF0000D7
:103B1000BB9B000000000000000000006D61000081
:103B2000746800002E610000646400000061000001
:103B300064640000732000007372000063310000B1
:103B4000206100006E6400002073000072630000BA
:103B500032200000746F00002064000065730000D4
:103B6000742C0000206500006C6500006D6500008D
:103B70006E7400002062000079200000656C000077
:103B8000656D0000656E0000740000008E9D0000F1
:103B9000979D0000FFFF0000FA970000FFFF000064
:103BA000B69B0000FFFF0000BB9B00000000000070
:103BB000000000006D610000746800002E610000CC
:103BC0006464000073630000616C000061720000B7
:103BD0000061000064640000207300006361000065
:103BE0006C61000072200000746F0000206500000E
:103BF0006163000068200000656C0000656D0000D6
:103C0000656E0000742000006F66000020730000E5
:103C100072630000206100006E64000020730000E9
:103C2000746F000072650000207200006573000070
:103C3000756C000074200000746F000020640000A8
:103C4000657300007400000073630000616C000085
:103C50006172000000000000DA9D0000E99D000094
:103C6000FFFF0000FA970000FFFF00009A98000095
:103C700001000000249E0000000000000000000081
:103C80006D610000746800002E660000696C000021
:103C90006C000000666900006C6C0000732000007E
:103CA00064650000737400002077000069740000F0
:103CB00068200000636F00006E73000074610000F4
:103CC0006E74000020760000616C000075650000D5
:103CD00000760000616C00007565000000000000C7
:103CE000409E00004A9E0000FFFF0000FA9700007F
:103CF00001000000699E00000000000000000000BC
:103D00006D610000746800002E6300006F70000099
:103D100079000000636F00007069000065730000A7
:103D20002073000072630000207400006F20000008
:103D30006465000073740000206500006C6500007D
:103D40006D6500006E7400002062000079200000A4
:103D5000656C0000656D0000656E00007400000079
:103D6000809E00008A9E0000FFFF0000FA9700007E
:103D7000FFFF00009A980000000000000000000013
:103D8000000000009301000024030000B7040000BD
:103D900048060000DA0700006B090000FC0A00007A
:103DA0008C0C00001C0E0000AB0F00003B1100004B
:103DB000C812000056140000E31500006E17000042
:103DC000F9180000831A00000C1C0000941D00006C
:103DD0001A1F0000A020000024220000A7230000DA
:103DE00029250000A826000027280000A42900009B
:103DF000202B0000992C0000122E0000872F0000BD
:103E0000FC3000006F320000DF3300004E35000050
:103E1000BA360000253800008D390000F33A000062
:103E2000573C0000B93D0000173F000074400000FF
:103E3000CE410000264300007B440000CD45000039
:103E40001D4700006A480000B4490000FC4A000019
:103E5000404C0000824D0000C04E0000FC4F0000AE
:103E600034510000695200009B530000CA54000006
:103E7000F65500001E57000043580000645900002A
:103E8000835A00009D5B0000B45C0000C85D000028
:103E9000D75E0000E45F0000EC600000F16100000C
:103EA000F2620000EF630000E9640000DE650000DC
:103EB000D0660000BD670000A76800008C690000A4
:103EC0006E6A00004B6B0000246C0000F96C00006F
:103ED000CA6D0000976E00005F6F00002370000045
:103EE000E37000009E71000055720000087300002E
:103EF000B67300006074000005750000A575000031
:103F000042760000D97600006C770000FB77000055
:103F100084780000097900008A790000067A0000A0
:103F20007D7A0000EF7A00005D7B0000C67B000018
:103F30002A7C0000897C0000E47C0000397D0000C0
:103F40008A7D0000D77D00001D7E0000607E00009D
:103F50009D7E0000D67E0000097F0000397F0000B2
:103F6000627F0000877F0000A77F0000C27F000003
:103F7000D87F0000EA7F0000F67F0000FE7F00008F
:103F8000FF7F00008C020000DF0200003003000011
:103F900080030000D103000022040000730400002D
:103FA000C204000014050000B30500005406000020
:103FB000F10600008F0700002D080000CA0800006D
:103FC00063090000FC090000340B00005C0C0000D9
:103FD000820D0000A40E0000BD0F0000D3100000F1
:103FE000E2110000E7120000EF140000CC16000000
:103FF00092180000401A0000D61B0000531D00005C
:10400000B51E00000B200000792200008D24000066
:104010006F2600001428000090290000E02A00000C
:10402000112C0000252D0000052F00008930000014
:10403000D3310000EC320000DD330000AE3400006C
:10404000673500000D36000020370000FB37000008
:10405000B23800004A390000CC3900003B3A000079
:104060009B3A0000F33A0000833B0000F43B000061
:10407000513C00009F3C0000E13C00001A3D000064
:104080004B3D0000783D0000C03D0000F93D0000C0
:10409000283E00004F3E0000703E00008D3E0000B4
:1040A000A53E0000BC3E0000E03E0000FD3E0000DA
:1040B000143F0000283F0000383F0000473F000049
:1040C000533F00005E3F0000703F00007F3F000054
:1040D0008A3F0000943F00009C3F0000A43F000086
:1040E000AA3F0000AF3F0000B83F0000C03F000003
:1040F000C53F0000CB3F0000CE3F0000D23F000094
:10410000D53F0000D83F0000DC3F0000E03F00004A
:10411000E33F0000E53F0000E83F0000E93F00000A
:10412000EB3F0000EC3F0000EE3F0000F13F0000DD
:10413000F13F0000F33F0000F43F0000F53F0000B6
:10414000F53F0000F73F0000F73F0000F93F000097
:10415000F83F0000FA3F0000FA3F0000FA3F00007D
:10416000FB3F0000FB3F0000FC3F0000FC3F000065
:10417000FC3F0000FE3F0000FD3F0000FD3F00004F
:10418000FD3F0000FE3F0000FE3F0000FE3F00003C
:10419000FE3F0000FE3F0000FE3F00000040000028
:1041A000FF3F0000FF3F0000FF3F0000FF3F000017
:1041B000FF3F0000FF3F0000FF3F0000FF3F000007
:1041C000FF3F0000FF3F0000FF3F000000400000F5
:1041D00000400000004000000040000000400000DF
:1041E00000400000004000000040000000400000CF
:1041F00000400000004000000040000000400000BF
:10420000004000000040000074680000796D00006C
:10421000696F00002D490000490000005F6900003F
:104220006400000065760000656E0000742E0000DA
:10423000736F000075720000636500000065000088
:10424000766500006E7400002E6100007267000049
:10425000730000005F660000777600006572000062
:10426000736900006F6E0000005F00007072000054
:104270006F64000075630000744900006400000072
:1042800062750000747400006F6E0000732E0000F1
:104290005F7200006177000000620000757400002A
:1042A000746F00006E2E000062610000636B0000FE
:1042B0007761000072640000006200007574000005
:1042C000746F00006E2E00006C65000066740000C4
:1042D0000062000075740000746F00006E2E000014
:1042E000636500006E7400006572000000620000EB
:1042F00075740000746F00006E2E0000666F000081
:1043000072770000617200006400000062750000B6
:10431000747400006F6E00002E7200006967000068
:10432000687400000062000075740000746F000083
:104330006E7300002E5F00006D650000616E00006E
:104340000062000075740000746F00006E7300005E
:104350002E5F00006E6F00006973000065000000B2
:10436000707200006F7800002E6800006F7200000D
:10437000697A00006F6E0000746100006C0000003C
:10438000707200006F7800002E670000726F0000EE
:10439000756E0000642E0000616D0000626900000F
:1043A000616E000074000000707200006F78000001
:1043B0002E670000726F0000756E0000642E000012
:1043C00072650000666C00006563000074650000A3
:1043D00064000000707200006F7800002E6700001B
:1043E000726F0000756E0000642E000064650000AE
:1043F0006C740000610000006D6F0000746F0000BD
:10440000722E00006C650000667400002E740000BF
:104410006172000067650000740000006D6F0000AD
:10442000746F0000722E000072690000676800005F
:10443000742E000074610000726700006574000053
:10444000005F00007662000061740000005F000001
:10445000696D00006F740000006D00006F74000053
:104460006F7200002E6C000065660000742E000064
:104470007370000065650000640000006D6F00004F
:10448000746F0000722E00007269000067680000FF
:10449000742E000073700000656500006400000069
:1044A0006D6F0000746F0000722E00006C650000DC
:1044B000667400002E700000776D0000006D000033
:1044C0006F7400006F7200002E72000069670000B8
:1044D000687400002E700000776D0000006100001D
:1044E0006363000000740000656D000070650000EB
:1044F00072610000747500007265000000720000B7
:10450000633500002E6100006464000072650000E5
:104510007373000000720000633500002E6300001A
:104520006F6D00006D6100006E640000006D0000A2
:10453000696300002E6900006E740000656E000063
:104540007369000074790000006D00006963000069
:104550002E7400006872000065730000686F000030
:104560006C640000006D0000696300002E5F0000B5
:104570006D650000616E000000740000696D000050
:10458000657200002E70000065720000696F000007
:104590006400000061630000632E00005F7400008F
:1045A000617000000000000004A100000100000094
:1045B0000EA100000100000012A100002000000078
:1045C0001FA10000020000002AA10000010000005D
:1045D00035A100000500000040A10000010000001E
:1045E0004DA10000010000005DA1000001000000DD
:1045F00069A100000100000077A100000100000097
:1046000086A100000500000093A100000500000045
:10461000A1A1000007000000B0A1000002000000FE
:10462000C0A1000002000000D4A1000002000000B0
:10463000EAA1000001000000FCA100000100000050
:104640000EA200000200000021A2000002000000F3
:1046500027A20000010000002DA2000001000000C0
:104660003EA200000100000050A200000100000076
:104670005FA20000030000006FA200000100000024
:1046800073A20000010000007FA2000001000000F2
:104690008BA200000100000097A2000001000000B2
:1046A000A5A2000001000000B3A20000020000006B
:1046B000BDA2000001000000CAA20000000000002E
:1046C00000000000DE000000AD000000CA00000095
:1046D000FE000000BE000000EF000000040000002B
:1046E000020000005F730000797300007465000031
:1046F0006D2E00007365000074740000696E000088
:10470000677300002E6600006C6100007368000093
:1047100000570000726900007465000020740000FA
:104720006865000020730000657400007469000073
:104730006E67000073200000696E0000746F000057
:10474000206600006C61000073680000005F0000DC
:104750007379000073740000656D00002E73000013
:1047600065740000746900006E670000732E00001D
:104770007772000069740000650000005772000045
:10478000697400006520000061200000736500006E
:1047900074740000696E000067000000616400002E
:1047A0006472000065730000730000007661000011
:1047B0006C750000650000005F73000079730000F5
:1047C000746500006D2E00007365000074740000B5
:1047D000696E0000677300002E72000065610000C2
:1047E0006400000052650000616400002061000068
:1047F0002073000065740000746900006E6700009B
:10480000005F00007379000073740000656D0000A4
:104810002E720000656200006F6F000074000000DF
:1048200052650000626F00006F7400002074000089
:1048300068650000206D000069630000726F000071
:10484000636F00006E740000726F00006C6C0000FB
:104850006572000000420000616300006B77000099
:104860006172000064200000627500007474000032
:104870006F6E00002073000074610000747500000A
:104880007320000063680000616E0000676500002F
:10489000640000004C6500006674000020620000A7
:1048A00075740000746F00006E20000073740000C7
:1048B00061740000757300002063000068610000EF
:1048C0006E6700006564000000430000656E000034
:1048D00074650000722000006275000074740000AE
:1048E0006F6E00002073000074610000747500009A
:1048F0007320000063680000616E000067650000BF
:1049000064000000466F00007277000061720000D2
:104910006420000062750000747400006F6E000077
:1049200020730000746100007475000073200000A3
:1049300063680000616E00006765000064000000AD
:104940005269000067680000742000006275000072
:10495000747400006F6E000020730000746100002A
:10496000747500007320000063680000616E000031
:104970006765000064000000627500007474000048
:104980006F6E000073000000427500007474000038
:104990006F6E000073200000766100006C750000EF
:1049A00065730000207500007064000061740000F1
:1049B0006564000000700000726F00007800000065
:1049C000507200006F780000696D0000697400008B
:1049D00079200000766100006C75000065730000AE
:1049E00020750000706400006174000065640000C0
:1049F000007400006170000000410000207400009D
:104A000061700000206900007320000064650000F0
:104A100074650000637400006564000000410000DC
:104A200063630000656C0000657200006F6D00003C
:104A3000657400006572000020760000616C000063
:104A4000756500007320000075700000646100004F
:104A500074650000640000006D69000063000000E0
:104A6000466900007265000064200000776800005D
:104A7000656E0000206D000069630000726F000029
:104A8000706800006F6E000065200000696E000015
:104A9000746500006E7300006974000079200000E6
:104AA0006973000020610000626F000076650000FD
:104AB000207400006872000065730000686F0000D9
:104AC0006C640000007300006F7500006E640000ED
:104AD0002E660000696E00006973000068650000C2
:104AE0006400000046690000726500006420000058
:104AF00077680000656E00002074000068650000A3
:104B0000207000006C6100007962000061630000A9
:104B10006B2000006F66000020610000207500001F
:104B20007365000072200000696E00006974000067
:104B3000696100007465000064200000736F00006C
:104B4000756E00006420000069730000206600009C
:104B5000696E000069730000686500006400000071
:104B6000546500006D700000657200006174000003
:104B70007572000065200000766100006C75000011
:104B8000652000007570000064610000746500001D
:104B90006400000072630000350000005243000012
:104BA000352000006D650000737300006167000030
:104BB00065200000726500006365000069760000F2
:104BC00065640000006D00006F7400006F720000EB
:104BD000004D00006F7400006F7200002074000030
:104BE000696D00006572000000740000696D0000CE
:104BF0006572000030000000546900006D6500001F
:104C00007220000030000000746900006D65000033
:104C10007231000000540000696D000065720000F0
:104C200020310000000000004DA100002BA4000076
:104C30005DA100004AA4000069A1000065A4000075
:104C400077A1000082A4000086A10000A0A40000BB
:104C5000BCA40000C4A40000DBA40000E0A4000089
:104C6000F9A40000FDA400006FA200000FA5000041
:104C70002CA5000030A5000063A5000072A500006F
:104C800073A20000B0A50000CAA50000CEA50000D8
:104C9000E3A50000E9A50000F5A50000FCA50000C3
:104CA00004A600000BA600000000000000000000A9
:104CB000416400006472000065730000732000000E
:104CC0006F750000742000006F6600002073000004
:104CD00065740000746900006E67000073000000D6
:104CE000536C000065650000702000006D6F0000CF
:104CF00064650000206E00006F74000020730000E7
:104D000075700000706F0000727400006564000030
:104D100000450000727200006F7200003A2000002F
:104D20006D6900006E2000003D3D00002030000055
:104D30007846000046460000464600004646000011
:104D4000462000002100000045720000726F000044
:104D5000723A0000205500006E610000626C000095
:104D600065200000746F0000206600006C61000088
:104D70007368000020620000797400006563000021
:104D80006F64000065200000283100002920000029
:104D90002100000045720000726F0000723A0000AE
:104DA000205500006E610000626C0000652000006C
:104DB000746F0000206600006C61000073680000E2
:104DC0002062000079740000656300006F640000D9
:104DD000652000002832000029200000210000008A
:104DE00045720000726F0000723A0000205500000A
:104DF0006E610000626C000065200000746F0000AE
:104E0000206600006C6100007368000020620000F2
:104E100079740000656300006F6400006520000085
:104E2000283300002920000021000000466C00000B
:104E300061730000686900006E670000204F000089
:104E40004B000000736F0000756E0000642E0000C0
:104E50007761000076650000005300006574000073
:104E60002074000068650000207000007269000076
:104E70006D6100007279000020770000617600000B
:104E8000652000006F660000207400006865000067
:104E9000207400006F6E0000652000006765000050
:104EA0006E65000072610000746F00007200000007
:104EB0007761000076650000007300006F750000E8
:104EC0006E6400002E660000726500007100000034
:104ED000506C0000617900002066000072650000DF
:104EE00071750000656E00006379000000480000E5
:104EF0007A00000064730000006C0000656400002C
:104F0000732E0000746500006D7000006572000073
:104F100061740000757200006500000053650000B8
:104F2000742000006E740000632000006C650000B7
:104F3000640000007265000064000000626C000004
:104F400075650000006C000065640000732E0000B1
:104F5000736F0000756E0000640000005365000070
:104F600074200000736F0000756E00006420000064
:104F70006C650000640000006C65000064000000C7
:104F80006C650000647300002E7200006300000076
:104F9000536500007420000072630000206C000064
:104FA00065640000006C000065640000732E000062
:104FB000707200006F7800002E7600000053000031
:104FC00065740000207600006572000074690000BE
:104FD000636100006C200000707200006F780000B8
:104FE000696D000069740000792000006C650000A4
:104FF00064730000006C0000656400002030000055
:10500000006C00006564000020310000006C0000AE
:1050100065640000732E0000707200006F7800005D
:105020002E68000000530000657400002068000036
:105030006F720000697A00006F6E000074610000FA
:105040006C200000707200006F780000696D000035
:1050500069740000792000006C6500006473000032
:10506000006C00006564000020320000006C00004D
:105070006564000020330000006C000065640000DF
:1050800020340000006C0000656400002035000042
:10509000006C00006564000020360000006C000019
:1050A0006564000020370000006C000065640000AB
:1050B000732E000062750000747400006F6E0000B3
:1050C000730000005365000074200000627500004A
:1050D000747400006F6E0000732000006C650000A7
:1050E00064730000006C000065640000732E000013
:1050F000626F0000747400006F6D00002E6C000081
:105100006566000074000000536500007420000014
:105110005247000042200000626F0000746F0000E0
:105120006D2000006C65000066740000206C0000BB
:10513000656400000067000072650000656E000095
:10514000006C000065640000732E0000626F0000B8
:10515000747400006F6D00002E720000696700001B
:1051600068740000005300006574000020520000C5
:1051700047420000206200006F7400006F6D000065
:10518000207200006967000068740000206C000055
:1051900065640000006C000065640000732E000070
:1051A000746F000070000000536500007420000060
:1051B0005247000042200000746F00007020000081
:1051C0006C650000640000006C6500006473000002
:1051D0002E63000069720000636C0000650000002F
:1051E00053650000742000006369000072630000D2
:1051F000756C00006172000020720000696E000092
:10520000672000006C6500006473000000730000FC
:105210006F7500006E6400002E730000797300004B
:10522000746500006D00000053740000617200009E
:1052300074200000706C0000617900006261000061
:10524000636B0000206F000066200000737900008F
:1052500073740000656D0000207300006F7500001E
:105260006E640000204E0000004E0000007300003D
:105270006F7500006E6400002E7200006570000003
:105280006C6100007900000053740000617200003E
:1052900074200000706C0000617900006261000001
:1052A000636B0000206F000066200000724E00005B
:1052B0002E77000061760000007300006F7500001B
:1052C0006E6400002E7000006C6100007900000028
:1052D000537400006172000074200000706C0000C4
:1052E0006179000062610000636B0000206F0000C4
:1052F00066200000704E00002E77000061760000EE
:10530000007300006F7500006E6400002E720000D4
:10531000656300006F7200006400000053740000B9
:10532000617200007420000072650000636F00006D
:1053300072640000696E0000672000006F66000064
:10534000207200004E2E0000776100007600000001
:105350005F6C000065640000732E00007365000040
:1053600074000000536500007420000074680000A1
:10537000652000006C65000064000000627200009F
:1053800069670000687400006E65000073730000B8
:10539000007000000000000000000000000000009D
:1053A000000000000000000000000000720000008B
:1053B00000000000000000000000000000000000ED
:1053C000000000000072000000000000000000006B
:1053D00000000000000000000000000000000000CD
:1053E000730000000000000000000000000000004A
:1053F0000000000000000000004500007272000084
:105400006F7200003A200000736100006D700000B0
:105410006C650000732000006D750000737400005F
:105420002062000065200000696E0000205B000023
:105430002D310000323800002C31000032370000DE
:105440005D200000726100006E67000065000000D2
:1054500030110000070000007C150000070000006C
:10546000C819000007000000000000000000000054
:1054700030110000070000007C150000070000004C
:105480000000000000000000C81900000500000036
:10549000BE0A000004000000000000000000000040
:1054A0009C27000002000000AB2200000100000069
:1054B0009D1C000002000000FB180000020000001C
:1054C0002D32000001000000322D0000010000001C
:1054D0004628000002000000E8260000010000004D
:1054E000BF22000002000000FB18000002000000C4
:1054F000FF32000001000000C62000000100000093
:10550000762F0000020000002C2E00000100000099
:10551000CE2C000001000000FD3900000200000058
:105520000000000000000000E40C00000700000084
:10553000301100000D000000C81900000700000035
:1055400000000000000000004C0400000700000004
:1055500098080000070000000000000000000000A4
:10556000781E00000D000000001900000700000078
:10557000EC130000070000003011000007000000DD
:10558000480D0000070000000000000000000000BF
:10559000480D00000D000000301100000700000061
:1055A000EC130000070000000019000007000000D5
:1055B000781E00000700000000000000000000004E
:1055C000733000002E770000617600000073000049
:1055D000322E000077610000760000007333000077
:1055E0002E7700006176000000730000342E00006A
:1055F0007761000076000000733500002E77000010
:105600006176000000730000362E00007761000014
:1056100076000000733700002E77000061760000EE
:1056200000000000809A0000904100008E410000C0
:105630008F800000454500004549000049490000B1
:105640008E8F000090920000924F0000994F000052
:1056500055550000599900009A9B00009C9D000040
:105660009E9F0000414900004F550000A5A5000085
:10567000A6A70000A8A90000AAAB0000AC2100006A
:10568000AEAF0000B0B10000B2B30000B4B500008E
:10569000B6B70000B8B90000BABB0000BCBD00003E
:1056A000BEBF0000C0C10000C2C30000C4C50000EE
:1056B000C6C70000C8C90000CACB0000CCCD00009E
:1056C000CECF0000D0D10000D2D30000D4D500004E
:1056D000D6D70000D8D90000DADB0000DCDD0000FE
:1056E000DEDF0000E0E10000E2E30000E4E50000AE
:1056F000E6E70000E8E90000EAEB0000ECED00005E
:10570000EEEF0000F0F10000F2F30000F4F500000D
:10571000F6F70000F8F90000FAFB0000FCFD0000BD
:10572000FEFF0000222A00002B2C00003A3B000064
:105730003C3D00003E3F00005B5D00007C7F0000C0
:10574000000000005A3A00005C6D00006F6C000021
:105750006F6C0000655C000069320000635C000053
:105760002F690000326300005F7000007269000062
:10577000762E0000680000005A3A00005C6D0000C0
:105780006F6C00006F6C0000655C00006932000007
:10579000635C00006D6100007374000065720000BE
:1057A0005F700000726F0000746F0000636F000094
:1057B0006C2E0000630000005A3A00005C6D00008F
:1057C0006F6C00006F6C0000655C000069320000C7
:1057D000635C00002F690000326300005F7000000E
:1057E00072690000762E0000680000005A3A00003E
:1057F0005C6D00006F6C00006F6C0000655C000069
:1058000069320000635C00006D6100007374000089
:10581000657200002E630000000000005249000085
:105820004646000000000000000000005741000054
:1058300056450000666D0000742000001000000056
:10584000000000000100000001000000841E0000B4
:1058500000000000841E00000000000001000000A5
:105860000800000064610000746100000000000096
:10587000000000005A3A00005C6D00006F6C0000F0
:105880006F6C0000655C0000746900006D650000CD
:10589000725C0000746900006D650000722E0000EB
:1058A000630000000100000000000000080000008C
:1058B00000000000400000000000000000010000A7
:1058C000000000005F4C00004F47000044550000FE
:1058D0004D5000002E23000040210000005F00001A
:1058E00054450000535400004D4F0000442E00006A
:1058F0002340000021000000564D0000434F0000EF
:10590000444500002E410000424F0000000000000E
:105910005A3A00005C6D00006F6C00006F6C000074
:10592000655C000069320000635C00002F690000C4
:10593000326300005F70000072690000762E000084
:10594000680000005A3A00005C6D00006F6C0000B7
:105950006F6C0000655C0000666C00006173000005
:10596000685C0000666C000061730000682E000037
:10597000630000005F7000006F7700006572000038
:105980006F66000066000000506F00007765000041
:10599000726F000066660000000000006D6D000080
:1059A0006137000036360000302E00006300000032
:1059B00000000000000000000000000000000000E7
:1059C0009EC0A9008EA4EF008AA4EF00AA24EF00D5
:1059D000AC24EF00AE24EF0020002000302588002A
:1059E000A824EF008644A900F00920008024880044
:1059F000602488008804A800010021004808DE0017
:105A0000C02488000000EB008018EB008018EB0039
:105A10000000E800EC0F5000FBFF3A009424A800BF
:105A20009624EF0094A4A9009424A90081002000EA
:105A300007003700512488005C70EF006270EF00AF
:105A400063D0BF006370EF0064D0BF006470EF00EC
:105A50008AC4BF000038A300F6FF3A0010002000FF
:105A6000C0838800D08388007C30EF007E30EF0058
:105A70008430EF000000EB0004052100A2042100A7
:105A800080007800E506210023072100001AEB00C2
:105A90000019EB0001F07A0001F079000000E80045
:105AA000E30F5000F9FF3A00800021008082880057
:105AB000D0002000502588000003210010808800BD
:105AC00080C0B30000F0B70040C8B30001F0B700D9
:105AD0004270EF004030EF00000006007810E20056
:105AE00022003A0014002000C4838800D183800083
:105AF0000100E0001D003A00D483880058D0BF00A8
:105B0000E24F500006003A00808280000148780091
:105B100081CCB30080828000114098000000060014
:105B200058D0BF00E14F500010003A0001848800B7
:105B300083C0B30030828000034878003182800047
:105B4000020321009200980040C8B30090409800E2
:105B500004848800408280000348780041828000ED
:105B60009200980000C8B300904098000000060022
:105B7000F082800083C0B300E70F50000A003E00AF
:105B8000F08280008041780010C0B3005650E200DF
:105B90000400320056D0BF00E14F500002003A002E
:105BA00020C0B30056F0B7000380FB005E30B500A4
:105BB00080828000034878008003210040838800B1
:105BC0005CD0BF000008A30002003200034178004F
:105BD00012003700034178008041EB0006003700D7
:105BE00040838000D1828000315878004083880053
:105BF000D18288000241E900834F5100F8FF3A004A
:105C00000000060040838000D18280003158780077
:105C100040838800D18288000241E9000204E0004C
:105C2000F8FF3A00000006007C30EF007E30EF0005
:105C300058D0BF00E24F500009003A0081C0B300C5
:105C4000408280000148780041828000800321006A
:105C50009000980080CCB3009040980000000600AF
:105C600036D0BF000080FB00710321009140780016
:105C7000C808DD0080807000F0828000808F5000B6
:105C80000700310061032100914078008180FB0012
:105C900037D0BF004800DD0001007000F0828800AE
:105CA000B3FF07008103210080828000110098006B
:105CB00081CCB30080828000114098000000060073
:105CC0000080FB00800140000180FB00008041005B
:105CD0004300DD000200210002014000124090005C
:105CE0000074A10010419800A00421000104E0000C
:105CF000010032000005210082317800124090003E
:105D00000064A10010419800E4004100114090009F
:105D10000064A0009040980000000600889FBE002C
:105D20008A1F780000447800014578008184FB00D8
:105D30000938A300020032008040EB00E0FF0700BA
:105D40000928A3000300320011C0B3000840780006
:105D5000DBFF07000880FB0000004000A14A200094
:105D60000AF078004F0578004F04BE0000000600DE
:105D7000014178000004E0000C003A0081C0B3004B
:105D800040828000014878004182800000032100A9
:105D900090009800C0C8B3009040980041C8B3007C
:105DA0008082800011409800000006008080FB0087
:105DB000818040000280FB0080804000C308DD003D
:105DC00002002100028140001240900043C8B3004D
:105DD0000340700010419800400021008080400086
:105DE00011409000034070009040980000000600B1
:105DF000004378000082FB00814378000104E0004A
:105E00000300320084004200000521000200370038
:105E100084004200A0042100E10278000500E000B7
:105E200002003A0005007800000006000682FB0030
:105E300092029800834A7800154090000044B20016
:105E4000904298001540900081C8B3000140700056
:105E5000904298000704E000030032000400420072
:105E6000010521000200370004004200A1042100C6
:105E7000010040001024A200050078000000060088
:105E80008040780094C4BF000058A300180032007E
:105E90000181FB000201410004052100E2017A00BA
:105EA0001300BE00050420000080620001002000F5
:105EB0008089BE00E2017A00000420000100200079
:105EC0009319680093916800040141001224A20014
:105ED00092007800114090000044B2009040980079
:105EE00092007800114090000540680090409800B2
:105EF000000006000000EB00A02488006024880059
:105F00000082880000000600018280000100E0009D
:105F100011003A00A124880061248800200020009C
:105F200030258800412588008644A900F00920001A
:105F300080248800602488009EC0A80001003700EB
:105F40009404A80094C4BF000008A300FCFF320022
:105F50001000200000828800000006000001780088
:105F600083FA800050032000808F51000A00320025
:105F700063004000808F51000E0032006600500028
:105F8000808F510010003A0092928800A192880000
:105F9000E482A8000C003700B29288009092800042
:105FA00000005100D0928800E482A900DCC2A80061
:105FB00005003700C1928800A09280000080500048
:105FC000E0928800DCC2A9008300E80081FA880022
:105FD00000322000808F500001003A00503FEF0057
:105FE00000000600DCC2A900E482A900000006004F
:105FF0000000FE000040060000000000000000005D
:106000000000000000000000000000000000000090
:106010000000000000000000000000000000000080
:106020000000000000000000000000000000000070
:106030000000000000000000000000000000000060
:109000008001EB000200370061F079008301E80085
:10901000828F5100FCFF3A00000006008001EB0047
:109020000200370001F079008301E800828F5100CF
:10903000FCFF3A0000000600889FBE008A9FBE0029
:109040008C9FBE008E1F7800000478000206BE00D0
:1090500050159000E0159000820F5500838F5D0041
:1090600034003200404090000004E0002100320053
:10907000EE022000080747001840900014C0B3001B
:109080000A01BE008E007800D72107000000E00032
:1090900026003A004044980078089000881090001C
:1090A00058099000E80990000000410081804900C3
:1090B000800F5500818F5D000E003100B844900094
:1090C0000A00370058089000E80890000A054000A0
:1090D0008B8548001840900014C0B3000A01BE0000
:1090E0008E007800C02107008944E900E1CF5400D8
:1090F000F4FF3E00E00F5600E08F5E000D003200EE
:10910000E1022000888040001840900014C0B300A5
:109110000C01BE00782107000000E00003003A00C7
:109120005C1498006D1498000300370010002000B4
:10913000010037000000EB004F0778004F06BE002B
:109140004F05BE004F04BE0000000600881F7800D7
:109150000004780062025100E0825900C0089000CB
:109160003008900062005000E08058006011B800A4
:10917000800F5200818F5A00090031002841900071
:109180000281FB00030020000400BE00A6DD0700F2
:1091900038119000C8119000000141008181490000
:1091A0000200BE004F04780000000600889FBE0049
:1091B0008A9FBE00000578000204BE00E10F510046
:1091C000E08F590079003600C00890003008900008
:1091D000800F5100818F5900740031001A407800CF
:1091E000E24F50002E003200E34F500043003200A7
:1091F000E14F500070003A00820478000200D10074
:10920000000441004941DE007A0890008A10900075
:1092100002014000E08148000A00780086FF070054
:109220000000E00064003A0008007800F01FB2007F
:10923000E002B0000A0040009085FB000804E8004E
:109240004941DE007A0890008A1090000201400037
:10925000E08148000A00780077FF07000000E00086
:1092600055003A00F81FB200E0022000080040005C
:109270000A0040001080FB004800DD00808075007F
:109280000908A300020032004408DE000200370093
:10929000F0FF20000080600001002000480037003F
:1092A0004818DD004811DE0002017000C819DE0018
:1092B0007A0890008A1090000201400083814800E3
:1092C0000A0078005CFF07000000E0003A003A0066
:1092D000E20220000A0141000800440089804C009D
:1092E000F01FB20000014100124090004800DD0074
:1092F0009280FB0001007000E7FF37004918DD0095
:109300004711DE0002017000C719DE007A089000E4
:109310008A10900002014000838148000A00780012
:1093200045FF07000000E00023003A00E4022000AF
:109330000A0242004248DD00CE40DE00810070009B
:109340004240DD00F01FB2000002420034419000B4
:10935000C811DD0002002000244090008080FB0046
:109360000000200000017100818171001440900014
:109370004800DD00010020000001710081817100C2
:10938000144078000080FB00010020000001710003
:1093900081817100F0FF20000300600080037800ED
:1093A000020378000600BE00050037001000200010
:1093B00001002000020037000080EB008080EB00FD
:1093C0004F05BE004F04BE0000000600E4874700C2
:1093D000889FBE008A9FBE008C9FBE008E1F7800B3
:1093E000000578000204BE000406BE00E10F510033
:1093F000E08F59009F003600C008900030089000B0
:10940000800F5100818F59009A0031001A40780076
:10941000E24F500044003200E34F50005900320048
:109420002B002000E14F50008F003A000200D100D5
:10943000800441004949DE007A0890008A109000BB
:1094400002014000E08148000A007800FAFE0700AF
:10945000800578000000E00083003A00EE02200062
:109460000A07470009007800F01FB200000147001A
:10947000610064000100200080BF9F000000E00048
:109480000500320012427800EF4062004460DD00C7
:1094900001407000010037000C407800004978005E
:1094A0000904E80010C0B300404598004941DE00BF
:1094B0007A0890008A10900002014000E081480084
:1094C0000A007800DCFE0700800578000000E0005C
:1094D00065003A00F81FB200880147000FB89700F6
:1094E0000000E000050032004C69DD004460DE0051
:1094F00000007100C468DE000800370002CFB3002E
:1095000013416100486ADD004860DE00000072001F
:10951000C868DE006F40600000407100804978003C
:109520008005EB00500037004818DD004811DE00D0
:1095300002017000C819DE007A0890008A109000BD
:1095400002014000838148000A007800BAFE07004B
:10955000800578000000E00043003A00E0022000AF
:109560000A0040000801440089814C00F21FB2004B
:10957000020040000C487800C860DE0011409800EE
:1095800039003700491ADD004711DE000201720080
:10959000C719DE007A0890008A109000020140008E
:1095A000838148000A007800A3FE07008005780048
:1095B0000000E0002C003A00E40220000A02420011
:1095C0004248DD00CE40DE00810070004240DD00F8
:1095D000F01FB20000024200E30342000483E800EF
:1095E0008402E80017417800C811DD000200200065
:1095F000164078008080FB00000020000001710010
:10960000818171001580FB004800DD000100200011
:109610000001710081817100144078000080FB001E
:1096200001002000000171008181710000002F0005
:109630000300600001002000C000DD0000002000E9
:109640000000760081807600004A78004801DE0044
:10965000824A78004009DE0003002000024B7800B7
:109660004808DE00804B780010C0B30040459800E9
:10967000010037002B0020000B0078004F07780016
:109680004F06BE004F05BE004F04BE004F00B100A4
:10969000000006000400FA00889FBE008A9FBE00FA
:1096A0008C1F78000006780092BF9F00A3BF9F0028
:1096B000E00F5100E08F59000B003A005005900078
:1096C000E0059000E00F5500E08F5D0015003200CE
:1096D000C008900030089000800F5500818F5D0019
:1096E00010003100110037001FB99700AFB9970083
:1096F000AEFE07000001BE00E10F5000E08F5800F1
:109700004D0036003C089000CC089000800F5100BE
:10971000818F59004C0039001FBD9700AFBD9700E5
:10972000020037001A0020000B0020000A04BE00CF
:1097300061044400E0844C003C089000CC08900098
:10974000800F5400818F5C0005003900E10F550047
:10975000E08F5D003B00360028002000090020005B
:109760000801BE000C00780090FE07000001BE005A
:10977000E00F5000E08F58000A003200E10F400077
:10978000E08F480030003200E10F5000E08F5800B9
:109790002D0032008A0F54008B8F5C0029003200AC
:1097A000E3FF3700F4FF2F00F5FF20000801BE00A3
:1097B0000C00780005FF07000000E0001A003A00E6
:1097C0001FB89700AFB89700E00F5000E08F580027
:1097D000060032000802BE000001BE000C00780046
:1097E000FAFE07000000E0000F003A00580698005B
:1097F000690698007C0090008C089000E10F400002
:10980000E08F48000600320061005000E080580000
:1098100070069800010E980010C0B30050469800E2
:109820000801BE00080037000081EB008081EB00DA
:10983000E10F50000400320012002000030020005D
:10984000010037006011B8000200BE004F0678002A
:109850004F05BE004F04BE000080FA000000060065
:10986000889FBE008A1F78000004BE002104980073
:1098700030019000C0019000E10F5100E08F5900CD
:10988000480032001002780034089000C4089000AC
:10989000800F5100818F590042003100E00F5100CC
:1098A000E08F590016003A0030C0B300944F10000A
:1098B00005003A0014119000A4119000E00F51002F
:1098C000E08F59000E003A006000B8005004980084
:1098D0006104980044009000808F540031003100F2
:1098E0004448DE0014119000A411900000004100D3
:1098F000E080490070049800010C98001F003700B8
:10990000244090000080FB004405DD00100037007B
:109910001800780025FE07000001BE00E10F40009E
:10992000E08F48001D003200E10F5000E08F58002A
:109930001C00360018007800C00890003008900025
:10994000800F5100818F5900160031008A84540025
:109950008A8F5400EEFF310052049800630498008F
:1099600018007800F9FD07004449DE0002014000BC
:10997000E081480072049800030C9800E002200087
:10998000980040006F8064004500DD00808040004A
:10999000110C98000000EB000300370010002000BD
:1099A00001003700200020004F0578004F04BE0062
:1099B00000000600889FBE008A9FBE008C9FBE00EC
:1099C0008004780001047800200090000006E80080
:1099D000770032007900900089089000E00F500075
:1099E000E08F580072003200EF06660068003A000F
:1099F00061004000E0804800F0049800810C98006D
:109A00001902780059019000E9019000E00F51001F
:109A1000E08F590004003A0044009000800F560087
:109A20005B00390062003700C460DE002440900013
:109A30000080FB000000E9008080600054003A00D4
:109A400004007800D9FD07000005BE00E10F5000BA
:109A5000E08F580058003600E10F4000E08F4800CA
:109A6000570032001902780034089000C4089000B2
:109A7000800F5500818F5D003E0039000800E00036
:109A80004B00320059019000E90190000400780079
:109A900000FF07000005BE0070002000E00F550029
:109AA000E08F5D0047003200E10F5500E08F5D0060
:109AB00041003200E10F4500E08F4D0040003200D0
:109AC0006011B800190078005BFD07000000E0009D
:109AD0003B003A00E10220001980400002202000F3
:109AE0008D0078004DFD0700190478000A01BE00C2
:109AF0000800780095FD0700501498006114980044
:109B00000D0478000F00370010C0B30040429800E9
:109B10006011B8001900780047FD07000804E8004C
:109B20000000E00026003A00190178005210900071
:109B3000E210900061004000E08048005011980061
:109B4000611198001902780024409000804F540061
:109B5000EDFF39000881FB00030020005410900045
:109B6000E4109000020050008380580050129800CA
:109B700061129800DA049800EB0498000A01BE0014
:109B80001900780071FD0700F0049800810C98001E
:109B9000AC049800E102200019804000C568DD0097
:109BA00001004000900C98000000EB000500370019
:109BB0004000200003003700200020000100370093
:109BC000100020004F06BE004F05BE004F04BE002F
:109BD00000000600881F7800E8022000000444000E
:109BE0001040900014C0B30088007800C21E070027
:109BF000320020000000E0003F003A0078F89300B7
:109C00004800DD00E8F893008180FB00010070004F
:109C10002200200051A52A00810F500036003A0092
:109C200018799000C811DD0002002000087890002B
:109C30008080FB0000002000000171008181710024
:109C4000787090004800DD000100200000017100E4
:109C500081817100687090000080FB00010020008D
:109C600000017100818171000380FB008002780097
:109C7000020278000400BE0066142400470520009C
:109C8000860F5000878F58001A00320058D190007C
:109C9000C811DD000200200048D090008080FB0049
:109CA00000002000000171008181710038D0900017
:109CB0004800DD0001002000000171008181710079
:109CC00028D090000080FB000100200000017100FE
:109CD000818171000380FB0080027800020278001D
:109CE0000400BE0012002000860F5000878F58002D
:109CF00001003A000001EB00020078004F047800F8
:109D000000000600000178000000E0000C003200B6
:109D10001004E0000A00320030009000810F500073
:109D200007003A00124090006C1E070061006000BE
:109D30003100200003003A00800078000100370065
:109D4000910020000100780000000600B200200011
:109D50000004E00009003A0072FA80000200E0000E
:109D600001003200004978000100E00001003200EB
:109D70008048780071FA88000001EB00020078004A
:109D800000000600EF03B000889FBE008A9FBE005F
:109D90008C9FBE008E1F7800E0B79F0001077800FF
:109DA0000008EB007F406100C0DF9F007E4461003F
:109DB0009100FB0000FD2F0000814000E90F5100E1
:109DC00008003E009E409000A0C3B30080CF50002A
:109DD00004003A000E87E800B90020000200E0000D
:109DE000A2013A007AFA80009AA79F00C9002000D9
:109DF0000A00E0009D0132001A04E0000A0032006F
:109E00001A409000351E07000080FB000008A300E8
:109E100005003A000804E000910132000028A30088
:109E20008D013A008E0137000040EB00004D7800B4
:109E3000104598009C1D07000080FB0039002000A1
:109E40000008A30089013A000804E0000200320083
:109E50000028A30080013A006011B8000A007800D1
:109E60005CFF07006011B80092B79F00A3B79F0086
:109E7000E14F50001B003A00E40220000A024200B9
:109E800024C093000004E0007701320014C993005D
:109E9000C811DD000200200004C893008080FB0090
:109EA00000002000000171008181710074C09300E6
:109EB0004800DD0001002000000171008181710077
:109EC00064C093000080FB000100200000017100CD
:109ED0008181710092B79F00A3B79F000A007800AC
:109EE0003CFF070019002000E34F50005F013200E3
:109EF0000004E0005C013A00EB0220008A85450086
:109F00002A7890004800DD009A7890008180FB005C
:109F10000100700001202000810F500052013A0022
:109F2000DAC09000C808DD004AC090000080FB0045
:109F300080807000610AB80012003A007B619000D6
:109F4000C811DD00020020006B6090008080FB00E3
:109F50000000200000017100818171005B609000B1
:109F60004800DD00010020000001710081817100C6
:109F70004B6090000080FB00010020000002710097
:109F800081827100540D9800650D9800EA78900068
:109F9000314598000140E900E14F500032013E0098
:109FA0000181FB00030020000400BE001EDA070050
:109FB000F0B79F0081BF9F00BA7B900027459800B3
:109FC0000704E000280132000780FB008000E90060
:109FD0000100600024013A000AC090004800DD0042
:109FE000FA7890008180FB0001037000460598001C
:109FF0006F0063001C013A00AAC09000C808DD0091
:10A000001AC090000080FB0080807000610AB800D8
:10A0100012003A003B619000C811DD0002002000F0
:10A020002B6090008080FB00000020000001710088
:10A03000818171001B6090004800DD00010020005C
:10A0400000017100818171000B6090000080FB00B5
:10A05000010020000002710081827100DA78900016
:10A06000C808DD004A7890000080FB000080700086
:10A07000FD0032006104B800C8B79F00D9B79F0047
:10A080007FB197008FB9970008004100898049008F
:10A090004431DE0002044000E0844800880F520092
:10A0A000898F5A00F00039000800520089805A0058
:10A0B0000781FB0003002000E9D90700E00F5000F2
:10A0C000E08F5800E800320013C0B300E3E79F00C0
:10A0D00054FF2000840F5000E08F58000700360026
:10A0E00035C0B300E5E79F00EB0F4000E08F58005C
:10A0F00002003E0022C0B300E2E79F00620640007B
:10A10000E08648003C0D98004D0D98001FB2970066
:10A11000AFB297000400440085804C0030159800D1
:10A12000411598004FB49700DFB497000400440035
:10A1300085804C00700D9800011598004A01900030
:10A14000EFE49700E3CF54001B003A000200E00068
:10A15000C5003A007B699000C811DD0002002000B4
:10A160006B6890008080FB000000200000017100FF
:10A17000818171005B6890004800DD0001002000D3
:10A1800000017100818171004B6890000080FB002C
:10A1900001002000000171008181710012159800FA
:10A1A000231598004268DD00CE60DE00810070005B
:10A1B0004260DD00170037000200E000AA00320014
:10A1C0007FB197008FB9970000004100818049005E
:10A1D0001015980021159800EFE19700E2CF51008B
:10A1E00003003A000C0046008D804E000900370045
:10A1F00032002000030020000C00BE008AD90700B6
:10A200008100D1000080D30061016600020040009F
:10A21000E0804800F01FB0000180B000C909DE00F6
:10A22000470ADD004901DE00020172005A08900071
:10A23000EA089000820F5000838F58008A0039008E
:10A240000080EB008080EB0070059800010D980005
:10A250006000B8005005980061059800EFE2970093
:10A26000E3CF520071003A000040EB0050459800E7
:10A270001B7190004811DD000B7090000080FB0006
:10A28000000171001FB49700AFB4970002014400B1
:10A29000E0814C00120D9800230D98001A409000A8
:10A2A00014C0B3008B007800131D07000000E0000D
:10A2B0005E003A007BF893004800DD00EBF8930065
:10A2C0008180FB000100700051A52A00810F500021
:10A2D00056003A003B419000C811DD00020020000A
:10A2E0002B4090008080FB000000200000017100E6
:10A2F000818171001B4090004800DD0001002000BA
:10A3000000017100818171006A6890000080FB008B
:10A3100001002000000171008181710020252500CD
:10A3200011162400800F5100818F59003F003A0020
:10A330007BE19300C811DD00020020006BE0930078
:10A340008080FB000000200000017100818171000D
:10A350005BE093004800DD00010020000001710077
:10A36000818171004BE093000080FB000100200020
:10A37000000171008181710020272700111426003F
:10A38000800F5100818F590028003A007BE993002B
:10A39000C811DD00020020006BE893008080FB0004
:10A3A0000000200000017100818171005BE89300D2
:10A3B0004800DD0001002000000171008181710072
:10A3C0004BE893000080FB000100200000017100B9
:10A3D0008181710052059800630598003BE9930064
:10A3E000C811DD00020020002BE893008080FB00F4
:10A3F0000000200000017100818171001BE89300C2
:10A400004800DD0001002000000171008181710021
:10A410000BE893000080FB000100200000017100A8
:10A420008181710072059800030D9800EFE4970098
:10A43000094D78004C1FEC0060FA88003005980048
:10A440006000B80050159800611598000040EB00BE
:10A450004045980002003700A900200003003700A3
:10A460008004EB0001003700D900200060FB2F00C2
:10A470000F004000B0AF9F000900E000CF003A009D
:10A480009E407800F0C2B30080CF5000050032003B
:10A49000C0C5B30080CF5000020032000E04780027
:10A4A000010037000E04E8006000B800C0A79F005C
:10A4B000D1A79F00F1C1B30098CF100009003E0062
:10A4C0008000EB0022FC2F000F004100E4FC07009D
:10A4D000800478000000EB00A0AF9F00B7003700B9
:10A4E0000804E80098407800F0C2B30080CF500024
:10A4F000FBFF3200C0C5B30080CF5000F8FF320030
:10A50000BFAC9700B20020000102200009007800D3
:10A51000C2FA07008041EB008002EB00850378005F
:10A5200086002000E8C07B00014178008703E80036
:10A5300000C2B30080CF5000350036006F404000AD
:10A5400080CF500032003200C0C5B30080CF500031
:10A550002F003200E0C2B30080CF50000200320072
:10A56000868F520008003900E80F530090003A002F
:10A5700080CF50008E003A00C219DD0086027800BC
:10A58000B6002000E7FF37000104E00005003D00B1
:10A590003340B3000180FB000008B10021B12A0064
:10A5A00060C178000282FB0021B92A000100370057
:10A5B0008100E800114078000004E000040032004F
:10A5C0000000FB00840F5000F9FF3A0078003700CC
:10A5D000F0CBB30000404100F94F500002003E00B4
:10A5E0000314A00007003700F0C9B3000040410089
:10A5F000F94F500003003E000304A00000CEB3005A
:10A600000041410082F27C008502E800C5FF37006E
:10A610000704440042C0B30000C2B30080CF500022
:10A620000600360004003700490020003E003700D5
:10A63000800478003C0037000041EB000500E0009A
:10A640005B00320054CEB300994F120002003A0072
:10A6500050C0B300804C7800E80F530001003A006E
:10A66000C219DD008380FB0063806000E10F5000B1
:10A6700001003A000244A0006C806000E40F50002A
:10A6800001003A000234A000B24C98008000EB00B8
:10A6900025FC2F000F80420071FC07008004780029
:10A6A0000000E00020003A000FA997009FA9970042
:10A6B0001FA0970060FA0700800478000000E00007
:10A6C00019003A00AFA897001104E000D6FF32004D
:10A6D000314890000038A3000E003A0001027800D3
:10A6E000BFA99700B2002000090078000201E9002C
:10A6F000E10F410005003200B480FB003380FB0015
:10A700000080500003003A00F8FF37000000E0002E
:10A71000C7FF32008000EB0029FC2F000F804400AF
:10A72000A4FC0700DDFF37003FA8970030489000E9
:10A730000900E00005003200E48F54001F003A00D9
:10A740000028A3001C0032001C0037000028A300D2
:10A750001A003A00AFA89700314890000048A300C3
:10A7600015003200515190004811DD004150900019
:10A770000080FB000001710003002000C011DD001B
:10A7800002002000315890004800DD00215A90005E
:10A790000482FB0004007000010020000001710031
:10A7A00081817100C2A79F00D3A79F004DFF370092
:10A7B000690020000100370059002000AFAE97006B
:10A7C0000900E00003003A000D00E00001003A003B
:10A7D000690020004FD897008080FB007C806000DB
:10A7E000A30032000900E0002E003200E48F540084
:10A7F00025003A008000EB0022FC2F000F004100F2
:10A8000017FC0700800478000000E0001E003A00FA
:10A8100023FC2F000F8441000FA997009FA99700E8
:10A820001800780004FA0700800478000000E000B7
:10A8300015003A002FA8970010407800FB4F400009
:10A84000D80032000004E000D600320011002000E1
:10A850000800780057FC0700EAFF37002FAC97008C
:10A86000020220000800BE00ECF90700BFA8970014
:10A87000B200200008007800E1F907009A00780093
:10A8800010C0B300C04098004FDA97000434A00015
:10A89000C4DF9F00AFAE97000900E000080032005F
:10A8A000D90037003D489000710060007900200019
:10A8B000D5003A00890020000128A300D2003A0008
:10A8C000CFDA97000538A3007C003200462A070043
:10A8D000E04E98004801DE00F24E98004009DE008C
:10A8E00003002000825698004808DE009056980029
:10A8F0008042EB00B54E9800C55E9800D55E98008A
:10A90000E55E9800F55E9800F58446007484460084
:10A91000FB8346007A8346001981FB004811DD0065
:10A920001880FB000001710003002000C011DD0051
:10A93000020020001780FB004800DD001682FB00AB
:10A94000040070000100200000017100818171008D
:10A95000F2AF9F0083B79F00054B7800854B7800CE
:10A96000054C7800854C780028FC2F000F0144002E
:10A970009200780010C0B300C04098007FA89700F4
:10A980008FB09700E00F5000E08F58004600320073
:10A99000120678005C119000EC119000C2AF9F008D
:10A9A000D3AF9F00E10F5000E08F58002E0036001B
:10A9B0003C089000CC0890007FAA97008FB29700C7
:10A9C000800F5200818F5A00270031000404BE001E
:10A9D0000801BE000C007800F4F907000005BE0075
:10A9E000E00F5000E08F580078003200E10F500077
:10A9F000E08F58001C003200E10F4000E08F48005B
:10AA0000800032006022B8000801BE000C0078000F
:10AA10006EFA0700800478000000E0007A003A0037
:10AA20007C0090008C089000E10F4000E08F48000F
:10AA30000600320061004000E08048007006980087
:10AA4000010E980010C0B300504698003C089000DA
:10AA5000CC089000800F5500818F5D005B003100B5
:10AA60000A04BE00DAFF3700290020006600370024
:10AA70000900E00064003A003D4890000080FB00BF
:10AA8000490020000048A3005F003A000118A3001D
:10AA900003003200790020000008A3005A003A00A9
:10AAA0000138A300050032008004EB00CFDA9700E4
:10AAB0000554A000C5DF9F00010037008004EB00B3
:10AAC0009FA2970055109000E51090006FB197007D
:10AAD00050099800610998007D099800CFD9970026
:10AAE000434198005D5190004811DD004D509000A9
:10AAF0000080FB000001710003002000C011DD0098
:10AB0000020020003D5890004800DD002D5A9000C2
:10AB10000482FB00040070000100200000017100AD
:10AB2000818171006FB2970072029800030A980049
:10AB30007D599000C811DD00020020006D58900082
:10AB40008080FB0000002000000171008181710005
:10AB50005D5890004800DD000100200000017100F8
:10AB6000818171004D5890000080FB0001002000A1
:10AB70000001710081817100520298006302980007
:10AB80006000B8003002980041029800300A980036
:10AB9000410A9800050A7800B50290001502980055
:10ABA0001900370025FC2F000F8542000FA99700E0
:10ABB0009FA997001A0078001FF907008004780009
:10ABC0000000E00030FF3A0024FF37001FA097008C
:10ABD0007FAC97008FB4970061015400E0815C0066
:10ABE00052009800630098004FA99700DFA99700D2
:10ABF00011F90700800478000000E000ABFF32008C
:10AC00000100370019002000090078004F07780084
:10AC10004F06BE004F05BE004F04BE00EF03B1005B
:10AC200000000600E6874700889FBE008A9FBE009E
:10AC30008C9FBE008E1F7800800478000207780089
:10AC400083BF9F00F1B79F008009EB009000900048
:10AC5000100078002BFC07000000E000AE003A0076
:10AC6000C9409000200020000104E000AA00350047
:10AC7000700020000108A300A70032000D0037007B
:10AC8000494090000074A000C044980020002000BB
:10AC9000A10037000174A000C144980003003700F0
:10ACA000494090000074A000C044980010002000AB
:10ACB0009900370059009000E90090003901900098
:10ACC000C901900002015000838158006170B800F2
:10ACD000820F5000838F58008C00360002077800E6
:10ACE0008A00370039029000C90290000400780001
:10ACF000F01FB2006C003A00990078004728DD0090
:10AD00004921DE0002017000C929DE0021409000C7
:10AD10000040E9008246600012003A00E00F520055
:10AD2000E08F5A0003003A007900900089089000F3
:10AD30000400370019099000A9099000010078006B
:10AD40001AF90700E10F5000E08F5800CCFF3600E1
:10AD5000E10F4000E08F4800D1FF3200900C9800D6
:10AD6000A10C98001906780019099000A909900013
:10AD70000C007800F5F807000001BE00E00F50005D
:10AD8000E08F5800BEFF32000D80FB000100200064
:10AD900002054000838548004974DE00250032002A
:10ADA000AC4090000D81FB00080041008180FB0059
:10ADB000810F500001003600028450001C409000BA
:10ADC000084278000A01BE00FFB097004A1A070047
:10ADD000C94090000000E000AEFF3A000168A30007
:10ADE0001200320039089000C90890000A01500092
:10ADF0008B8158006140B800800F5100818F59004D
:10AE00000A0031000102200089804000491ADD005B
:10AE1000C711DE00830172004911DD007FB2970087
:10AE2000020042000220200075F807004944DD00BE
:10AE30002A00370039099000C90990008A0F510093
:10AE40008B8F590016003200494090000068A30023
:10AE50000A00320001022000898040001C4090005E
:10AE600014C0B300601A0700C94090000000E00061
:10AE700088FF3A000164A100C1449800010220004B
:10AE800089804000190078001040900014C0B30081
:10AE90000A01BE00181A07000000E00080FF3A0017
:10AEA000BA0C9800CB0C9800B9019000F31FB200C7
:10AEB00000202000030450008E0F540001003600D3
:10AEC0000E04780001022000898040008380400049
:10AED000080178007FB0970049F807007FB097001D
:10AEE00008004000F0B79F0039009000C9009000B2
:10AEF00008004000E0804800B0049800C1049800B9
:10AF00000FBA9700140A4400080757000E00E0002B
:10AF100074FF3A000E0078004F0778004F06BE001D
:10AF20004F05BE004F04BE006F00B10000000600D8
:10AF3000E6874700889FBE008A9FBE008C9FBE00A8
:10AF40008E1F7800000478008206780083BF9F007F
:10AF5000F1B79F008009EB0090009000100078008E
:10AF600068FB07000000E000CE003A00C8409000F7
:10AF7000200020000104E000CA003500700020001D
:10AF80000118A300C70032000D0037000174A000B3
:10AF90004144980008003700484090000074A00029
:10AFA0004044980020002000BE0037004840900038
:10AFB0000074A0004044980010002000B900370041
:10AFC00058019000E80190000D004100E080490028
:10AFD000820F5000838F5800A5003900A20037006F
:10AFE00038029000C802900004007800F01FB20000
:10AFF00081003A00980078004728DD004921DE00F2
:10B0000002017000C929DE00214090000040E900E3
:10B01000024760001E003A00E00F5200E08F5A0025
:10B020000B003A007801900088099000E00F510071
:10B03000E08F59000E003A000100780095F90700F2
:10B040000001BE0070049800010C98000500370054
:10B0500018099000A8099000010078008DF90700F8
:10B060000001BE00E00F5100E08F59008000320067
:10B07000E10F5100E08F5900C7FF3200E10F41009E
:10B08000E08F4900C9FF3200120C9800230C980091
:10B09000484090000068A3000D003200380990007D
:10B0A000C8099000180078001040900014C0B30048
:10B0B0000102200088804000CB190700C8409000A2
:10B0C0000000E000B1FF3A000164A1004144980093
:10B0D0001806780018099000A80990000C00780064
:10B0E0001AF807000001BE00E00F5000E08F580082
:10B0F000A9FF32000E80FB00010020000205400085
:10B1000083854800C96CDE0025003200AC40900009
:10B110000E81FB00090041008180FB00810F50007F
:10B1200001003600828450001C40900009427800E3
:10B130000A01BE00FFB09700AB1907000000E00055
:10B140009AFF3A0038089000C80890000A015000A1
:10B150008B8158006148B800800F5100818F5900E1
:10B160000D0031004918DD00C710DE0081007000BD
:10B170004910DD007FB197008000410002202000CF
:10B1800000022000080040009DF7070048409000A2
:10B190000064A10040449800C94CDD00260037003F
:10B1A00038089000C80890008A0F50008B8F580014
:10B1B0000F00320038019000C80190005800900044
:10B1C000E8009000800F5100818F59000800310085
:10B1D0001C40900014C0B3000A01BE000102200010
:10B1E00088804000441907000000E0006FFF3A002B
:10B1F0003A0C98004B0C9800B8019000F31FB20075
:10B2000000202000830450008D8F54000100360080
:10B210008D04780000022000080040000300400078
:10B2200009017800FFB0970075F7070048409000CB
:10B230000064A000404498007FB0970009004000DF
:10B24000F0B79F0038009000C8009000090040004F
:10B25000E080480030049800410498000FB997003E
:10B2600012894400898656000D00E0005CFF3A0018
:10B2700038019000C801900058009000E80090004C
:10B28000800F5100818F590002003600520498004F
:10B2900063049800484090000054A0004044980087
:10B2A0000000EB004F0778004F06BE004F05BE00C0
:10B2B0004F04BE006F00B10000000600889FBE0072
:10B2C0008A9FBE00800478009000900010007800F3
:10B2D0008CFA0700000578000000E00082003A00C8
:10B2E000494090000080FB000058A3007D00320020
:10B2F0000068A3000D00320039099000C9099000D0
:10B300000102200089804000190078001040900060
:10B3100014C0B300341907000000E0006F003A00C9
:10B32000494090000064A100C04498005909900071
:10B33000E9099000190078003FF707000005780040
:10B340000000E00068003A00790C90006B004400B7
:10B350001054A00029489000405C980039489000A3
:10B36000505C980049489000605C980059489000F3
:10B37000705C980069489000205C980079489000C3
:10B38000305C98000950900040549800195090008B
:10B390005054980094270700605498004801DE003C
:10B3A000725498004009DE0003002000025C9800FF
:10B3B0004808DE00105C9800494090000054A1004D
:10B3C000C0449800190078001BC0B3004B4098009F
:10B3D000990478006011B8000900780016F707009A
:10B3E000000578000000E0003F003A0030C0B300E4
:10B3F000994F100033003A00594090000004E000DB
:10B40000300032006000B800D0149800E1149800B9
:10B41000E802200009044400022020008A0078008D
:10B4200008007800FDF6070050C5B30060FC9B00E3
:10B43000A0CAB30070FC9B0020C5B300004C78008C
:10B44000F06C980012C6B3008274980011C4B30067
:10B450009174980020C7B30040E49B0050E49B0027
:10B4600061E49B0072E49B006948900000EC9B0043
:10B470007948900010EC9B000950900020EC9B0054
:10B480001950900030EC9B002948900040EC9B0044
:10B490003948900050EC9B004948900060EC9B00BC
:10B4A0005948900070EC9B0019099000A909900080
:10B4B000194090000B42780088007800CA180700F5
:10B4C000DA449800194090000001EB008040EB0046
:10B4D000131907000000E000020032001A002000EB
:10B4E000010037000005EB000A0078004F05BE00A0
:10B4F0004F04BE0000000600881F7800000478009A
:10B500006EFF07000000E00001003A00000C780028
:10B510004F047800000006000800FA00889FBE0073
:10B520008A9FBE008C9FBE000005780082BF9F00EE
:10B5300093BF9F009000900010007800F1F9070081
:10B54000000178000000E000EC003A004A40900062
:10B55000220020000004E000E80035005A019000BD
:10B56000EA0190000FBA97009FBA9700820F52002D
:10B57000838F5A00040036000018A30002003A002E
:10B5800082BF9F0093BF9F003A019000CA019000C4
:10B590006000B80030059800410598000FB897008A
:10B5A0009FB89700E00F5000E08F58009A003200DB
:10B5B0009A0578002B4090000080FB0001002000DD
:10B5C000490ADD00C702DE00850272004902DD0083
:10B5D000E4B79F00F5B79F00E00F5100E08F5900DE
:10B5E0002400320061065100E08659000FB997002F
:10B5F0009FB9970061005100E08059000401BE002E
:10B6000097D407000004BE006FB19700FFB1970008
:10B610000C00BE0092D40700800F5400818F5C00A4
:10B62000140039006FB29700FFB29700600012005B
:10B63000E0801A000C0160000D806000800278003C
:10B64000020278000400BE00300598004105980011
:10B650000FB997009FB997000001510081815900EF
:10B6600082BF9F0093BF9F001A099000AA09900013
:10B67000120037007A0190008A099000E00F510013
:10B68000E08F59000B003A000B00780001F807002A
:10B690000001BE00E10F5000E08F58005000320062
:10B6A000E10F4000E08F48008900320070059800EB
:10B6B000010D9800120D9800230D9800E00F510025
:10B6C000E08F59002E003A00530037004A409000A6
:10B6D0000018A3000B0032001A007800EDF70700F5
:10B6E0000001BE00E00F5000E08F580008003A0053
:10B6F0006FB29700FFB2970084BF9F0095BF9F0075
:10B70000260037001A007800A8F607000001BE00E6
:10B71000E10F4100E08F49006D003200E10F510060
:10B72000E08F59002E0036001A007800C008900003
:10B7300030089000800F5100818F5900280031009F
:10B74000120D9800230D98003A009000CA00900056
:10B750006FB29700FFB29700040040008580480058
:10B7600030059800410598000FB897009FB89700E2
:10B77000040050008580580080BF9F0091BF9F004B
:10B780000FBA97009FBA97006FB09700FFB097006D
:10B79000800F5200818F5A00CCFF3E003A0090008B
:10B7A000CA0090000FBA97009FBA970004004000AB
:10B7B0008580480030059800410598000FB8970033
:10B7C000F01FB200140032001A0078005FF6070084
:10B7D0000001BE00E00F5000E08F580005003A0065
:10B7E0004A4090000074A0004045980022002000CC
:10B7F000420037000FBA97009FBA9700472BDD0031
:10B800004920DE0000007300C928DE000206400067
:10B8100083864800010037006066B8003A00900057
:10B82000F01FB200210032003A099000CA099000CE
:10B83000820F5600838F5E001C0032004A40900049
:10B840000068A3000E003200010220008A80400040
:10B850001A0078001040900014C0B300E2170700EF
:10B86000CA4090000000E000030032000174A00014
:10B8700041459800190037000164A1004145980036
:10B88000010220008A8040001A00780010409000D9
:10B8900014C0B3000C01BE00971707000000E000C1
:10B8A0000B003A003C0D98004D0D98003A029000B4
:10B8B000CA0290005A009000EA0090000001EB00DC
:10B8C000800F5200818F5A000C00360005003700AF
:10B8D0004A4090000074A0004045980012002000EB
:10B8E0000600370054059800650598004A4090000E
:10B8F0000054A000404598000001EB0002007800D1
:10B900004F06BE004F05BE004F04BE000080FA0087
:10B9100000000600889FBE008A1F7800000578009E
:10B920008104780002047800302207000841780082
:10B93000894078000A4078003A22070008417800E0
:10B94000894078000A407800442207004F057800BB
:10B950004F04BE0000000600E40F50001F0032003C
:10B9600009003E00E10F5000110032000041EB00E1
:10B970001B003900E20F500010003200E30F5000AE
:10B9800025003A0011003700E60F50001600320083
:10B9900002C2B3008040EB000A003900E70F5000FC
:10B9A00015003200E80F50001B003A001600370067
:10B9B0000041EB0001C2B300110037000041EB0071
:10B9C00001C2B300014078000E0037000041EB00D7
:10B9D0008240780000C2B3000A00370002C2B30000
:10B9E00082407800F7FF370002C2B300824078003F
:10B9F0000040EB000300370002C2B3008040EB00C0
:10BA000002407800F921370052C0B300F1C0B30002
:10BA100000C2B300F521070000000600881F78006F
:10BA2000000478000001EB006000B800B9FF0700D7
:10BA30008043EB0007437800874278000742780094
:10BA400087417800074178008740780007407800F8
:10BA5000BE2107008040EB0000C1B3000F210700AA
:10BA60008040EB0010C1B3000C2107008040EB00C8
:10BA700040C1B300092107008040EB0050C1B30072
:10BA8000062107008040EB0020C1B300032107001E
:10BA90008040EB0030C1B300002107008040EB0084
:10BAA00060C1B300FD2007008040EB0070C1B3000F
:10BAB000FA2007008040EB0001407800F7200700E3
:10BAC0008040EB0010C0B300F4200700E40F5400E6
:10BAD0001400320006003E00E20F54000E00320057
:10BAE0000B003E00E10F540022003A000A0037002C
:10BAF000E60F54001B0032000C003900E70F540021
:10BB000018003200E80F54001A003A0017003700FE
:10BB1000001020004D360700400020004B36070083
:10BB20000D003700080078001100370040002000A9
:10BB30004636070000012000443607008040EB0035
:10BB4000E0C1B300D52007008032EF00E11C2100E6
:10BB5000F0DF2F00910860005E32EF006032EF00EE
:10BB6000040037005E32EF006032EF00400020003A
:10BB7000363607004F047800000006000010200051
:10BB80002536070000202000233607000001200092
:10BB900021360700400020001F360700100020005B
:10BBA0001D360700000120001B363700881F780073
:10BBB0000004780068FF0700E40F54002200320000
:10BBC00006003E00E20F54002A00320015003E003D
:10BBD000E10F540029003A0008003700E60F540036
:10BBE000240032001A003900E70F54001F00320011
:10BBF000E80F540021003A001E0037008043EB009C
:10BC00000743780005C2B3000542780085417800FB
:10BC10000741780087407800074078004B210700F3
:10BC20001400370000102000FB3507004000200002
:10BC3000F93507000041EB0082407800F0C0B30006
:10BC40006A2107000D003700080078000A0037005D
:10BC500040002000F035070000012000EE3507000D
:10BC6000A00F20000094880004003700F62FEF009A
:10BC7000F42FEF0040002000E73507004F04780064
:10BC80000000060000417800FF4F500002003E0017
:10BC90008000FB00070037008000EB00F0C3B3001A
:10BCA000804F510003003E000040E8000240500079
:10BCB0008000FB000100780000000600C27F8000C9
:10BCC000010040000100370069005000E80F5000FB
:10BCD000FDFF3C0001003700690040000000E0006B
:10BCE000FDFF3500E40F5000F5FF3200E80F500073
:10BCF000F3FF32000000E00002003A000200E00022
:10BD0000EFFF320000000600EC874700889FBE006E
:10BD10008A9FBE008C9FBE008E1F7800F14FEC0002
:10BD200080407800F1EFB70040C6B30080CF5000EC
:10BD30001C0036000040E800F1EFB700B1CFBF00B3
:10BD40000400320010C0B30011002000B85EE20011
:10BD5000010032008000EB00B8FEB7000104E000F3
:10BD600010003200D07F80002CFF0700917F800000
:10BD70000100E00012003200D07F8000808F500070
:10BD800004003A000000EB0088FF0700FA2FEF00E4
:10BD9000040037000100780084FF0700917F8000D5
:10BDA000D17F88008F340700D17F80008001780028
:10BDB0000000E000060032000100780017FF0700D5
:10BDC00000402000A13507006CFF07002D0537005B
:10BDD000E38F5000B001320004003E00E18F5000BC
:10BDE00044003200E5003E0007003700E68F5000B7
:10BDF000BA033200E78F500068043200E58F50002C
:10BE000020053A00B7023700AFCFBF000400320070
:10BE100010C0B30011002000B75EE2000100320044
:10BE20008000EB00B7FEB7000104E0000400320020
:10BE3000907F80008080EB00A0FF0700907F88004B
:10BE4000B0CFBF000400320010C0B30011002000CA
:10BE5000B65EE200010032008000EB00B6FEB700E3
:10BE60000104E00004003200907F80008080EB003D
:10BE700092FF0700907F8800B2CFBF00040032001D
:10BE800010C0B30011002000B55EE20001003200D6
:10BE90008000EB00B5FEB7000104E00004003200B2
:10BEA000907F80001100200084FF0700907F8800B1
:10BEB000B3CFBF000400320010C0B3001100200057
:10BEC000B45EE200010032008000EB00B4FEB70077
:10BED0000104E00004003200907F80001100200087
:10BEE00076FF0700907F8800907F80009AFE070011
:10BEF000E4043700289280000100780062242100C9
:10BF000092007800888F500002003400010478000D
:10BF1000800178000000E8000281E800E50F500091
:10BF2000F7FF3A0075F880006280110024002000BD
:10BF300000017800110009008402D8000001FD0012
:10BF40000280B90000057800C0DA20008000EB0014
:10BF5000800F540004003400080050001100090054
:10BF60000400D8008000FD0000FA2000800F54007B
:10BF7000020034008500EA000D00370070BB20008D
:10BF8000800F540007003C0080C12F0000004400D7
:10BF900072002000110009000200D800C112200028
:10BFA00080805000F07C2000800F5400020034009C
:10BFB000858F500001003400850078008504EA0078
:10BFC000898F50000100350081047800301F200067
:10BFD000800F540003003C005E32EF006032EF003F
:10BFE0000400370009004500009388000A805400CF
:10BFF000F0928800F04FEC008000FB00F0EFB700FB
:10C000000004E000090034000001EB000000EB0038
:10C0100040FE070080C2B300F04FE3000B00340085
:10C0200000C8B300F0EFB700080037008100EA0055
:10C0300042002000110009008200D8008000FD00AD
:10C040000001EB000000EB0032FE0700B2CFBF00A2
:10C050000400320010C0B30011002000B35EE20003
:10C06000010032008000EB00B3FEB7000104E000E5
:10C070000700320070F880002003B00070F88800DC
:10C08000411F2000810F50000100340071F888002A
:10C09000AFCFBF000400320010C0B3001100200079
:10C0A000B25EE200010032008000EB00B2FEB70099
:10C0B0000104E00007003200E0FC2F000E1FB40076
:10C0C00070F8880041ED2F00810F500001003D0005
:10C0D00071F888008040EB00401F2000800F540062
:10C0E0000400340011C0B30010002000B15EE20073
:10C0F000010032000000EB008000FD00B1FEB7003F
:10C100008000FD000004E00002003200600020001A
:10C11000522C07000A00E0000C003A000900E00081
:10C1200054043A00EF4FE20052043A00401F20004E
:10C13000800F54004F04340010C0B300EFEFB7007D
:10C1400070002000452C0700C8003700EF6FEF009B
:10C15000C6003700E0928000810F5000C700340015
:10C160008040EB0080C0B3004C1F07008040EB0014
:10C17000B0C0B300491F0700420437007881570060
:10C1800084CD2A0007000900345978008200B100EC
:10C19000ED4FEC0080407800EDEFB7004240A90081
:10C1A00008003400034178001020070080C2B3006B
:10C1B000ED4FE3000B00340000CCB300EDEFB7000F
:10C1C000080037000000FB000000EA002200200009
:10C1D000110009000200D800034178008040780077
:10C1E00002200700EECFEC0080417800EEEFB700B0
:10C1F0000080FB004500DE0002C2B300F8005000E2
:10C2000082F07F008000E900E7806000FFC16100EC
:10C2100003415100F880500082F07F000000E800E8
:10C22000670060007800500003F07F00FFEB97008C
:10C230002FE997009FE897006FEB9700DFEA9700E0
:10C240004FEA9700BFE997000FE89700BF1F07006C
:10C25000B2CFBF000400320010C0B30011002000B4
:10C26000B05EE200010032008000EB00B0FEB700DB
:10C270000104E0000700320060F880002003B000F5
:10C2800060F88800411F2000810F50000100340039
:10C2900061F88800AFCFBF000400320010C0B300C7
:10C2A00011002000AF5EE200010032008000EB00D0
:10C2B000AFFEB7000104E00007003200E0FC2F00F1
:10C2C0000C1FB40060F8880041ED2F00810F500072
:10C2D00001003D0061F888006EF880000E00E0006B
:10C2E0005100350028928000349280006145B900E9
:10C2F00004004200CF80DE000A0540008B85480024
:10C30000409280006300B900CF80DE000A05400043
:10C310008B8548005292800002004100CF80DE00F1
:10C320000A0540008B854800669280006130B900A4
:10C330000A0540008B854800C0FF2F0000C4B900EB
:10C34000CFC4DE00D0FF2F0000A2B900CFA2DE00D4
:10C350000804420089844A006311B900CF91DE00CD
:10C3600008044100898449004233DD00CFB3DE0078
:10C370000804430089844B000A0044008B804C0071
:10C380006176B9000C01BE0027D10700027D2000B4
:10C39000811F7800110009004208D800CF00780002
:10C3A0000000570080BF9F00F092880008055500EC
:10C3B00089855D000C01BE000A00BE001AD107008D
:10C3C000047D2000811F7800110009004408D80076
:10C3D000CF007800000057000093880081DA2F001A
:10C3E0000FB89700810F500001003D00F1928800C6
:10C3F00000938000810F500001003D0001938800F0
:10C4000081252000F0928000810F5000010034004F
:10C41000F192880000938000810F500013003400D7
:10C420000193880011003700809280000E80B900CF
:10C4300042ED2F00811F7800110009004208D8004A
:10C44000CF00780000004700F092880070928000D2
:10C450000E80B900811F7800110009004208D80041
:10C46000CF007800000047000093880011082000EA
:10C47000D0928000810F500036FF3C005E32EF000A
:10C480006032EF0001C2B30080C0B300831E07001A
:10C4900001C2B30036FF370050F880008000400032
:10C4A00080804000909380000000E00001003D008B
:10C4B0000000EA0080804000A09380000000E000BF
:10C4C00001003D000000EA0080804000B093800041
:10C4D0000000E00001003D000000EA000080400094
:10C4E0004200DE0050F8880083007800ED0F500015
:10C4F00001003E0011002000810478008340780094
:10C50000EE0F50000400360011C0B30013002000ED
:10C51000AE5EE200010032008001EB000100780015
:10C52000AEFEB7000304E000040032000041EB005F
:10C5300082407800F0C0B3002C1F070050F8800044
:10C54000ED0F50000F003E00EA0FEC00507F880016
:10C55000E50F500007003400EA0F500001003A00D8
:10C56000EA2FEF000041EB008240780000C2B300E8
:10C57000190037000041EB0082407800024078004B
:10C5800015003700EC4FEC008001FB00ECEFB7002A
:10C590000004E0000A0034000001EB008000EB0022
:10C5A00003007800DBFC070080C2B300EC4FE3001F
:10C5B0000A00340000CCB300ECEFB70007003700EE
:10C5C0000300EA0022002000110009000200D80048
:10C5D0000041EB0082407800041F07008812E2004F
:10C5E000030032008832EF00500020001B2B0700B0
:10C5F00037928000813E2000818F53001700340065
:10C6000040928000810F500014003400509280004E
:10C61000810F50001100340070928000810F500093
:10C6200003003C0080928000810F50000B0034001A
:10C6300021082000D0928000810F500007003400B4
:10C64000E0928000810F5000040034005E32EF0061
:10C650006032EF0019002000580037002892800057
:10C66000823E2000820F54000B003C00828F53005A
:10C6700009003C0040928000820F500006003C0000
:10C6800050928000820F500003003C0060928000B6
:10C69000820F5000380034005400200011000900BF
:10C6A0000404D800000378004200200011000900B3
:10C6B0008203D8000003430040928000110009006B
:10C6C0000200D80000034300509280006592800071
:10C6D000801F7800110009000200D80000017800D6
:10C6E0004F007800801F7800110009008402D800F4
:10C6F000800078004F0078000101410002034300F0
:10C7000062002000801F7800110009000204D80098
:10C71000800078004F00780080017800811F780049
:10C72000110009008403D8008001FD00CF007800CB
:10C7300083804000811F7800110009000400D800A8
:10C74000CF007800809FBE00110009008202D8004F
:10C75000800278004F00BE0005004000808050003D
:10C76000010043000000EA00F0928800868050003B
:10C77000019388001100370071928000828F500071
:10C7800003003C0080928000820F500009003400BA
:10C7900042002000110009008200D800F0928800B9
:10C7A00080928000110009000200D80000938800E8
:10C7B000020037005E32EF006032EF001108200007
:10C7C000D0928000810F500003003400E09280007E
:10C7D000810F50000A003C005E32EF006032EF0033
:10C7E0000041EB008240780000C2B3008D1E0700BC
:10C7F0000041EB008240780000C2B3000700370020
:10C800000041EB008240780002407800851E07005E
:10C810000041EB0082407800024078008F1E070044
:10C8200081DA2F00F0928000810F500001003D005E
:10C83000F192880000938000810F500001003D00BC
:10C840000193880081252000F0928000810F500024
:10C8500001003400F192880000938000810F5000A5
:10C8600001003400019388008040EB000900E000E3
:10C870000400320011C0B30010002000AD5EE200E1
:10C88000010032000000EB008000FD00ADFEB700AB
:10C890008000FD000004E0000200320040002000A3
:10C8A000702A07008040EB000900E00004003A0015
:10C8B00011C0B30010002000AC5EE20001003200A5
:10C8C0000000EB008000FD00ACFEB7008000FD0022
:10C8D0000004E0006B0232000080EB005F2A0700DA
:10C8E00068023700E11C2100708E80000098A300D0
:10C8F00040003200F0DF2F009108600077FE20003A
:10C90000974378000704E0000C003A000700780025
:10C91000E8EFB70010C0B300E7EFB70007437800B7
:10C920008742780007427800874178000741780005
:10C93000874078007F40400014003700E1CF53006B
:10C9400014003A0081FE200091407800E2CF5000B0
:10C9500028003400FDCF500026003C0020C0B3006A
:10C96000E7EFB7000140E800E3EFB700FFC3430083
:10C970000043EB008642780006427800864178004A
:10C98000064178008740780007407800EF1D0700D7
:10C9900018003700E2CF530016003A0081FE200055
:10C9A0009140780001407800E34FE30011003D0022
:10C9B00070C2B30080CF50000E003C0030C0B30006
:10C9C000E7EFB700FEC34300074378008042EB0067
:10C9D000054278008541780007417800874078005B
:10C9E00007407800D91D0700700020001B2A0700AF
:10C9F000E96FEF0081FE20009140780030C6B3005F
:10CA000080CF500002003C000140E800E8EFB70092
:10CA100020C3B300E84FE3000A003400E76FEF00E3
:10CA20008043EB0007437800874278000742780094
:10CA300087417800074178008740780007407800F8
:10CA4000C21D070081FE200091407800E5CF500014
:10CA500019003A00E4CFBF00E14F50000A003A004D
:10CA600070FE200011C0B30090CF100032003A00D9
:10CA700020C0B300E4EFB70000052000F09288006A
:10CA800000FB2F000A003700E24F50002A003A0056
:10CA900070FE200012C0B300904F110026003A0033
:10CAA00002407800E4EFB70000052000F092880013
:10CAB0000093880020003700FECF50000F003A009E
:10CAC00070FE2000E44FE20005003A0024C0B300ED
:10CAD000904F120018003A0010C0B300F1FF370069
:10CAE00021C0B30090CF100013003A00E46FEF00B4
:10CAF0005E32EF006032EF000F00370080C2B300FB
:10CB000080CF50000C003A0070FE200032C0B3000D
:10CB1000904F110008003A0011C0B30001007800E6
:10CB2000E4EFB70000052000F09288006032EF00CB
:10CB300001007800E6EFB70011082000D0928000D5
:10CB4000810F500003003400E0928000810F5000FC
:10CB50000A003C005E32EF006032EF000041EB0063
:10CB60008240780000C2B300AE1D07000041EB0018
:10CB70008240780000C2B300070037000041EB009C
:10CB80008240780002407800A61D07000041EB00BB
:10CB90008240780002407800B01D0700E64FE200B6
:10CBA00036003200E54FEC00E5EFB70001C6B300F8
:10CBB000814F500001003400E56FEF00E5CFBF006A
:10CBC00004C2B3008444400081CF54000100360009
:10CBD00081C4540002C4B30002444000814F540099
:10CBE000010036000144540026FC0700004578008F
:10CBF0000940780023FC0700804478000840780052
:10CC000020FC07000044780000417800894078004B
:10CC10000A407800751D0700094178008A407800B5
:10CC2000084078008D1D07000A4178008840780090
:10CC3000094078007B1D0700E94FEC008040780038
:10CC4000E9EFB700F0C7B30080CF50008D013A0084
:10CC5000E66FEF00E96FEF000041EB0082407800E3
:10CC6000024078007D1D07000041EB008240780003
:10CC7000024078006B1D070082013700E94FEC008D
:10CC800000417800E9EFB7004240A90009003400F4
:10CC90008040EB0001407800541D070080C2B300C3
:10CCA000E94FE3007701340000C8B300E9EFB700B3
:10CCB000740137000001FB000201EA00430020007C
:10CCC000110009000301D800000178008040EB004A
:10CCD00001407800451D07006A013700E24FEC0073
:10CCE00000417800E2EFB7004240A900090034009B
:10CCF00080407800034078003C1D070080C2B300EC
:10CD0000E24FE3000C00340000CCB300E2EFB700C8
:10CD1000090037008000FB008100EA0022002000AB
:10CD2000110009008200D8008000FD000141780058
:10CD3000034078002D1D0700AF4FE20009003200CC
:10CD4000B24FE20007003200E09280005A12B400B5
:10CD500022002000110009000200D8006009B00084
:10CD600040F88800B04FE2000F003200B34FE200FD
:10CD70000D003200E09280005A12B4002200200020
:10CD8000110009000200D80030F888005109200085
:10CD9000810F500002003E00800C200030F8880017
:10CDA000A0F62F00063FB400D092800042F8800029
:10CDB000820F500001003100E06FEF0031F8800079
:10CDC000810F50000200360010C0B300E0EFB70042
:10CDD000E0928000820F500001003100E16FEF000F
:10CDE000810F50000200360010C0B300E1EFB70021
:10CDF00001FE2000914078000104E00002003200B2
:10CE0000E1CF500005003A00E14FE20003003A0094
:10CE100001007800DFEFB7001300370010FE20009C
:10CE200012C0B300904F110004003A000104E0006A
:10CE300002003A00DFEFEF000B003700DFCFBF004A
:10CE40004240A9000200340020C0B30005003700B2
:10CE50000004E00002003D00E0CFB3000100370015
:10CE6000A0C0B300DFEFB700F7FD200097437800C4
:10CE70000704E0000B003A00C0122000F092880086
:10CE800000938800074378008742780004C2B3000B
:10CE90008741780007417800874078000440780097
:10CEA00036003700E1CF53000B003A00C0122000DB
:10CEB000F09288006032EF008043EB000743780077
:10CEC000874278000742780003C2B3000741780028
:10CED0008340780028003700E1CF43000A003A0081
:10CEE0005E32EF00C01220000093880007C2B3003A
:10CEF0000043EB00874278000642780086417800C4
:10CF0000064178001B003700E2CF43000D003A00D5
:10CF100040ED2F00F0928800C0122000009388009E
:10CF20008043EB0006C2B3008742780007427800D6
:10CF300087417800074178008740780007407800F3
:10CF40000E003700E2CF53000E003A00C01220005E
:10CF5000F092880040ED2F00009388008043EB00A2
:10CF600007437800874278000742780087417800BD
:10CF700002C2B3008640780006407800731C0700A8
:10CF8000C0003700EACF5300BE003A00C0122000B4
:10CF9000F092880040ED2F00B4003700DE4FEC0027
:10CFA00000417800DEEFB7004240A90008003400DD
:10CFB000834078008D1C070080C2B300DE4FE30081
:10CFC0000B00340000CCB300DEEFB70008003700E0
:10CFD0000000FB000000EA00220020001100090010
:10CFE0000200D80000417800834078007F1C0700D1
:10CFF00005FB200095427800054078000504E0001C
:10D000000400320010C0B30011002000AB5EE2004B
:10D01000010032008000EB00ABFEB7000104E0002D
:10D020000200320080F32F00A07F880034FB200034
:10D0300014427800044078000404E0000400320048
:10D0400010C0B30011002000AA5EE200010032000F
:10D050008000EB00AAFEB7000104E00002003200ED
:10D06000800C2000A07F8800F3FA20009341780014
:10D07000034078000304E0000400320010C0B30055
:10D0800011002000A95EE200010032008000EB00E8
:10D09000A9FEB7000104E00006003200F40FE20030
:10D0A00002003200F42FEF000200370080F32F005F
:10D0B000F62FB40021FB2000914078000140780059
:10D0C0000104E0000400320010C0B3001200200090
:10D0D000A85EE200010032000001EB00A8FEB700EC
:10D0E0000204E00006003200F40FE2000200320009
:10D0F000F42FEF0002003700800C2000F62FB40060
:10D100000304E00003003200100020000104E000EE
:10D1100001003A000000EB00804078000004E000CD
:10D120000300320010002000A75EE2000100320080
:10D130000000EB008000FD00A7FEB7008000FD00AE
:10D140000004E00001003200F62FEF000404E000CC
:10D1500003003200100020000504E00001003A0046
:10D160000000EB00804078000004E0000300320083
:10D1700010002000A65EE200010032000000EB007B
:10D180008000FD00A6FEB7008000FD000004E00066
:10D1900001003200F42FEF00E09380000000E00077
:10D1A0001B003200E40F50000D00320003003C0071
:10D1B000E20F500015003A0005003700E60F50005E
:10D1C00010003200E80F500010003A00060037004F
:10D1D000800C2000F40FE200080032000500370048
:10D1E00080F32F000800370080F32F00F40FE200D7
:10D1F00002003200F42FEF0004003700F62FB400D5
:10D2000002003700800C2000A07F88007C32EF00F5
:10D2100082252000B07F8000820F50000100340082
:10D22000B27F880081DA2F00B07F8000810F50002C
:10D2300001003D00B17F8800A07F8000820F500078
:10D2400001003400A27F8800A07F8000810F500081
:10D2500001003D00A17F8800B07F8000A27F800098
:10D2600082004000F1928800020050000093880084
:10D2700004003700301F2000800F5400B3FB34003F
:10D280007AFC37004F0778004F06BE004F05BE00FE
:10D290004F04BE00CF00B10000000600C07F880030
:10D2A0000000EB0041FA0700F80FE2000200320034
:10D2B000F22FEF000300370010002000907F88005D
:10D2C000A5F90700B0462000533037000040200089
:10D2D0005A3007008080EB000000E00001003200BF
:10D2E000D17F80000100780000000600E80F5000A8
:10D2F00002003400000040007100500000000600F1
:10D300008000EB00E80F5000010034001100200005
:10D3100001007800000006000200FA00F0BF9F0044
:10D32000E30F50001700320006003C00E10F5000F0
:10D330000E00320010003C000000E0000800320047
:10D3400016003700E90F50000B003200EA0F5000C2
:10D350000F003200E40F500010003A000C003700BC
:10D360009460A9008460A9001100370094E0A9002E
:10D3700084E0A9000E0037009500A9008500A900EF
:10D380000B0037009760A9008760A90008003700EC
:10D390009780A9008780A900050037008F81E900E8
:10D3A00042102000913F2000A0C32A001A3107003C
:10D3B0000080FA00000006000400FA00E0BF9F00B1
:10D3C000F1BF9F00E18F5000040036008F81E9001B
:10D3D00062102000912220003E0037006FB89700B5
:10D3E000E30F50002800320006003C00E10F50001F
:10D3F000140032001B003C000000E0000800320076
:10D4000031003700E90F50000D003200EA0F5000E4
:10D410001C003200E40F50002B003A0022003700BD
:10D42000E1C0600081C0400004C1BF000014A10041
:10D430000140700004E1B70005A1A90027003700F2
:10D4400013A1A900E1C0600081C0400010C1BF006D
:10D450000014A1000140700010E1B70011A1A90063
:10D460001E003700E1C0600081C0400012C1BF0053
:10D470000014A1000140700012E1B70013A1A9003F
:10D480001600370021A1A900E1C0600081C0400062
:10D490001EC1BF000014A100014070001EE1B700D2
:10D4A0001FA1A9000D003700E1C0600081C040004D
:10D4B00020C1BF000014A1000140700020E1B700AE
:10D4C00021A1A90005003700E48157004210200087
:10D4D00011262000A0C32A00CF3007000080FA00E8
:10D4E000000006000200FA00F0BF9F00E30F5000AA
:10D4F0002300320006003C00E10F50001200320011
:10D5000018003C000000E000080032002A0037004C
:10D51000E90F50000C003200EA0F500018003200F2
:10D52000E40F500024003A001C003700E1C0600006
:10D53000C608DD0004C1BF000064A1000140700006
:10D5400004E1B70021003700E1C06000C608DD003B
:10D5500010C1BF000064A1000140700010E1B700DD
:10D560001A003700E1C06000C608DD0012C1BF002C
:10D570000064A1000140700012E1B7001300370001
:10D58000E1C06000C608DD001EC1BF000064A1004C
:10D59000014070001EE1B7000C003700E1C06000E0
:10D5A000C608DD0020C1BF000064A100014070007A
:10D5B00020E1B700050037008F81E900421020000C
:10D5C00041292000A0C32A00933007000080FA0000
:10D5D000000006000200FA00F0BF9F000141780041
:10D5E000EA0F50001A003E0010002000FFB897001C
:10D5F0008100DD00010078006020B20006003A00E2
:10D6000080412000008060000A003A000108A30069
:10D6100014003A000E003700E1406100C308DD004D
:10D6200010C1BF000034A1000140700010E1B7003C
:10D630000C003700E1406100C308DD001EC1BF00DF
:10D640000034A100014070001EE1B7000500370062
:10D650008F81E90042102000A1462000A0C32A00CB
:10D660006D3007000080FA00000006000200FA009A
:10D67000F0BF9F00E30F50002C00320006003C007A
:10D68000E10F5000150032001E003C000000E000D9
:10D690000800320039003700E90F50000F00320057
:10D6A000EA0F500021003200E40F500033003A002E
:10D6B0002800370063C060004400DD0041102000F6
:10D6C00091407800F2CCB30082C0600080C070004E
:10D6D0000100780004E1B7002D00370063C060004E
:10D6E0004400DD000111200091407800F2CCB3002D
:10D6F00082C0600080C070000100780010E1B700B7
:10D700002300370063C060004400DD0021112000C9
:10D7100091407800F2CCB30082C0600080C07000FD
:10D720000100780012E1B7001900370063C0600003
:10D730004400DD00E111200091407800F2CCB300FC
:10D7400082C0600080C07000010078001EE1B70058
:10D750000F00370063C060004400DD0001122000AC
:10D7600091407800F2CCB30082C0600080C07000AD
:10D770000100780020E1B700050037008F81E90043
:10D7800042102000214A2000A0C32A0022300700B6
:10D790000080FA00000006000200FA00F0BF9F00BF
:10D7A000E30F50001600320006003C00E10F50006D
:10D7B0000E0032000F003C000000E00008003200C4
:10D7C00013003700E90F500007003200EA0F500045
:10D7D0000A003200E40F50000D003A000A00370042
:10D7E000020888000F0037004308880032088800CC
:10D7F0000C003700520888000A003700B308880080
:10D80000A208880007003700C2088800050037001A
:10D810008F81E90042102000D11E2000A0C32A0001
:10D82000FD2F07000080FA00000006000200FA0049
:10D83000F0BF9F00E30F50001800320006003C00CC
:10D84000E10F50000D00320012003C000000E0002B
:10D85000080032001E003700E90F50000A003200B5
:10D86000EA0F50000F003200E40F500018003A0099
:10D8700015003700000880000100370030088000E4
:10D8800001002000170037003208800040088000A7
:10D890000600370050088000F9FF3700A00880001C
:10D8A000F7FF3700A2088000B008800003002000C6
:10D8B00001002000C000DD00000020000000710019
:10D8C0008180710007003700C0088000ECFF37003E
:10D8D0008F81E9004210200051212000A0C32A00BE
:10D8E000CD2F07000080FA00000006000200FA00B9
:10D8F000F0BF9F00E30F50001F00320006003C0005
:10D90000E10F50001100320016003C000000E00062
:10D910000800320024003700E90F500011003200E7
:10D92000EA0F50001A003200E40F50001E003A00C7
:10D930001700370094C0BF004300DE0061006000A4
:10D940009460A8008460A8001C00370094C0BF0049
:10D950000080FB004700DE0094E0A80084E0A800FF
:10D960001600370095C0BF00610060009500A80058
:10D970008500A8001100370097C0BF004300DE00FB
:10D98000610060009760A8008760A8000B00370066
:10D9900097C0BF004400DE00610060009780A800CF
:10D9A0008780A800050037008F81E9004210200021
:10D9B000F1332000A0C32A00972F07000080FA004F
:10D9C000000006000200FA00F0BF9F00E30F5000C5
:10D9D0001600320006003C00E10F50000D0032003E
:10D9E00010003C000000E000080032001600370084
:10D9F000E90F50000B003200EA0F50000E00320019
:10DA0000E40F500010003A000B00370084C0BF0044
:10DA10000700370084C0BF000080FB004700DE0025
:10DA20000E00370085C0BF000500370087C0BF006B
:10DA30004300DE000200370087C0BF004400DE0064
:10DA400061006000050037008F81E900421020006E
:10DA500011372000A0C32A006F2F07000080FA00B2
:10DA6000000006000200FA00F0BF9F00E30F500024
:10DA70002700320006003C00E10F50001300320086
:10DA80001B003C000000E0000800320032003700BC
:10DA9000E90F500016003200EA0F50002400320057
:10DAA000E40F50002C003A002100370084C0BF0072
:10DAB0004300DE0061016000E1C06000C308DD00DA
:10DAC00084C0BF000034A1000600370084C0BF003E
:10DAD0000080FB004701DE00C708DD0084C0BF00F6
:10DAE0000074A1000140700084E0B7001F003700FF
:10DAF00085C0BF0061016000E1C0600085C0BF005B
:10DB00000004A1000140700085E0B7001700370055
:10DB100087C0BF004300DE0061016000E1C060001B
:10DB2000C308DD0087C0BF000034A1000700370034
:10DB300087C0BF004400DE0061016000E1C06000FA
:10DB4000C408DD0087C0BF000044A1000140700090
:10DB500087E0B700050037008F81E9004210200000
:10DB6000613B2000A0C32A002B2F07000200780091
:10DB70000080FA00000006000200FA00F0BF9F00DB
:10DB8000E30F50001400320006003C00E10F50008B
:10DB90000D0032000E003C000000E00008003200E2
:10DBA00011003700E90F500007003200EA0F500063
:10DBB00009003200E40F50000B003A000800370063
:10DBC00004C1BF000D00370010C1BF000B003700BB
:10DBD00012C1BF00090037001EC1BF000700370097
:10DBE00020C1BF00050037008F81E90042102000EE
:10DBF00091422000A0C32A00072F07004400DE0046
:10DC000063006000E10F5000090032000600390097
:10DC1000E20F500008003200E30F500007003A0006
:10DC2000001020000500370010002000030037001E
:10DC30008000200001003700000420000080FA006E
:10DC400000000600EF02B000889FBE008A9FBE0061
:10DC50008C9FBE008E1F780080B79F0092B79F00F8
:10DC6000A3B79F00B1B79F006000B8006011B80073
:10DC7000C0A79F00D1A79F00E2A79F00F3A79F0026
:10DC800061FC2F008F8040006A80400022C52A007E
:10DC900007000900321878000001B1008FB6970024
:10DCA000EC8F560004003600FA814000421020003C
:10DCB000211020000F003700E88F560002003C00C2
:10DCC0000D007800020037000D8046007100500002
:10DCD0004200DD00C1E22100608078000018A3004E
:10DCE00006003A0000FE2F008F0140003210200095
:10DCF00061102000A0C32A00C72E07003FB697007E
:10DD00000C00E00012003200E30F56001000320059
:10DD1000E60F56000E003200E90F56000C003200EC
:10DD2000E10F46000A003200E20F46000800320010
:10DD3000E30F460006003200E40F46000400320004
:10DD4000FA81570052102000B1102000E9FF37007F
:10DD50000C00E000150035001FB49700AFB4970029
:10DD60006055B8000007EB0009003700A400200050
:10DD7000050020006033B8000800BE000A01BE00A4
:10DD8000D6CA07000205BE000004BE000E07E80068
:10DD900069001600800F5700F4FF3500C8A79F00E8
:10DDA000D9A79F00EAA79F00FBA79F00E88F560016
:10DDB00083003C008040EB000D00780005FE07006A
:10DDC0003FB097000000E000510035004FA49700DD
:10DDD000DFA497006FA59700FFA59700502E0700BE
:10DDE0006011B8000040E10001C8E10002D0E1008C
:10DDF00003D8E100130039004FA49700DFA4970077
:10DE00006FA59700FFA59700452E07006011B80089
:10DE100004F02F00F50F20006033B800AFCA0700F0
:10DE20000040E10001C8E10002D0E10003D8E100B8
:10DE300004003E000006EB0001FD2F008F8640002D
:10DE40000600370082FC2F008F01410012102000D5
:10DE5000D1112000A7FF37000C06E8004FA497005F
:10DE6000DFA497006FA59700FFA597002C2E070051
:10DE70003D01BE00C2B79F00D3B79F008001EB00F9
:10DE8000E3B79F00F3B79F000001EB004FB297008C
:10DE9000DFB297006FB39700FFB397008FCA0700F8
:10DEA000F4FF2F00050020006033B8008BCA070084
:10DEB0000040E10001C8E10002D0E10003D8E10028
:10DEC000E5FF3E004FA49700DFA497006FA59700E1
:10DED000FFA59700122E07006011B8004FB29700FF
:10DEE000DFB297006FB39700FFB397007BCA0700BC
:10DEF0000203BE000002BE000800BE000A01BE0010
:10DF00001ECB07000205BE000004BE000B00370058
:10DF10000086EA001FB09700AFB09700E10F400005
:10DF2000E08F580004003600FE81570012102000D8
:10DF3000711220006FFF37000004BE000FB0970081
:10DF40008C007800C9FD07000FB09700B0A79F00B4
:10DF5000E20F50000F00320005003C000000E0001E
:10DF600008003200E10F500010003A0007003700AF
:10DF7000E30F500009003200E40F50000B003A009C
:10DF80000800370018088800790037006808880002
:10DF9000770037007808880075003700D8088800B7
:10DFA00073003700E80888007100370063FC2F0019
:10DFB0008F81410042102000014D20004DFF3700AD
:10DFC00011C0B3000D00780082FD07003FB097003C
:10DFD0000000E0004D0035004FA49700DFA497003B
:10DFE0006FA59700FFA59700CD2D07006011B80021
:10DFF0000040E10001C8E10002D0E10003D8E100E7
:10E00000150039004FA49700DFA497006FA5970073
:10E01000FFA59700C22D07006011B80004F02F0083
:10E02000F5FF2F00F60F2000070020002BCA070085
:10E030000040E10001C8E10002D0E10003D8E100A6
:10E0400005003E000007EB0000FD2F000F00400020
:10E0500080BF9F000600370081FC2F008F814000A9
:10E0600012102000A113200022FF37000E07E80045
:10E070004FA49700DFA497006FA59700FFA5970016
:10E08000A72D07000FB997003206BE0082BF9F0080
:10E090000C01BE00E4C907000002BE006033B800F6
:10E0A0000800BE000A01BE00B4CA0700F4FF2F003A
:10E0B000F5FF2F006033B8000400E1000588E1009F
:10E0C0000690E1000798E100E8FF3E004FA49700AA
:10E0D000DFA497006FA59700FFA59700902D07007C
:10E0E0000002BE006033B8000800BE000A01BE0096
:10E0F000A2CA07000C02BE006033B8009FCA070026
:10E100000205BE000004BE00030037000087EA00DD
:10E110001FB49700AFB497000FB097008E0078003F
:10E1200052FD07000800BE000FB19700B2A79F0084
:10E13000E90F510003003200EA0F510007003A00D6
:10E14000030037006808880071088800080037005D
:10E15000D8088800E10888000500370063FC2F001C
:10E160008F81410042102000A14F2000E1FE3700C6
:10E170000FB097006011B80087FD07004F077800C7
:10E180004F06BE004F05BE004F04BE00EF02B100B7
:10E1900000000600E80F50000200340000004000BC
:10E1A00071005000C200DD00C0E221006100780073
:10E1B00061006000000006000200FA00F0BF9F004E
:10E1C0000001BE00EC0F5000040036008F81E90012
:10E1D00042102000E11920000C003700E80F500029
:10E1E0000200340000004000710050004200DD00D9
:10E1F000C1E22100608078000018A30005003A0009
:10E200008F81E90032102000211A2000A0C32A00CB
:10E21000812D0700E30F51002000320006003C0072
:10E22000E10F51001100320016003C000200E00036
:10E230000800320025003700E90F51000B003200C2
:10E24000EA0F510015003200E40F51001F003A00A0
:10E2500018003700C718DD0005C1BF000074A10019
:10E260000140700005E1B7001C003700C718DD0051
:10E2700011C1BF000074A1000140700011E1B7009E
:10E2800016003700C718DD0013C1BF000074A100DD
:10E290000140700013E1B70010003700C718DD001F
:10E2A0001FC1BF000074A100014070001FE1B70052
:10E2B0000A003700C718DD0021C1BF000074A100AB
:10E2C0000140700021E1B700040037008F81E900B0
:10E2D00042102000511C2000CCFF37000080FA00C3
:10E2E000000006008000EB00B3FF370011002000A3
:10E2F000B1FF37000400FA00E0BF9F000102780080
:10E30000F2BF9F0000017800EC0F500004003600BF
:10E31000E481570042102000812A200007003700C6
:10E32000FFB997000300E900E60F50000500360032
:10E330008F81E90022002000912A2000A0C32A003A
:10E34000352D0700E80F510002003C000200780064
:10E35000020037000200410071005000C200DD00E1
:10E36000A0E2210084307800E30F51003100320038
:10E3700006003C00E10F51001700320022003C0073
:10E380000200E0000800320041003700E90F5100B0
:10E390001D003200EA0F510032003200E40F51003C
:10E3A0003B003A002F00370067C061004400DD00E9
:10E3B000510A200091407800F2C8B30082C060008A
:10E3C00080C0700001007800A5E0B7008460A9005B
:10E3D0009460A8003200370067C061004400DD008F
:10E3E000710A200091407800F2C8B30082C060003A
:10E3F00080C0700001007800A7E0B70084E0A900A9
:10E4000094E0A8002600370067C06100810A200060
:10E410009140780082CFB30082C0600080C070005D
:10E4200001007800A8E0B7008500A9009500A800C9
:10E430001B00370067C061004400DD00110B2000A5
:10E4400091407800F2C8B30082C0600080C07000C4
:10E4500001007800B1E0B7008760A9009760A800CC
:10E460000F00370067C06100210B20009140780049
:10E4700082CFB30082C0600080C0700001007800CD
:10E48000B2E0B7008780A9009780A8000400370099
:10E49000E481570042102000D12E2000A7FF370052
:10E4A0000080FA00000006000200FA00889FBE000B
:10E4B0008A1F7800C0BF9F000204BE0001057800DB
:10E4C00000017800EC0F500004003600E88157008E
:10E4D00042102000210C20000C003700E80F5000F3
:10E4E0000200340000004000710050004200DD00D6
:10E4F000C1E22100608078000008A30005003A0016
:10E50000E881570022102000610C2000A0C32A00DF
:10E51000C12C0700E80F510002003C000200780007
:10E52000020037000200410071005000C201DD000E
:10E530000380E800A4E22100840040001110A00044
:10E540001100A100E80F5100050034006680410071
:10E55000040040001000A1001120A00001003700BD
:10E560001120A100020078006BFB07008A007800F0
:10E570000801BE004FB89700B2FD07008000EB0015
:10E580004FB897008CFB07008000EB004FB8970056
:10E59000D4FB07004F0578004F04BE000080FA004E
:10E5A000000006000200FA00F0BF9F008000780023
:10E5B000EC0F5000050036008F81E900421020006A
:10E5C000E1152000A0C32A00932C0700E80F50009B
:10E5D0000200340000004000710050004201DD00E4
:10E5E0000280E800A3E22100030040001010A10017
:10E5F0001000A000E88F50000300340066004100C6
:10E60000030040001000A0000080FA000000060097
:10E6100090089000E0019000018140006281790043
:10E620008100E9001108980002007800000006004F
:10E630000200FA00889FBE00800478000104780080
:10E640000000E00005003A00000028000100E000A2
:10E65000620035000900780060003700010378008F
:10E660000100E00001003D000103EA00090078001C
:10E670000900E00001003D000900EA00010024005B
:10E680000800E00050003200CF80DE0066815700B5
:10E69000811F7800110009004688D8000109780020
:10E6A000CF007800DFB89700610AB800C021DD0014
:10E6B00002002000809FBE00110009004699D8008A
:10E6C000000178004F00BE0002027800800278004E
:10E6D00040A8DE00CF80DE008080CF000100E00097
:10E6E0000300320000022000010150000400370046
:10E6F0000281CF000200E000010032007001110031
:10E70000EC0151000A003B00C22820000300200059
:10E710000400BE0044C80700440BDD004C00DE00CE
:10E7200000007300CC88DE008000780022003700F3
:10E730001000200001002000020378000603E90019
:10E74000030033000000400081804800FBFF3700D9
:10E750000000520081805A00680151000201E90066
:10E76000030033008180D1000080D300FBFF37001D
:10E770007F0360004319DD004580DE000001410099
:10E780000201410021FC290062827800030220007E
:10E790000680510000A2B9000281E8006280780082
:10E7A0000680B9000402400085824800110009007B
:10E7B000432AD800800078000800E00002003D00F5
:10E7C00000002800810050000900E0000200340031
:10E7D00001007800010037000100EA004F04BE008C
:10E7E0000080FA0000000600800078000000E000D1
:10E7F0000C003D0002002C00820F500003003D0081
:10E8000000002800008040000400370010002800AD
:10E81000828F5000200034000100EA001700200021
:10E820000800370000002400808F500002003C00E8
:10E8300001007800020037000000280001005000AD
:10E840008003EB004781DE0000027800F407B2008D
:10E850000201410006EC29000008200004005000DD
:10E86000E2017B000380B9000281E80062017B00C5
:10E8700002A2B9000000420081804A004909DD007F
:10E880004700DE0000007100C788DE000700E000DE
:10E89000010032000000EA00000006000100240030
:10E8A00001004000D0FF37000100240001003700C4
:10E8B000C288DE00808F5000FDFF3C0080017800A0
:10E8C0000000EB0007003700010140000080D1008C
:10E8D000828F51000200350082815100010040000A
:10E8E000C288DE000100E000F7FF3A0000000600E9
:10E8F000889FBE008A1F7800800478000104780099
:10E90000010278008003EB005A0020001900370054
:10E910006420B800809FBE00110009004A88D8001A
:10E92000000278004F00BE00890078000400420019
:10E9300080814400840278008003EB000B003700E4
:10E940001103780013017800020053004240A9002F
:10E950000300340082087800860978001700200040
:10E960008502E8008180E8008381E800888F5200FA
:10E97000F3FF3900E10F5200E5FF3E000700E00021
:10E98000E9FF3A004F0578004F04BE000000060082
:10E99000889FBE008A1F7800000578001CFF0700D2
:10E9A000800478000A00780019FF0700000478004E
:10E9B0000A00780016FF0700000278000981440071
:10E9C000880044008001EB00050037004A009000F9
:10E9D000613178008301E8000281E8008180E8006D
:10E9E000848F5100F9FF39004F0578004F04BE00B5
:10E9F00000000600889FBE008A1F7800000578008E
:10EA000003FF0700800478000A00780000FF070079
:10EA1000000478000A007800FDFE070080017800FD
:10EA200008044400898044000001EB000400370022
:10EA30004A009000E83078000201E8008180E80098
:10EA4000830F5100FAFF39004F0578004F04BE00D4
:10EA500000000600889FBE008A9FBE0080057800E7
:10EA6000EBFE0700800478000B007800E8FE07004A
:10EA7000000478000B007800E5FE07000005780030
:10EA80000B007800E2FE0700800278004B00900047
:10EA90008A0045006102780089844400080144002E
:10EAA0008001EB0007003700CB0090006280780007
:10EAB0000000420080B478008301E8008984E80007
:10EAC0000281E800858F5100F7FF39004F05BE0035
:10EAD0004F04BE0000000600889FBE008A9FBE0053
:10EAE00080057800CAFE0700000578000B0078005A
:10EAF000C7FE0700800478000B007800C4FE070002
:10EB0000000478000B007800C1FE070000027800C6
:10EB10000A05450089844400080444008001EB0094
:10EB2000090037004B009000E90078006801780088
:10EB300082804000013578008301E8000A85E80002
:10EB40008984E8000884E800848F5100F5FF3900CB
:10EB50004F05BE004F04BE0000000600889FBE00A7
:10EB60008A9FBE0080057800A9FE07000005780096
:10EB70000B007800A6FE0700800478000B007800E8
:10EB8000A3FE0700000478000B007800A0FE070039
:10EB9000000278000A054500898444000804440006
:10EBA0008001EB00090037004B009000E90078007D
:10EBB0006801780082805000013578008301E80008
:10EBC0000A85E8008984E8000884E800848F510001
:10EBD000F5FF39004F05BE004F04BE0000000600DF
:10EBE000889FBE008A9FBE008C1F78008005780039
:10EBF00087FE0700000578000B00780084FE070000
:10EC0000800478000B00780081FE07000004780083
:10EC10000B0078007EFE0700000678000A0345001E
:10EC200089824400080244008003EB000900370099
:10EC30004B00900065017800E40078000191B90074
:10EC4000023378008703E8000683E8008582E80045
:10EC50000482E8008C8F5300F5FF39004F067800DE
:10EC60004F05BE004F04BE0000000600889FBE0096
:10EC70008A9FBE008C9FBE008E1F780080057800A2
:10EC800063FE0700000578000B00780060FE0700B7
:10EC9000800478000B0078005DFE07000004780017
:10ECA0000B0078005AFE0700000778000A064500AE
:10ECB00009854400880444008006EB0016003700F4
:10ECC0004B0490006A007C006102B90069007C007E
:10ECD0006101B9000A85E8008984E8000000E000CD
:10ECE000060032000400BE00EDC6070000367C00BE
:10ECF0008D06E8000C86E80007003700230020009E
:10ED0000F305980070814500710029000B00780020
:10ED10009D1B0700020037008E8F5600E8FF390068
:10ED20004F0778004F06BE004F05BE004F04BE00DF
:10ED300000000600889FBE008A9FBE008005780004
:10ED400033FE0700000578000B00780030FE070056
:10ED5000800478000B0078002DFE07000004780086
:10ED60000B0078002AFE0700098344008802440053
:10ED70000A0245008003EB000B0037004B019000B6
:10ED8000E6017900E5007900838F5000010034002E
:10ED900083007800013279008703E8000683E800E9
:10EDA0008582E8000482E800808F5300F3FF390079
:10EDB0004F05BE004F04BE0000000600889FBE0045
:10EDC0008A9FBE008005780011FE070000057800CC
:10EDD0000B0078000EFE0700800478000B0078001E
:10EDE0000BFE0700000478000B00780008FE070007
:10EDF00009834400880244000A0245008003EB00B6
:10EE00000B0037004B019000E6017900E500790026
:10EE1000838F500001003D008300780001327900AB
:10EE20008703E8000683E8008582E8000482E800A2
:10EE3000808F5300F3FF39004F05BE004F04BE0022
:10EE400000000600889FBE008A9FBE008C9FBE0007
:10EE500080047800EEFD07000005780009007800C6
:10EE6000EBFD07000006780009007800E8FD0700C8
:10EE7000800578004904900009007800E4FD07004F
:10EE80000000400060047C0009007800E0FD0700FD
:10EE90008006780000022000800F540005003C002E
:10EEA0000B8345008C0146006022B8008003EB0014
:10EEB0000D003700C90090000A0045000100400025
:10EEC0000008EB001200370063807800668178004C
:10EED0000280B90004024000858248008703E800F0
:10EEE0000683E8008381E800C90090008D8F5300FD
:10EEF000F5FF39000A0045000804E900030033006B
:10EF00008582D1000482D300FBFF370004B0780073
:10EF10004F06BE004F05BE004F04BE0000000600B5
:10EF2000889FBE008A9FBE008C1F78000004780076
:10EF3000B7FD07008004780008007800B4FD0700E2
:10EF40008005780008007800B1FD07000005780012
:10EF500008007800AEFD0700000678000800780081
:10EF6000ABFD0700000378000000E0002400320041
:10EF7000C800900009804400608078006102B900F8
:10EF80008B85450080B578000A05450000B57800FE
:10EF90000900E8008001400017002000010178000E
:10EFA0000F003700E30079000B004100908F500004
:10EFB00001003D0001087800480090000000450075
:10EFC000908F500001003400010878006108B900FA
:10EFD00004024000858248008703E8008381E8003E
:10EFE000868F5300EFFF39000C04460002044400F2
:10EFF0006131B8000400BE0029C60700000C78008B
:10F000004F0678004F05BE004F04BE00000006000A
:10F01000889FBE008A9FBE00800478007CFD0700A8
:10F02000800578000900780079FD07000005780068
:10F030000900780076FD07000004780009007800D8
:10F0400073FD0700000278000000E00016003200A7
:10F05000880344008A0245000B814500F8FF270021
:10F06000060028008001EB000D00370049009000E9
:10F07000E2007800888F500002003D008332780063
:10F0800001047800868F500003003400490090008E
:10F0900083337800010378008301E8000281E800EF
:10F0A000848F5100F1FF39004F05BE004F04BE00B0
:10F0B00000000600889FBE000004780054FD070091
:10F0C000800478000800780051FD07008000780077
:10F0D00009814400480090000000410004FE070040
:10F0E0004F04BE0000000600E8874700889FBE006E
:10F0F0008A9FBE008C9FBE008E1F7800000678009D
:10F1000043FD0700800578000C00780040FD0700F3
:10F11000000578000C0078003DFD070080047800B1
:10F120000C0078003AFD0700000478000C0078001D
:10F1300037FD070080BF9F008B854500EBB79F0020
:10F140000A07450089864400880444000000EB005B
:10F15000F0B79F001F0037004C0490006E007C0049
:10F160006102B9006D007C006101B90069007C009A
:10F170006105B9000E87E8008D86E8008984E80003
:10F180000000E0000C0032000400BE00A6C507002D
:10F190000A01BE00C2C507006FB1970000317C00B4
:10F1A0007FB097000000E800F0B79F000281E80000
:10F1B000E2B79F0007003700230020007306980085
:10F1C00070014600710029000C0078006E1A0700DB
:10F1D00004003700FFB097000FB99700828F5000EE
:10F1E000DDFF39004F0778004F06BE004F05BE0017
:10F1F0004F04BE008F00B10000000600889FBE00D3
:10F200008A9FBE008C9FBE008E1F7800000678008B
:10F21000FFFC0700000578000C007800FCFC0700EC
:10F22000800478000C007800F9FC070000047800E6
:10F230000C007800F6FC0700000778008985440080
:10F24000880444000A0545008006EB0009003700E9
:10F250004C049000E9007C006B007C00F4FC07008B
:10F2600000357C008D06E8008B85E8008984E80085
:10F270000A85E8008E8F5600F5FF39004F077800A9
:10F280004F06BE004F05BE004F04BE000000060042
:10F29000889FBE008A9FBE008C9FBE0080057800BC
:10F2A000DBFC0700800478000B007800D8FC070026
:10F2B000000478000B007800D5FC07008006780079
:10F2C00008054400898444000006EB00070037006D
:10F2D0004B0490006A007C0043FD070080347C00F2
:10F2E0000C06E8000A85E8008984E8008D0F5600C6
:10F2F000F7FF39004F06BE004F05BE004F04BE00A9
:10F3000000000600889FBE008A9FBE008C9FBE0042
:10F3100080057800BEFC0700800478000B007800B0
:10F32000BBFC0700000478000B007800B8FC070065
:10F330008006780008054400898444000006EB003C
:10F34000070037004B0490006A007C0053FD070063
:10F3500080347C000C06E8000A85E8008984E80017
:10F360008D0F5600F7FF39004F06BE004F05BE0057
:10F370004F04BE00000006000C00FA00889FBE008B
:10F380008A9FBE008C9FBE0000047800A0FC07008E
:10F3900080057800080078009DFC07008004780054
:10F3A000080078009AFC0700480590008984440012
:10F3B0000000400060047D000800780037FD070071
:10F3C0006101B90082BF9F0093BF9F0069007D006B
:10F3D0006101B900E2B79F00F3B79F000800780011
:10F3E00001FD07006101B900C2B79F00D3B79F00BC
:10F3F00009004500100090006106B9008B854500AA
:10F400006FB19700FFB197000FB897009FB89700B2
:10F4100005C507000004BE000C01BE004FB09700F8
:10F42000DFB0970000C507000004540081845C0031
:10F43000C149DD004F44DE0008847100CFCCDE00FE
:10F4400088357D000B0545000C01BE000FB8970004
:10F450009FB89700F4C407000004BE006FB1970086
:10F46000FFB197004FB09700DFB09700EEC40700E0
:10F4700008044000898448004148DD004F44DE0014
:10F4800008047000CFCCDE00180598004F06BE00BF
:10F490004F05BE004F04BE000080FA0000000600C9
:10F4A000889FBE008A9FBE008C9FBE0080057800AA
:10F4B00057FC0700800478000B00780054FC07001C
:10F4C000000478000B00780051FC070080067800EB
:10F4D00008054400898444000006EB00070037005B
:10F4E0004B0490006A007C00EFFC070080347C0035
:10F4F0000C06E8000A85E8008984E8008D0F5600B4
:10F50000F7FF39004F06BE004F05BE004F04BE0096
:10F5100000000600889FBE008A9FBE008C9FBE0030
:10F52000000478003AFC0700000578000800780025
:10F5300037FC0700800578000800780034FC0700DD
:10F54000800478000800780031FC07000002780091
:10F55000C802900009804400E0847A000B804500D6
:10F56000008042008000EB00040037008100E800CA
:10F570000080E800848F500048003E001000E0004A
:10F58000FAFF3A0001804500000040000080420080
:10F590000080E800810378008703E800848F53002F
:10F5A000090036000100E000400032000100E900DF
:10F5B0000A014500890F5000400039000000D100C9
:10F5C00000B17A00430037003000E000F2FF320063
:10F5D0000003EB0006047800860678002C0020006B
:10F5E0008681430006017800040037000201E8002C
:10F5F0008301E800840F5100080031001100090068
:10F600008481D8008000FD000B0040000000400015
:10F61000050040001000E000F4FF3A0086005100B1
:10F62000888F50000700340006004100811F7800D9
:10F63000110009000C00D80080067800CF00780087
:10F6400001047800840F51001000310082814300D2
:10F65000040037000201E8008301E800840F510034
:10F660000A003100110009008481D8008000FD00EB
:10F670000B00400000004000050040001000E000CA
:10F68000F4FF320002037800D5FF37000A0145007D
:10F69000890F54000B003D00080037000A004500A8
:10F6A000050040000008EB000A0037000A00450092
:10F6B000050040000088EB0006003700050041000F
:10F6C000FCFF37000D804300110009000480D800C2
:10F6D00001B17A004F06BE004F05BE004F04BE00C8
:10F6E00000000600C0FA880000000600C2FA800090
:10F6F000502526000091B9009061230002004000CF
:10F70000C0FA880000000600889FBE0080047800D0
:10F71000BFFB07000004780009007800BCFB07006D
:10F7200000027800C0FA8000080444008001EB0069
:10F730005625260095612300060037000680B90093
:10F740000080420049019000003479008301E80004
:10F750000884E800848F5100F8FF3900C0FA88005F
:10F760004F04BE00000006000080FB00C300DE0066
:10F77000B27F240002814000C308DD000100500078
:10F78000110020008008DD0012C970000000060092
:10F7900010FA800021FA800061014000E0814800F9
:10F7A00012FA880023FA880000302A002100200085
:10F7B000800F5100818F590007003A00423FEF004F
:10F7C000443FEF00A17F240011407800E14F40004A
:10F7D000010032008048E800000006000001EB0054
:10F7E00011022100000120004727070061012000CD
:10F7F000807E24005527070076270700F03F8A0007
:10F800000000060020C0B300D7FF370031FA8000A7
:10F810008100E80031FA880000A62E00808F500099
:10F8200027003A00463FEF00403F8200E10F4000D2
:10F83000020032000000E800403F8A00A3F6070003
:10F840000000E00006003D00917F24001140780098
:10F85000E14F4000090032008048E800070037000F
:10F86000E8004000807E24000080400010417800C5
:10F87000E14F4100010032000248E80084C4BF00AB
:10F880000038A3000E003200D62507000000E0007B
:10F8900006003200503F8200E10F400008003200B5
:10F8A0000000E800503F8A0000000600603F820030
:10F8B000E10F4000020032000000E800603F8A00D3
:10F8C000000006008000780060042000808F500057
:10F8D0000B0039000000E800808F50000400360063
:10F8E00070004000808F500005003A000200370091
:10F8F00070C0B3009CFF370000C1B3009AFF07003F
:10F90000000006008000780020052000808F500055
:10F910000E003E000080E900808F50001A00310088
:10F92000A0022000808F50001F00390064004000BA
:10F93000808F50001000360070FC2F0000804000C7
:10F94000EC0F500018003E000D003700500520005D
:10F95000808F500004003E000000E900808F5000BE
:10F960000D0031000A00370060052000808F500034
:10F970000D003A000A003700F0C0B300070037005E
:10F9800080C0B30005003700E0C0B30003003700BB
:10F9900090C0B3000100370010C1B30072FF370000
:10F9A00000C1B30070FF070000000600889FBE0082
:10F9B0008A1F78000005EB001800200029002000B5
:10F9C00011D5800000D58000910F10003100360065
:10F9D00095003700E9007800E0FF2F00010050009B
:10F9E00001002000EF0F5000E08F580021003E0082
:10F9F000006001000F0037000E0037000D003700D7
:10FA00000C0037000B0037000A0037000B003700EE
:10FA10000C0037000B0037000C00370015003700D2
:10FA2000100037000B0037000C0037000F003700C4
:10FA30000E003700F0C0B3000D00370080C0B300E7
:10FA40000B003700E0C0B3000900370000C1B3006D
:10FA50000700370010C1B3000500370070C0B300C5
:10FA60000300370040C1B3000100370050C1B300AC
:10FA70003DFF070009007800A21AB40010009000B2
:10FA80008A0F500001003600000578000884E80065
:10FA9000E484440010D58000900F5400CDFF39005D
:10FAA0005E00370014D580008801440063017A00AD
:10FAB0004C10DE0001002000ED0F5000E08F5800D8
:10FAC00055003E00006001000D0037005200370075
:10FAD0001D0037000D0037001000370013003700FD
:10FAE000160037004C0037004B0037001800370075
:10FAF000150037001A003700240037001D003700BA
:10FB00008A0F54004800310043003700F0FF200006
:10FB1000000061007BFF07003F003700F0FF20007E
:10FB20000000610067FF07003B003700F0FF200086
:10FB30000000610073FF070003003700F0FF2000A2
:10FB4000000061005FFF07000884E8003300370011
:10FB50004410DD004480DE00000044000700370050
:10FB6000030042001000900066FF07006304440099
:10FB70002A003700F0FF2000000061008A0F5000CB
:10FB8000250036000005780023003700F0FF200034
:10FB900000006100010020007B005000E080580060
:10FBA000ED0F5000E08F58001B003E000060010088
:10FBB0000D0037000C0037000B0037000C00370039
:10FBC0000D0037000C0037000B003700060037002F
:10FBD0000B0037000C0037000B0037000C0037001B
:10FBE0000B0037000A003700A0C0B300090037003F
:10FBF000D0C0B30007003700C0C0B3000500370015
:10FC000020C1B30003003700B0C0B30001003700CB
:10FC100030C1B300D4FE07000804E80000D580001E
:10FC2000800F54009FFF39004F0578004F04BE003D
:10FC300000000600F17E240011407800E14F4000F2
:10FC4000010032008048E80058FF3700889FBE005E
:10FC50008A9FBE000004BE0000402000010020007A
:10FC600008054000898548000B0037000800BE00E9
:10FC700001130700F2FF2F00F30F2000820F500046
:10FC8000838F580002003200100020000600370069
:10FC900062044400E0844C008A0F54008B8F5C00A7
:10FCA000F2FF39000000EB004F05BE004F04BE001C
:10FCB000000006004A00FA00881F78008A9FBE00F4
:10FCC0008C9FBE0055FC2F000F8242000006BE0034
:10FCD00092BF9F00A3BF9F00E00F5100E08F59002B
:10FCE00005003A00D20220008000EB0004007800FA
:10FCF0006FC40700DC00370084017800D2022000C6
:10FD00001FB89700AFB89700F11207004FE89700AF
:10FD10000040E800C0EF9F001FB89700AFB8970001
:10FD20007E054000E0854800C600370001FB2F003B
:10FD30000F84400088017800520120000A00BE00B4
:10FD4000E31207001FE89700EF7097000140700072
:10FD500090EF9F002FE89700FF7097000140700020
:10FD6000A0EF9F003FE897008F7897000140700058
:10FD7000B0EF9F00FFE097008180FB000FE8970045
:10FD80004800DD0001007000BFC097008180FB00CB
:10FD900001004000F0E79F004800DE0080EF9F0078
:10FDA000DFE097008180FB006FE097004800DD00F6
:10FDB00001007000AFC097008180FB00010040008F
:10FDC000D0E79F004800DE00E0E79F00BFE097001B
:10FDD0008180FB004FE097004800DD0001007000CB
:10FDE0009FC097008180FB0001004000B0E79F00AA
:10FDF0004800DE00C0E79F009FE097008180FB0085
:10FE00002FE097004800DD00010070008FC09700D0
:10FE10008180FB000100400090E79F004800DE0069
:10FE2000A0E79F00FFD897008180FB000FE09700BC
:10FE30004800DD0001007000FF7897008180FB0022
:10FE400001004000F0DF9F004800DE0080E79F00D7
:10FE5000DFD897008180FB006FD897004800DD0055
:10FE600001007000EF7897008180FB0001004000E6
:10FE7000D0DF9F004800DE00E0DF9F00BFD8970082
:10FE80008180FB004FD897004800DD000100700022
:10FE9000DF7897008180FB0001004000B0DF9F0009
:10FEA0004800DE00C0DF9F009FD897008180FB00E4
:10FEB0002FD897004800DD0001007000CF78970030
:10FEC0008180FB000100400090DF9F004800DE00C1
:10FED000A0DF9F00FFD097008180FB000FD8970024
:10FEE0004800DD0001007000BF7897008180FB00B2
:10FEF00001004000F0D79F004800DE0080DF9F0037
:10FF0000DFD097008180FB006FD097004800DD00B4
:10FF100001007000AF7897008180FB000100400075
:10FF2000D0D79F004800DE00E0D79F009FD0970009
:10FF30008180FB002FD097004800DD000101700098
:10FF4000BFD097008180FB004FD097004800DD00B4
:10FF5000810170002800900000004100E08049000D
:10FF600090D79F004801DE00A2D79F00B1D79F0025
:10FF70004808DE00C0D79F00DFC897008180FB00E3
:10FF80006FC897004800DD0001017000FFC89700AE
:10FF90008180FB000FD097004800DD0081017000D8
:10FFA0001F98970000004100E0804900D0CF9F00DB
:10FFB0004801DE00E2CF9F00F1CF9F004808DE003D
:10FFC00080D79F009FC897008180FB002FC89700B3
:10FFD0004800DD0001017000BFC897008180FB0070
:10FFE0004FC897004800DD008101700018007800BC
:10FFF00000004100E080490090CF9F004801DE00F2
:020000040001F9
:10000000A2CF9F00B1CF9F004808DE00C0CF9F0065
:10001000FFC097008180FB000FC897004800DD00FB
:10002000010070009F7897008180FB000100400074
:10003000F0C79F004800DE0080CF9F006E0545009E
:10004000E0854D0000402000010020001FB997000E
:10005000AFB997000200400083804800800F550030
:10006000818F5D0031FF390053FC2F000F84410068
:100070008042EB0062CC7200E5C79F000C00BE001E
:10008000F2FE07000000E000100032000C00BE008D
:10009000621207000D003700C1FA2F008F80400068
:1000A00008007800B0587800B05878009048780080
:1000B0006F919700FF9197000C00BE006E12070031
:1000C00062064600E0864E00630444006E805700DE
:1000D000800F5400F0FF3A004F06BE004F05BE00EF
:1000E0004F0478000080FA00000006002E00FA009D
:1000F00023FD2F008F814100D2022000F411070060
:100100009FA897000110A2000100EA000100700002
:100110004F00DE00610010000080FA0000000600C1
:100120001600FA00889FBE008A9FBE000005BE0030
:100130007E044000E084480009003700FE8157003B
:10014000520120000800BE00E11107000FE89700EF
:100150000008A3000A003A006E044400E0844C004A
:1001600000402000010020000A0040008B80480071
:10017000800F5400818F5C00F0FF39006044B800AC
:100180000800BE004F05BE004F04BE000080FA000C
:1001900000000600817E2400F20F2000114861005B
:1001A0009140900011409800A37E240093006100CC
:1001B000214098009341900033409800C17E240074
:1001C0001101610042409800914090005140980018
:1001D000B17F24009140780061409800C17F2400E5
:1001E0009140780071409800D17F240091407800C0
:1001F00001489800E17E2400914078001148980061
:10020000F17E24009140780021489800017F24006D
:100210009140780031489800117F24009140780087
:1002200041489800217F240091407800514898006F
:10023000317F24009140780061489800617F24005C
:100240009140780071489800717F240091407800B7
:1002500001509800517F240091407800115098007F
:10026000917F24009140780021509800A17F2400C4
:100270009140780031509800000006001A00FA0002
:10028000881F78008A9FBE000001EB001102210048
:10029000000120009C24070061012000807E2400D2
:1002A000AA240700CB240700E17F2400910F50000F
:1002B00004003200820120008000EB00807E2400D8
:1002C000FBC2070040C7BF000018A30003003200B4
:1002D00010C0B30024FD07004027A900A07F240020
:1002E0001004E00004003A00817E2400005A20003F
:1002F000910F1000650036006232EF000004EB0041
:100300006212E20006003A001000200026250700D5
:100310000804E80000712200800F5400F8FF3A0042
:1003200011938000F0282000808F50005700340087
:1003300000C02300110020006CFF07000000E00057
:1003400007003A00000024001100200067FF0700AA
:100350006011B8000000E0001E00320014003700F9
:1003600000C02300110020006DFF07000005BE0043
:10037000E00F5000E08F58001B003A0000002400FE
:100380001100200059FF07000000E00008003A00BB
:1003900002C02300130020000000240011002000F0
:1003A00044FE0700EA0124001B0020000E00370075
:1003B000000024001100200059FF07000005BE00C6
:1003C000E00F5000E08F580007003A0002002400C0
:1003D0001300200000C023001100200035FE07009C
:1003E000EAC123001B0020007C845700080078002D
:1003F00068FF07000D00370001FE2F008F804000CE
:1004000008007800B0587800B0587800904878001C
:100410000FB197009FB197000A00BE009611070028
:1004200062054500E0854D00630444006780570085
:10043000800F5400F0FF3A00020024001300200057
:10044000820F5500838F5D0004003A0002C0230034
:10045000130020000A00BE000700370000402400FF
:1004600011002000800F5500818F5D0003003A00CD
:1004700000C02300110020000EFE070082012000B2
:100480008000EB00807E240089C20700E17E24000A
:1004900011407800E14F4000010032008048E80040
:1004A0004F05BE004F0478000080FA0000000600EF
:1004B0001C00FA00889FBE008A1F780000057800A3
:1004C00050019000E001900013EC070008C02300E9
:1004D000190020000800BE00E710070080B79F0049
:1004E00091B79F00E3FD2F008F8141003200200073
:1004F0008380E8000A0078008DEA07007FA8970053
:10050000E30F500024003A0062044400E0844C00F1
:100510000040240011002000800F5400818F5C00F7
:10052000ECFF3A007C8457000800780019FF0700B0
:10053000E3FD2F008F8141005201200088007800E8
:100540000A0078007AEA0700820120008000EB00B0
:10055000807E240056C2070000C023001100200046
:10056000BAFD07000000E0000300320000C02300D5
:1005700011002000291107000000240011002000B4
:10058000B2FD07000000E00003003200000024007C
:1005900011002000211107004F0578004F04BE0014
:1005A0000080FA00000006008000EB0001089800BF
:1005B000710098002118980020019000010978002E
:1005C00030019000020141004000900038C2370025
:1005D0002001900012037800150020002300200065
:1005E000090037006482410062807900810F500069
:1005F00003003A00030041001000900000000600D4
:100600008582E80084017800868F5200F5FF39006A
:10061000000005000400FA0080089000E1BF9F0080
:10062000F0009000F1BF9F0043002000648157005C
:10063000A1002900541507000080FA000000060000
:10064000889FBE0000047800E1FF07008004780066
:100650000000E00012003200780090000008A300C3
:1006600005003200700144002300200081002900B1
:100670000800780044150700090C98000080EB0082
:10068000100C9800780090000000A0007004980002
:100690000018A3000200320008007800DDFF070008
:1006A000090078004F04BE0000000600889FBE00CD
:1006B00080047800020478006119B800F10F51003D
:1006C000E08F59005B003E0002600100110037001E
:1006D00012003700130037001400370015003700F0
:1006E000170037002A0037002D0037002E00370092
:1006F0002F00370030003700330037003600370056
:10070000390037003C0037003F0037004200370017
:10071000440037000809DD00490037000889DE0081
:10072000470037000881400045003700088150002D
:10073000430037000888B900000178004000370006
:100740000800E0000E003A0020C027000000E00092
:1007500003003200880078000900780029FC0700B7
:1007600023002000F30498007081440071002900E8
:1007700009007800041507000801780030003700F0
:10078000110009008800D800000178002C00370013
:10079000110009008800D800010178002800370006
:1007A00008817000260037000881680024003700A7
:1007B00008816000220037000001EB00888F5000A4
:1007C0001F003A001D0037000001EB00888F500029
:1007D0001B003200190037000001EB00888F500029
:1007E00017003400150037000001EB00888F50001F
:1007F00013003500110037000001EB00888F500016
:100800000F003D000D0037000001EB00888F500005
:100810000B003C00090037000100E00007003A002F
:10082000020037000100E000020032000800E00092
:1008300002003A000001EB00010037001200200026
:10084000020078004F04BE00000006000600FA0017
:10085000889FBE000004780020029000800A90006B
:1008600005814200E2047A004C48DE0001002000CD
:10087000EE0F5000E08F5800F6003E0000600100CF
:100880000E0037001100370019003700270037002D
:10089000320037003D0037004F003700730037004B
:1008A0008A003700990037009C003700C2003700EB
:1008B000CF003700D5003700DF0037007800900008
:1008C0000000A10070049800E20037006801900069
:1008D000180890000000E800100C9800000040008C
:1008E000C448DD00C488DE0001307900C400370050
:1008F000E8019000980890008100E800110C980031
:10090000818040000808900028019000000040000D
:10091000020040001000900080B0790008089000AC
:100920000080E800000C9800CA003700E801900041
:10093000980890008100E800110C98008180400028
:10094000F0FF20000080640048019000000040009B
:100950006001790082B07900A90037001809900081
:10096000F0FF20000080640048029000000040007A
:10097000E801900082004100E181790003307A00B3
:100980000201E900120C98009D003700F0FF2000E2
:10099000808164000200420010029000180890005C
:1009A00000004000E80090000101400012007800C3
:1009B000840F500003003900B5BF9F00C4BF9F00E3
:1009C0001300370003004000C80090000000400002
:1009D00060897800D1FF3700F0FF2000808164003B
:1009E0000200420010019000E800900018089000FA
:1009F000000040008080400071BA9700110078002C
:100A0000820F500011003900B5BF9F00C2BF9F0088
:100A1000D0BF9F00200020007004980063002000D9
:100A20006A81570061002900080078005614070009
:100A300020C027000000E000860032008000EB00AC
:100A4000080078006FFB07008200370003004000B9
:100A5000C80090000000400004B078001808900022
:100A60000080E900100C9800ACFF370018089000D7
:100A700000004000E8009000810140001301780070
:100A800009007800F00FB200E10F500007003200BB
:100A9000040039008000EB00E20F500009003A002A
:100AA000070037008200EA00060037008200780065
:100AB0000200E00003003D008200EA000100370070
:100AC0008280EA00810978004D003700E80090003C
:100AD000180890000000400060817800808040008D
:100AE000F1B897008981FB0008007800EFFE07004D
:100AF000980890008100E900110C980068019000AE
:100B000081804000803079003D0037004448DD009E
:100B10004480DE000080420082FF3700E800900041
:100B2000180890000000400060817800808040003C
:100B3000F1B897008981FB0008007800DBFE070010
:100B400000027800180890000080E900100C98005E
:100B50000400E000040032000988A3000A0032000B
:100B60000998A300080032002801900008089000AE
:100B70008000400001004100900190000400E0006E
:100B800002003A0007003700230020000808900008
:100B900000004000A8009000010040001090A0005C
:100BA00002003700010041001090A10008089000E9
:100BB000008041005BFF370002004200A00190006E
:100BC0001001900002014100480090000001410026
:100BD000F1FF2000818064008381410008007800DB
:100BE000E913070008089000630040004DFF37003C
:100BF000F1FF20008180640008007800E40A07000B
:100C0000080890000000E80046FF370068019000E7
:100C1000180890000000E800100C98000000400048
:100C2000880890008100E80001307900F0FF200082
:100C3000008064003BFF37001808900068019000B6
:100C40008000400061017900020C98000000E9007A
:100C5000100C98004F04BE000080FA00000006004F
:100C60000000FA00889FBE008A9FBE008C9FBE00D5
:100C700080057800010578008F0678000100780073
:100C800092C0070000047800630640006500400041
:100C90000000A100808747008D04780020C0270055
:100CA0000000E000030032008A0078000B007800AA
:100CB000D4FA070020002000F00598000B089000EF
:100CC000800C7800A84498006380440008017800F4
:100CD0008A00780083C007008C0178000901780041
:100CE000910029000B007800A71307008D077800FA
:100CF0004F06BE004F05BE004F04BE000080FA0044
:100D00000000060080007800201A9000F4014000E6
:100D10000001EB000800370001089000B30F10003D
:100D200004003A00710090000010A000F00098004C
:100D3000100005000201E800840F5100F6FF3900A1
:100D400000000500889FBE008A1F7800000478001C
:100D500001057800700090000020A0007004980049
:100D60008004EB000100E00004003A000D003700B1
:100D700008007800B5FE07008904E80078009000BC
:100D80000008A3000C0032000028A3000A00320073
:100D90008A8F5400F6FF3A000700370008007800F9
:100DA000AAFE0700780090000008A30002003200AD
:100DB0000028A300F9FF3A00780090000020A1006D
:100DC000700498004F0578004F04BE000000060034
:100DD000889FBE008A1F7800000478000105780013
:100DE000700090000020A000700498008004EB00C8
:100DF0000100E00008003A001B00370008007800FE
:100E0000C0FF07008904E8000000E0000A003A0083
:100E1000080078008DFE0700780090000008A3000D
:100E2000160032000028A300140032008A8F5400FC
:100E3000F2FF3A0011003700780090000010A00087
:100E40007004980008007800F2FD07000E003700DB
:100E500008007800ABFF07000000E000F6FF3A0052
:100E60000800780079FE0700780090000008A300D1
:100E7000020032000028A300F5FF3A00780090003D
:100E80000020A100700498004F0578004F04BE00B8
:100E90000000060000017800700090000008A30028
:100EA0000B0032000018A30009003A00221890003D
:100EB0000000E0000300320002007800C4FF0700D9
:100EC00002003700020078009EFF070010000500B6
:100ED0000000050080017800201990000000EB0060
:100EE000EF0F510006003E00020041007400400078
:100EF00001B079000200E800A0199800100020005D
:100F0000000006000001780001037800A01990009D
:100F1000740240000000EB008302E9001400370077
:100F20008000E800B40F130010003A002519980063
:100F300081804000F4804000800178000502780044
:100F40000000400074004000010141000100500019
:100F500003003700123079008301E8000281E800C5
:100F6000848F5100FBFF390010000500010078005C
:100F7000830F5000EAFF3900000005008000EB00FD
:100F80002118980000000600000278009200780006
:100F90000100E000060035008DFD07008001EB0038
:100FA0000000E0000F003A00130020000D003700A1
:100FB00013002000F0FF2900808F50000900360048
:100FC000120190008001EB000000E800808F5000CB
:100FD00004003200940069000100EA000100700082
:100FE000CF01DE0003007800000006000400FA00D4
:100FF000881F7800000478008102780000002A0031
:10100000808F500003003A00080078001213070098
:101010007700370012007800980F500074003A00F3
:101020000282E800F0FF2500F1FF2F0005004000DC
:10103000E0804800EE0F5000E08F58006C003E004A
:10104000006001000E0037001A0037002100370051
:101050002B00370030003700350037002B003700F9
:1010600035003700400037004300370045003700A7
:101070004900370056003700580037005A00370043
:101080008381E900140078000001400084007800AA
:101090000002EB00040037002800900011317800B6
:1010A0000402E8000281E8008180E800830F52001A
:1010B000F9FF390020002000700498008080EB00C8
:1010C000080078005EFD07000000E00048003A00DC
:1010D0000E003700780090000010A1007004980006
:1010E000080078004BFD0700A0E127000000E000A9
:1010F0003F00320008007800CEFA07003C003700BD
:10110000780090000010A00070049800080078009B
:1011100040FD070036003700780090000008A3006B
:101120003300320008007800C8FD0700F7FF3700E1
:1011300020002000F4FF370094007800D1BF9F000A
:101140000800780063FF07000080FB00E0BF9F00FD
:101150004300200066815700B10029000800780094
:1011600089120700220037009400780008007800F8
:1011700064FF07001E0037000000EB00201C9800F1
:101180001B003700220190009400780008007800CE
:1011900093120700160037008381E90014007800DD
:1011A00000014000840078000002EB0004003700DA
:1011B00048009000113178000402E8000281E80044
:1011C0008180E800830F5200F9FF390008003700E2
:1011D000080078007609070005003700080078004D
:1011E000270907000200370008007800630907009C
:1011F0004F0478000080FA00000006000080FB0029
:101200004013880060C2BF000008A300FDFF320049
:10121000401380000080FB0000000600401F2000FB
:1012200090F9880000C0EB00F4FF070000C0EB005D
:10123000F2FF0700E14F400002003200321FE200DF
:10124000FAFF3A000080FB0000000600CDC2A800B3
:1012500000C0EB00E9FF3700CDC2A900EFFF070097
:1012600011002000E14F400002003200F7FF0700AC
:101270008000EB000100780000000600889FBE009F
:101280000004BE0040062000A0F9880000C0EB006A
:10129000DAFF0700E14F400003003A00341FE2008C
:1012A00025003200F9FF3700E24F400022003A00EB
:1012B000F10F20004113880060C2BF000008A300A6
:1012C000FDFF320040138000004C7800411388007D
:1012D00060C2BF000008A300FDFF32004013800081
:1012E000104498004113880060C2BF000008A300AA
:1012F000FDFF320040138000204498004113880015
:1013000060C2BF000008A300FDFF32004013800050
:101310003044980064044400E4845400E5FF3A003B
:1013200000C0EB00B5FF070000C0EB00B3FF0700F3
:1013300010002000010037000000EB004F04BE0049
:1013400000000600889FBE000004780081447800F9
:10135000B2FF0700E14F400015003A000940780055
:10136000A6FF0700E3CF440013003200092020004D
:1013700018407800A1FF0700184090000884E8009A
:101380009EFF07008984E900F9FF3A0000C0EB00E6
:101390009AFF070000C0EB0098FF070000C0EB00B9
:1013A00096FF07007F006000E50F5000020032004A
:1013B0000000EB0001003700100020004F04BE00C9
:1013C00000000600889FBE008A1F78000045780054
:1013D0000204BE000004E00006003D000A74A10003
:1013E0006011B80070C3B300F6FF0700E14F500072
:1013F00028003E0095FF070097FF0700F10F20002F
:101400000000E000240032000A4078000064A000E0
:101410007AFF07004848DE000100200077FF070040
:101420004048DE000100200074FF07004849DD004D
:101430004840DE0000007100C848DE006FFF070072
:10144000084078006DFF070050C9B3000A04E000AF
:10145000040032006E405000E84F55000100320099
:1014600010C0B30065FF0700A8C0B300EC4F5500E3
:1014700002003A0000C0EB0060FF070000C0EB0074
:101480005EFF07000004E00002003D000844E900A0
:10149000FAFF3A008080FB00010078004F057800D9
:1014A0004F04BE00000006000400FA00889FBE0042
:1014B0008A1F7800110020000004E00082003A003A
:1014C000CBC2BF000068A3007D003200CDC2A800DF
:1014D000C9C2A900B0132000101388006422EF00D5
:1014E00061E2A80061E2A90062C2BF0031CEB30090
:1014F000014060004041B30062E2B70062C2BF0039
:10150000C1CFB300014060000004A00062E2B70058
:1015100061E2A800A8C0B30000C0EB0037FF0700DD
:101520000844E900FCFF3A006011B8000840780068
:10153000A4FF070080447800E14F50004A003A00C1
:10154000803E2000A0F98800A21A2000030020009D
:1015500080C0B3009BFF0700E14F50002A003A0013
:10156000EA84570000C0EB0024FF0700805C78008D
:1015700066805700808F5400FAFF3A000FF89700FA
:10158000E14F500038003A009FF89700A0CAB3001E
:1015900080CF500034003A00341FE20006003200D1
:1015A000020020000300240090CAB30085FF07005A
:1015B0000004E000F8FF3A00341FE2002A00320085
:1015C0006011B800A0C3B3007EFF07000004E00074
:1015D00025003A006A84570000C0EB0007FF0700AF
:1015E000005C7800890F5400FBFF3A00EFF0970091
:1015F0000180FB00C8C0B3000068A3001B003A00D4
:1016000048C0B300190037006011B80090CAB30099
:101610006CFF070028C0B3009ACAB300E14F500026
:10162000020036000944780009457800341FE200C2
:10163000050032006011B8000A40780061FF070021
:101640000004E000F9FF3A00341FE2000600320017
:10165000022020000300200000C1B30059FF070052
:101660000004E000010032000044EB000880FB00B1
:1016700080F98800F5FE07000804E0000B00320046
:10168000561FA90061E2A90062C2BF0031CEB300BB
:10169000014060008041B30062E2B70030C0B30097
:1016A0006262B70061E2A80005003700EAFE0700A9
:1016B000E6FE0700C9C2A80061E2A900561FA80003
:1016C00056DFBF008080FB00010078004F057800E6
:1016D0004F04BE000080FA00000006001100200048
:1016E0000004E00002003A0056DFBF008080FB00EB
:1016F0000100780000000600889FBE008A1F780065
:1017000001057800844478000004E00032003A00CB
:101710000404E0003000320056DFBF0061046000C6
:10172000300020002D003A00307FAB0004003A006A
:101730004918DD00C711DE00830170004911DD008A
:10174000E1CF54000B003A0010C1B3001DFF0700A9
:101750000004E00019003A00012020000A0078008F
:10176000C6FE07000000E000140032008844780044
:101770001300370020C1B30012FF07000004E0008F
:101780000F003A0009447800012020000A00780088
:10179000BAFE07000000E000030032000A20B0009B
:1017A0000844E900F8FF3A00884478006011B80066
:1017B000C0C0B30003FF07000100370019C0B30029
:1017C000A2FE07000000EB000904E0000300320065
:1017D0001000200001003700400020004F05780075
:1017E0004F04BE0000000600889FBE008A9FBE0016
:1017F0008C1F7800810578000204BE000445780043
:101800000004E00040003A000404E0003E00320022
:1018100056DFBF00310020000008A3003B003A0063
:1018200056DFBF00640660002100200037003A0048
:1018300080F980000038A30004003A00C918DD00D8
:10184000C714DE00898470004914DD00E14F5500A3
:101850000C003A000801BE0080C1B300D9FE0700A9
:101860000004E00021003A00E1CFB3000B00780053
:10187000B4FE07000000E0001C0032000C457800B8
:101880001B00370066006000040032000A81FB0084
:101890000300200070C9B300CAFE07000801BE00A3
:1018A00090C1B300C7FE07000004E00010003A003A
:1018B0000A447800C1CFB3000B007800A1FE0700F6
:1018C0000000E000030032000B20B0000844E900F3
:1018D000F8FF3A0008457800D1CFB3000000EB00D4
:1018E00098FE07000000E00001003A001AC0B300B3
:1018F00056FE07008000EB000A04E00003003200FF
:101900001100200001003700410020000100780094
:101910004F0678004F05BE004F04BE0000000600D1
:101920001000FA00889FBE008A1F78000205780028
:10193000480020000004E000D1003A0056DFBF005C
:10194000E104600038002000CD003A00EACF5000EA
:10195000A400320008003E00E1CF50001600320023
:1019600010003900E2CF50004F003200E3CF5000AA
:101970000A003A004F003700ECCF50009C003200C4
:101980006011B80090C0B3009B003900EDCF50004B
:101990009E003200EECF5000A90032004800200027
:1019A000B60037002CFE07000000E000B000320057
:1019B00026FE07001B0037006011B80090C0B3007E
:1019C00080FE07000004E000A9003A0001012000A9
:1019D0007680570029FE07000000E000A4003200D6
:1019E000AFE897000180FB004600DE003FF2970061
:1019F000AFF09700E14F50000C003A000480FB006C
:101A00004809DD00020040000000E800010020005D
:101A10004A09DD00C600DE00810071004A00DD00D9
:101A2000008DBE0009047800940037000181FB009E
:101A30004611DE001FF097000080FB004200DD0031
:101A4000000141000FF09700630060004A00DD00D4
:101A5000000141000201E80003002000FFE89700B8
:101A6000EFC060004FF097000008B2004780DE0032
:101A700080C04000630062000000400080C0400061
:101A800081C0E8008180FB00E98050008100E9000E
:101A9000030033000201410083814900FBFF37004E
:101AA000028DBE00DFFF3700002020000009780013
:101AB000DCFF370080F98000640460001D00320004
:101AC0006011B800D0C8B3003EFE07000004E0007B
:101AD00067003A0000C0EB00C8FD070001012000CC
:101AE00076805700E5FD07000000E000600032004E
:101AF00008C3B30000C0EB00C0FD07000844E900C4
:101B0000FCFF3A004FF197000281FB004411DE0018
:101B100000012000010020000201E9000300330061
:101B20000000400081804800FBFF3700008DBE00B0
:101B3000510037006011B80090C0B30021FE0700CB
:101B40000004E0004A003A000101200076805700BE
:101B5000CAFD07000000E000450032005FF1970079
:101B6000CFF0970080F98000620260000F00320021
:101B700001007800F003B200000040000208B2004B
:101B80004711DE00020040000000E8007FF19700EE
:101B90000281FB004611DE000201E9000200DD00C7
:101BA00001002000008DBE00340037000280FB00E1
:101BB00001017800C207B2004291DE000201E80094
:101BC000E3006000C308DD004500DE0080804000C7
:101BD0008100E8000191B900028DBE000404780084
:101BE0002600370030DFBF00004978008DFF370046
:101BF0006011B800A0C0B300F2FD07000101200091
:101C00000004E00016003200190037006011B8002F
:101C1000A0C3B300EBFD07000004E00014003A008D
:101C20000904780000C0EB0074FD070000757C001B
:101C30000804E800E40F54000F003200F9FF3700F9
:101C40006011B800D0C8B300DEFD07000004E0005A
:101C500007003A0000C0EB0068FD07000104200007
:101C60000A00780085FD07000000E00002003A004D
:101C700018002000010037000004EB0073FD07008E
:101C8000080078004F0578004F04BE000080FA007D
:101C900000000600A0F980000000E0000200320011
:101CA0000000E900A0F9880090F980000000E00041
:101CB000020032000000E90090F9880000000600F0
:101CC000889FBE00800478000004EB00030037000A
:101CD000803E2000B41E07000804E800890F54006D
:101CE000FBFF39004F04BE00000006008040EB00FF
:101CF00050C0B3006908070001C2B30000C1B300BF
:101D000066080700E0152000EDFF07008040EB00AB
:101D100000C1B3006108070001C2B30010C1B300E5
:101D20005E080700E0152000E5FF07008040EB009B
:101D300010C1B3005908070001C2B30040C1B3008D
:101D400056080700E0152000DDFF07008040EB008B
:101D500040C1B3005108070001C2B30050C1B30035
:101D60004E080700E0152000D5FF07008040EB007B
:101D700050C1B3004908070001C2B30020C1B3003D
:101D800046080700E0152000CDFF07008040EB006B
:101D900020C1B3004108070001C2B30030C1B30045
:101DA0003E080700E0152000C5FF07008040EB005B
:101DB00030C1B3003908070001C2B300D0C1B3007D
:101DC00036080700E0152000BDFF07008040EB004B
:101DD000D0C1B3003108070001C2B300E0C1B300B5
:101DE0002E080700E0152000B5FF07008040EB003B
:101DF000E0C1B3002908070001C2B30050C0B3001E
:101E000026080700E0152000ADFF07008040EB002A
:101E100050C0B3002108070001C2B30060C0B30086
:101E20001E080700E0152000A5FF07008040EB001A
:101E300060C0B3001908070001C2B30070C0B3004E
:101E400016080700E01520009DFF07008040EB000A
:101E500070C0B3001108070001C2B300C0C1B300D5
:101E60000E080700E015200095FF07008040EB00FA
:101E7000C0C1B3000908070001C2B30040C2B300EB
:101E800006080700E01520008DFF07008040EB00EA
:101E900040C2B3000108070001C2B30050C2B30042
:101EA000FE070700E015200085FF07008040EB00DB
:101EB00050C2B300F907070001C2B300F0C1B3007C
:101EC000F6070700E01520007DFF07008040EB00CB
:101ED000F0C1B300F107070001C2B30080C1B30035
:101EE000EE070700E015200075FF07008040EB00BB
:101EF00080C1B300E907070001C2B30090C1B3007D
:101F0000E6070700E01520006DFF07008040EB00AA
:101F100090C1B300E107070001C2B300A0C1B30044
:101F2000DE070700E015200065FF07008040EB009A
:101F3000A0C1B300D907070001C2B300B0C1B3000C
:101F4000D6070700E01520005DFF07008040EB008A
:101F5000B0C1B300D107070001C2B30020C2B30073
:101F6000CE070700E015200055FF07008040EB007A
:101F700020C2B300C907070001C2B30001407800C6
:101F8000C6070700E01520004DFF07008040EB006A
:101F900000C2B300C107070001C2B30030C2B300E2
:101FA000BE070700E015200045FF07008040EB005A
:101FB00030C2B300B907070001C2B30010C2B300BA
:101FC000B6070700E01520003DFF07008040EB004A
:101FD00010C2B300B107070001C2B30060C2B30072
:101FE000AE070700E015200035FF07008040EB003A
:101FF00060C2B300A907070001C2B30070C2B300FA
:10200000A6070700E01520002DFF07008040EB0029
:1020100070C2B300A107070001C2B3000040EB008B
:102020009E070700E015200025FF07008040EB0019
:10203000014078009907070001C2B300E0C0B30077
:1020400096070700E01520001DFF07008040EB0009
:10205000E0C0B3009107070001C2B30010C0B30095
:102060008E070700E015200015FF07008040EB00F9
:1020700010C0B3008907070001C2B30060C1B300FC
:1020800086070700E01520000DFF07008040EB00E9
:1020900060C1B3008107070001C2B30070C1B30083
:1020A0007E070700E015200005FF07008040EB00D9
:1020B00070C1B3007907070001C2B30080C0B3004C
:1020C00076070700E0152000FDFE07008040EB00CA
:1020D00080C0B3007107070001C2B30090C0B30015
:1020E0006E070700E0152000F5FE07008040EB00BA
:1020F00090C0B3006907070001C2B300A0C0B300DD
:1021000066070700E0152000EDFE07008040EB00A9
:10211000A0C0B3006107070001C2B300B0C0B300A4
:102120005E070700E0152000E5FE07008040EB0099
:10213000B0C0B3005907070001C2B300C0C0B3006C
:1021400056070700E0152000DDFE07008040EB0089
:10215000C0C0B3005107070001C2B300D0C0B30034
:102160004E070700E0152000D5FE07008040EB0079
:10217000D0C0B3004907070001C2B30020C0B300BC
:1021800046070700E0152000CDFE07008040EB0069
:1021900020C0B3004107070001C2B30030C0B30044
:1021A0003E070700E0152000C5FE07008040EB0059
:1021B00030C0B3003907070001C2B30040C0B3000C
:1021C00036070700E0152000BDFE07008040EB0049
:1021D00040C0B3003107070001C2B30020C0B30004
:1021E0002E07070001C2B30000C1B3002B07070090
:1021F00001C2B30010C1B3002807070001C2B30039
:1022000040C1B3002507070001C2B30020C1B300DD
:102210002207070001C2B30030C1B3001F07070047
:1022200001C2B3000040EB001C07070001C2B3006D
:1022300010C0B3001907070001C2B300E0C1B3002A
:102240001607070001C2B30070C2B30013070700EE
:1022500001C2B30080C1B3001007070001C2B30080
:1022600090C1B3000D07070001C2B300A0C1B300C5
:102270000A07070001C2B300B0C1B3000707070097
:1022800001C2B300C0C1B3000407070001C2B3001C
:1022900040C2B3000107070001C2B30050C2B3003F
:1022A000FE06070001C2B300F0C1B300FB06070041
:1022B00001C2B300D0C1B300F806070001C2B300E9
:1022C00060C1B300F506070001C2B30070C1B300DE
:1022D000F206070001C2B30080C0B300EF0607009A
:1022E00001C2B300D0C0B300EC06070001C2B300C6
:1022F000E0C0B300E906070000802000461C07008C
:1023000010002000DF173700889FBE0070F32F00F9
:102310007812B400A1122000810F500004003E008A
:102320003E1FA8008040EB0070C2B300DB06070030
:10233000219380001093800080804000803E200028
:102340000088B900A2F82000801F78001100090061
:102350004288D800800078004F007800C118B10092
:1023600010022000808F500004003E008040EB00EF
:10237000D0C0B300C90607003E3FA800B9C72F0070
:10238000090078004412B400A8C12000880F500052
:1023900004003E008040EB0000C1B300BF06070010
:1023A0003E5FA800090078004612B400880F500074
:1023B00004003E008040EB0010C1B300B7060700E8
:1023C0003E7FA800090078004812B400880F500032
:1023D00004003E008040EB0040C1B300AF060700A0
:1023E0003E9FA800090078004A12B400880F5000F0
:1023F00004003E008040EB0020C1B300A7060700A8
:102400003EBFA800090078004C12B400880F5000AD
:1024100004003E008040EB0030C1B3009F0607007F
:102420003EDFA800090078004E12B400880F50006B
:1024300004003E008040EB00014078009706070052
:102440003EFFA800090078005012B400880F500029
:1024500004003E008040EB0010C0B3008F06070070
:102460003F1FA800B9F92F00090078005A12B400E4
:10247000E8312000880F500004003E008040EB004F
:1024800060C1B300850607003F3FA800090078003F
:102490005C12B400880F500004003E008040EB0046
:1024A00070C1B3007D0607003F5FA8007C12E20008
:1024B00002003A007A12E200040032008040EB0091
:1024C000D0C1B300750607003F7FA800F1938000DC
:1024D00080022000808F50000B0034001194800097
:1024E000800C2000808F500007003400B0122000C4
:1024F000808F500004003C003F9FA8008040EB000C
:10250000E0C1B300650607003FBFA8008040EB00B4
:10251000C0C1B300610607003FDFA8008040EB00A8
:1025200050C2B3005D0607002A12E2000D0032001F
:102530008040EB0090C1B300580607008040EB00DC
:10254000B0C1B300550607008040EB0040C2B300A5
:10255000520607008040EB00F0C1B3004F060700B1
:102560003FFFA8002C12E200040032008040EB0084
:1025700080C1B30049060700401FA8002E12E200E8
:10258000040032008040EB00A0C1B3004306070006
:10259000403FA8008B1A07000000E0000400320052
:1025A0008040EB00E0C0B3003C060700405FA8009D
:1025B0007212EC00E20F50000A003E007412EC00B0
:1025C000E20F500007003E00B0938000F40F50006F
:1025D000040034008040EB0080C0B3002F060700E9
:1025E000407FA800F2F9800003FA8000F0FF2F007E
:1025F000F1002000800F5100818F590006003A0041
:102600008040EB0020C0B3002406070001C2B300E5
:1026100030C0B30021060700E1F980008101E80025
:10262000E3F98800700C2000808F510002003E000A
:102630000000E800F092880084F32F00048040003E
:10264000620C2000820F500001003E00F4928800CE
:1026500000E72F0000804000820F500003003E0082
:102660005E32EF00800C20000093880080DA2F009B
:1026700000804000820F500001003E00049388005B
:1026800000CE2F0000804000E1182000810F500094
:1026900001003E006032EF00004B2000808F5100AF
:1026A00001003A003C3FEF004F04BE00000006006E
:1026B00090089000E0019000018140006281790063
:1026C0008100E9001108980002007800000006006F
:1026D000889FBE008A1F780000047800C004900024
:1026E000F3FF07000000400060857C00C8049000F4
:1026F00008007800EEFF070000004000E0807C004A
:10270000EF0F5500070032000A00E0000500350019
:1027100070022000800F550002003C000A40780043
:10272000DE0507004F0578004F04BE0000000600DC
:10273000800178000003EB000271220054002000A9
:10274000A5002000811F7800110009008281D800B7
:1027500081017800CF0078000000E00004003A001A
:102760000600E00002003A00E10F510003003A00C9
:1027700006C3B3008658400016002000811F780071
:10278000110009000581D80000017800CF00780011
:102790000402E900EBFF3A00E0C2B3008048780091
:1027A00070C7B3009040980076405000A040980059
:1027B00075404000B0409800C440980000000600FA
:1027C0000E00FA00881F7800F0805700929C2A00C3
:1027D0000C000900B2587800D100B100400490000C
:1027E000B3FF07000000400060047C0010002000E0
:1027F000161B0700E51107000000EB00E10F440085
:1028000004003200EF80570008007800C8FF07007E
:10281000708057002B1207004F0478000080FA00E8
:10282000000006000E00FA00881F7800F0805700B4
:10283000629D2A000C000900B2587800D100B10056
:10284000400490009AFF07000000400060047C00F4
:10285000E10F440002003A00260B07000700370092
:1028600010002000F91A0700EF80570008007800D8
:10287000AFFF070070805700F60A07004F0478008A
:102880000080FA00000006000E00FA00881F7800A1
:10289000F0805700329E2A000C000900B2587800E0
:1028A000D100B1004004900081FF0700000040000B
:1028B00060047C0010002000E41A0700B311070038
:1028C0000000EB00E10F440004003200EF805700ED
:1028D0000800780096FF070070805700F911070084
:1028E0004F0478000080FA00000006000E00FA0095
:1028F000881F7800F0805700029F2A000C00090012
:10290000B2587800D100B1004004900068FF070081
:102910000000400060047C0010002000CB1A07007B
:102920009A110700080078004C1207000000E00030
:1029300005003200EF805700080078007CFF070098
:1029400070805700DF1107004F0478000080FA0004
:1029500000000600E6874700889FBE008A9FBE00F1
:102960008C9FBE008E1F780000047800C004900089
:102970004FFF070000004000E0847C0089BF9F00FB
:10298000C80490000800780049FF070000004000DC
:10299000E0847C00F9B79F00C8049000080078002C
:1029A00043FF07000000400060877C00C8049000DF
:1029B000080078003EFF070000004000E0867C0031
:1029C000C80490000800780039FF070000004000AC
:1029D00060867C00C80490000800780034FF07007F
:1029E00000004000E0857C00C804900008007800EA
:1029F0002FFF07000000400060857C00C8049000A5
:102A0000080078002AFF07000000400060847C0076
:102A1000001020008D1A0700884378000A437800D0
:102A20008B4278000C4278008D4178000E4178008E
:102A3000EFE897000FF09700C40507004F077800F4
:102A40004F06BE004F05BE004F04BE006F00B10030
:102A500000000600889FBE008A9FBE000004780028
:102A6000C004900012FF070000004000E0857C00D9
:102A7000C8049000080078000DFF07000000400027
:102A800060857C00C80490000800780008FF0700FB
:102A90000000400060817C008A4078000B40780094
:102AA000D20507004F05BE004F04BE00000006001F
:102AB000889FBE008A9FBE0000047800C00490007A
:102AC000FBFE070000004000E0857C00C804900089
:102AD00008007800F6FE07000000400060857C00DA
:102AE000C804900008007800F1FE070000004000D4
:102AF00060817C008A4078000B407800C90507009F
:102B00004F05BE004F04BE0000000600889FBE00B7
:102B10008A9FBE0000047800C0049000E4FE070015
:102B200000004000E0857C00C804900008007800A8
:102B3000DFFE07000000400060857C00C8049000B4
:102B400008007800DAFE07000000400060817C0089
:102B50008A4078000B407800C00507004F05BE0092
:102B60004F04BE0000000600889FBE008A9FBE0082
:102B70008C1F780000047800C0049000CCFE070091
:102B80000000400060867C00C804900008007800C7
:102B9000C7FE070000004000E0857C00C8049000EC
:102BA00008007800C2FE07000000400060857C003D
:102BB000C804900008007800BDFE07000000400037
:102BC00060847C0020002000201A07008C407800E0
:102BD00000C2B300B10407008B40780030C2B300DC
:102BE000AE0407008A40780010C2B300AB040700AF
:102BF0008840780020C2B300A80407004F06780080
:102C00004F05BE004F04BE0000000600E6874700E7
:102C1000889FBE008A9FBE008C9FBE008E1F7800DA
:102C200000047800C0049000A1FE070000004000EE
:102C3000E0847C0089BF9F00C804900008007800F1
:102C40009BFE070000004000E0847C00F9B79F0075
:102C5000C80490000800780095FE070000004000BE
:102C600060877C00C80490000800780090FE070090
:102C700000004000E0867C00C80490000800780056
:102C80008BFE07000000400060867C00C8049000B6
:102C90000800780086FE070000004000E0857C0008
:102CA000C80490000800780081FE07000000400082
:102CB00060857C00C8049000080078007CFE070056
:102CC0000000400060847C0040002000DF19070005
:102CD0008FF0970000C1B30070040700EFE8970081
:102CE00010C1B3006D0407008E40780040C1B300EE
:102CF0006A0407008D40780050C1B30067040700E4
:102D00008C40780020C1B300640407008B40780039
:102D100030C1B300610407008A4078000040EB0036
:102D20005E0407008840780010C0B3005B04070011
:102D30004F0778004F06BE004F05BE004F04BE008F
:102D40006F00B10000000600889FBE008A1F780057
:102D500000047800C004900055FE07000000400009
:102D600060857C00C80490000800780050FE0700D1
:102D70000000400060847C0040002000B319070080
:102D80008A40780060C1B30044040700884078009E
:102D900070C1B300410407004F0578004F04BE0026
:102DA00000000600881F78004004900040FE0700E5
:102DB0000000400060047C0000042000A31907000C
:102DC00088407800D0C1B300340407004F04780075
:102DD00000000600881F78004004900034FE0700C1
:102DE0000000400060047C000001200097190700EB
:102DF00088407800E0C1B300280407004F04780041
:102E000000000600889FBE008A1F7800000478003A
:102E1000C004900026FE07000000400060857C0092
:102E2000C80490000800780021FE07000000400060
:102E300060847C0000202000841907008A4078000C
:102E400060C2B300150407008840780070C2B30068
:102E5000120407004F0578004F04BE000000060072
:102E6000889FBE008A1F780000047800C00490008C
:102E70000FFE07000000400060857C00C804900041
:102E8000080078000AFE07000000400060847C0013
:102E9000100020006D1907003C1007008800780022
:102EA0000A007800FC1007004F0578004F04BE00B0
:102EB00000000600889FBE00800478004004900057
:102EC000FBFD070000004000800144000001EB0012
:102ED000630079000008B000F10F2000810F50005E
:102EE00004003600D19F2A00090078005CF7070033
:102EF000060037000281E800C0112000800F510059
:102F0000F3FF3A0003007800241807004F04BE00C6
:102F1000000006005E1F00005210000000000000CC
:102F20009E1A000014010000020000000000FE00D4
:102F3000059E1F005C02D200112000005E1F0000F1
:102F40000000000000000000000000000000000081
:102F50000000000000000000000000000000000071
:102F60000000000000000000000000000000000061
:102F700000000000541B44001B341B002C1BB0003D
:102F80009E709E002C9EC6009D7A9D00269DD400BA
:102F90009C869C00289CC6009B569B00109B9E0014
:102FA0009A629A00089ABC00997899003099F400C6
:102FB00098A8980000989E000F920F00860F7A0044
:102FC0000F6E0F00460F32000F0A0F001E0F820017
:102FD0000EF20E00CA0EBA000EAE0E00A20E920045
:102FE0000E760E00181F00000072A30089A30000D7
:102FF00000000000A7A3BE00A3010000CEA30100B3
:1030000000D6A3000000000000DCA300F2A3010032
:1030100000CEA3000100D600A300000000000100C4
:10302000A410A40000000000005A9B005E9B8E00CC
:103030009BB69C00C874FA00742A75006C75AE00CB
:1030400075F0750036769A0076DE7600227790006D
:10305000770878005A78740078FE78004879820002
:1030600079BC7900507A8A007A847B0068931200D8
:1030700094E093004494760094AA94002A958600E4
:10308000955895003097B40095069600A496D20006
:1030900096EA960002975A0097CEB400C611000037
:1030A000C404000000000000B21B0000B4000000D7
:1030B00000000000FC0F0000040000000000000001
:1030C000B02F0000DC00000000000000AE0F000088
:1030D0003000000000000000501F0000020000004F
:1030E00000000000101F00000800000002000000A7
:1030F000661C0300800F0F000F000000661C00001C
:10310000A000000000000000181F000008000000E0
:1031100002000000BAACC400AC00000000000000D7
:10312000EA1E00000E00000000000000D830000081
:103130000C00000000000000521F00000200000010
:10314000000000009C1D0000300000000000000096
:10315000481F000004000000000000007E1E000068
:103160001400000000000000201F00000800000004
:1031700000000000281F0000080000000000000000
:10318000BA1E00001000000000000000541F0000E4
:1031900002000000000000000008000076060000A9
:1031A00000000000F81E00000E00000000000000FB
:1031B0008A1600000C020000000000004C1F0000F6
:1031C0000400000000000000561F00000200000084
:1031D0000200000001000000301F00000600000097
:1031E00000000000581F0000020000000000000066
:1031F000961800000802000000000000921E000067
:1032000014000000000000002A1E0000240000003E
:1032100002000000000001000000000001000000AA
:10322000000100000000010000000000010000009B
:10323000000100000000010000000000010000008B
:10324000000100005A1F0000020000000200000000
:10325000E8030000361F0000060000000000000028
:103260005C1F0000020000000200000008CC00000B
:103270004E1E00001800000000000000C0110000F9
:10328000060000000200000076117A001190110083
:10329000BE11000002000000020000003211000018
:1032A000901100002E000000020000002E035400C8
:1032B0000068000079006D00006900006F002D00BB
:1032C00000490000490020000020000020002000EC
:1032D000002000002000200000200000200020002E
:1032E0000020000020002000000000007A110000F3
:1032F000160000000200000016034D00006F0000E1
:10330000620073000079000061002E00006F000071
:103310007200670000000000761100000400000049
:103320000200000004030900040000003211000044
:1033300044000000020000000902430000020100F6
:103340000080FA00090400000001020002010000F0
:1033500005240000100104002402020005240600D8
:103360000001050024010000010705008103080099
:103370000002090004010000020A0000000007002A
:103380000502020040000000070582000240000024
:1033900000000000201100001200000002000000E8
:1033A000120100000202000000081700060A0000D7
:1033B00000000100020001001E11000002000000D8
:1033C00000000000161100000800000000000000CE
:1033D000CC1D00003000000000000000661E000050
:1033E0001800000000000000061D0000960000000C
:1033F00000000000CA1E00001000000000000000D5
:10340000DA1E00001000000000000000FC1D00009B
:103410002E00000002000000101114001213000022
:103420000116170000840300840384000384030052
:1034300084038400038403000000000000A00F0048
:10344000A00FA0000FA00F00A00FA0000FA00F0062
:103450008403840003000000A61E00001400000086
:1034600000000000DE0F00001E0000000000000051
:10347000061F00000A000000020000009001040086
:103480000120000096002C00010000003C1F0000FD
:103490000600000000000000760E00003801000069
:1034A0000200000022A72D00A78E000058A70000F0
:1034B000000000005DA76800A701000077A70100D9
:1034C000007AA70000000000007DA7008EA7010081
:1034D000009AA70001009E00A70000000000A300C2
:1034E000A7AEA7000100BC00A70000000000C000BC
:1034F000A7C8A7000100BC00A70000000000D3007F
:10350000A7DFA7000100FB00A701000001A8000041
:103510000000000007A81300A8010000FBA701009D
:103520000001A80001003100A801000037A8010037
:10353000003DA80001004300A801000049A80100C7
:10354000004FA800000000000055A80062A801007C
:1035500000FBA70001000100A801000031A8010044
:103560000037A800000000000073A80084A8010034
:10357000009AA70001009B00A80100009EA7000080
:1035800000000000A1A8B300A80100009AA7010054
:10359000009BA80001009E00A70000000000CB00D7
:1035A000A8D4A80001009A00A70100009BA8010070
:1035B000009EA7000000000000E4A800F0A80100A1
:1035C00000FBA70001000100A801000031A80100D4
:1035D0000037A80001003D00A801000043A8010039
:1035E0000049A80001004F00A800000000000700EB
:1035F000A914A90001003500A9000000000037004F
:10360000A944A90001003500A900000000005D00E8
:10361000A968A90001003500A90000000000810090
:10362000A98EA90001003500A90000000000A80033
:10363000A9B2A9000100BC00A7010000BEA90000BA
:10364000000000008C3000002C0000000000000092
:10365000421F000006000000000000000000000003
:1036600090089000E00190000181400062817900A3
:103670008100E900110898000200780000000600AF
:10368000B20C070000003700080C07000000E00043
:10369000FDFF3A00000037009A0F07000000E0002D
:1036A000FDFF3A009EC0A900004804000100000090
:1036B000000006000000FE0000000600889FBE001B
:1036C0008004780040049000E5FF070000004000FF
:1036D00060047C0009007800E1FF070080007800AA
:1036E00090052000800F54000400360081652A00F8
:1036F000090078005AF5070006003700C90190005C
:10370000018140008800440020BB21006100780056
:1037100000B179004F04BE0000000600889FBE0083
:103720008004780040049000CDFF070000004000B6
:1037300060047C0009007800C9FF07008000780061
:1037400090052000800F54000400360081652A0097
:103750000900780042F507000600370088014400A0
:10376000490190008180400020BB21006101790067
:10377000823178004F04BE000000060001672A0075
:1037800037F5370040612A000000060000000600FF
:1037900081804000C2B52100E100790001400100B4
:1037A000402D2A000000060040AD21000000060068
:1037B000F0874700889FBE008A9FBE008C9FBE0096
:1037C0008E1F780080BF9F00588E8000698E800019
:1037D00020009000D0B79F0050C0B300E2EF070078
:1037E0000085EB008085EB006066B8003E0020009D
:1037F0000800BE00200407008A0F50008B8F58007D
:10380000020031000005BE000806BE000080200056
:103810000100200008044000898448000E07E900E8
:10382000F3FF3A0091682A00E10F4500E08F4D0058
:103830004600320061054500E0854D00EAB79F0073
:10384000FBB79F000C04BE002A0020000800BE0049
:10385000720407000A05E900004020000100200072
:1038600008044000898448000A00E000F7FF3A009D
:103870000C00BE009C0407006FB09700FFB09700DB
:10388000C70407008FB8970021009000C1BF200037
:10389000EB0407001A0507000C00BE00F603070042
:1038A0006FB19700FFB19700800F5100818F5900D1
:1038B00002003200416A2A002400370062054600F7
:1038C000E0854E00E93F20007A84570088017800A7
:1038D000320020000A00BE00FD0307003200200075
:1038E000DFB097000800780057B507000000E0003F
:1038F00013003A00DFB19700E3814100D3B79F0086
:1039000062054500E0854D008904E900EEFF3A00BC
:10391000FC815700220020000A00BE00EC030700D3
:1039200022002000DFB097007C80570046B50700DA
:10393000016F2A000000E00004003A000200370096
:10394000A16C2A000100370061712A000FB89700AE
:10395000C3F407004F0778004F06BE004F05BE00B6
:103960004F04BE000F01B10000000600889FBE009A
:103970008A9FBE008C9FBE003A8E80004B8E8000D6
:103980000A04BE000006EB002D362A000800BE0027
:10399000C20307009D0F500007003A000C06E80024
:1039A0000808B0000980B0008D86E800E80F5600D6
:1039B00005003200F5FF37000C00E0000200320085
:1039C000E80F560003003A000A00BE001304070087
:1039D0000006EB004760DD00CF80DE000A004000FB
:1039E0008B80480040040700B2DBBF008080FB00F2
:1039F000000020008C01460022362A006301790075
:103A0000030020000200700083807000640407003F
:103A1000310B200030BB210089040700B8040700E7
:103A20004F06BE004F05BE004F04BE00000006005A
:103A3000889FBE008A9FBE008C9FBE003C8E800087
:103A40004D8E80000C04BE000005EB002B362A00D2
:103A50000800BE00910307009B0F500007003A00CA
:103A60000A05E8000808B0000980B0008B85E8006E
:103A7000E80F550004003200F5FF37000080EB002E
:103A80000A00E0000F0032000A04E9004744DD00AC
:103A9000CFC4DE000C0444008D844C000800BE003E
:103AA00084030700B2FBB70062044400E0844C00CA
:103AB00033BB2100320B20000800BE008403070046
:103AC0000000EB004F06BE004F05BE004F04BE00D5
:103AD000000006000000FE00FEFF37000400FA00B0
:103AE000889FBE008A9FBE008C1F780010002000B7
:103AF000F0D488000200230000002000800078003D
:103B000002007800508E8800618E880000402400FA
:103B100011002000308E8800418E8800B3202000E4
:103B2000A2B922008300780050DA2200C50A0700FB
:103B300094C4BF000008A300020032009EC0A80089
:103B4000010037001E150700CFC0BF0081CFB300B2
:103B5000014060005040B300CFE0B700E0A9210071
:103B600091F20700F0D48000908E88008000200041
:103B7000D0908800588E8000698E80006055B80013
:103B80009ABF9F00ABBF9F003C0020000800BE0012
:103B9000390307008A0F50008B8F5800030039004B
:103BA0000005BE0098BF9F00A9BF9F0000802000B5
:103BB0000100200008044000898448000C06E90048
:103BC000F2FF3A00E00F5500E08F5D0002003A007E
:103BD0000C047800080037001FB99700AFB99700B0
:103BE00062004100E080490013D58000C2BF200080
:103BF0003703070018002000A0D629000817070087
:103C0000080078004F0678004F05BE004F04BE0044
:103C10000080FA0000000600CE31EF00D031EF0046
:103C20008080EB00E0A9210085F20700670B070008
:103C3000813E2000E0A9210096F40700E0A92100C0
:103C40008D080700320B070069D580000900D100FC
:103C5000E105600002003A000908A300F3FF3A0002
:103C6000EA1C210020042000010C200010C8700074
:103C70001A04CF000A003900620545001A04CF007B
:103C800006003900740A07000000E000040032005A
:103C9000C8CB02000000000001003700700444009F
:103CA00020042000F101200010C860000800E0009E
:103CB000DEFF32000B00E000020032000908A30022
:103CC000DAFF3A008801E900EF8F510005003C005F
:103CD000100020000300DD000080EA001A0D6000E3
:103CE00006003700021D2100F100540010002000E2
:103CF0000100DD000080EA0012096000F0D48000BD
:103D0000A08E8800E1FF2F0083805000C5FF3700A0
:103D10000600FA006680570021F121000400090026
:103D2000315878005000B10067DCBF0001C8B30013
:103D300001406000BFF8970001407000B0FF9F0095
:103D400060C6210061D02100E6815700040009000F
:103D5000335878005000B1005300B10065004000B6
:103D6000810F5000F8FF3A000080FA0000000600C2
:103D7000889FBE008A9FBE008C1F7800804278001A
:103D800001427800834478008181FB000980FB00B8
:103D90000080410001022000810F500002003C0021
:103DA000094478000100370004C450008280FB0001
:103DB000100020008105DD008880FB000585FB00E8
:103DC0006519B900020045006CC621000C004000D6
:103DD0000B41780090110700894F54000500320014
:103DE00088C054008180FB000C0045000B41780026
:103DF000891107004F0678004F05BE004F04BE0032
:103E000000000600889FBE008A9FBE008C1F7800BD
:103E10008042780001427800834478008181FB0071
:103E20000980FB000080410001022000810F50004A
:103E300002003C00094478000100370004C450002F
:103E40008280FB00100020000100DD0080C5EA0038
:103E50008880FB000585FB006519B900020045005C
:103E60006CC621000C0040000B417800AF11070028
:103E7000894F54000500320088C054008180FB0047
:103E80000C0045000B417800A81107004F06780090
:103E90004F05BE004F04BE0000000600889FBE0014
:103EA0008A9FBE00004178008144780070C2B30050
:103EB000804F51004A003E000280FB00C305DE0037
:103EC0000B457800674461008880FB0010002000EB
:103ED0000102DD00044178008B81FB0020F121000C
:103EE0006340780080406200FFCF540039003E00FC
:103EF0000904E00007003A0060C621000104E00068
:103F000002003200008041000F00370004C1EA00C7
:103F1000050037000104E0000E003A001D003700E4
:103F200002C1EA0060C621000080410001022000B9
:103F30007E1107002A0037000A80FB0061C62100BD
:103F40000100400004417800010220003211070006
:103F500023003700894178000841780088407800C4
:103F60000B407800A7FF070089404400FFCF5000B6
:103F70000200360000CEB30080C0400003C2B30090
:103F800089C15100084178000B40780078FF070094
:103F90001300370089417800084178008840780094
:103FA0000B40780072FF070089404400FFCF5000AB
:103FB0000200360000CEB30080C0400003C2B30050
:103FC00089C15100084178000A4078008DFF070040
:103FD000030037000104E000D1FF3A00D6FF3700AC
:103FE0004F05BE004F04BE0000000600D5A2A90088
:103FF000F8150700803E2000EB1507004022EF0077
:104000004382A9004362A9004342A9004322A900B8
:104010004302A90042E2A90042C2A90042A2A800AC
:1040200042C2BF0031CEB300014060008041B30006
:1040300042E2B70030C0B3004262B7001000200077
:104040002012880041E2A80012DFBF000080FB00C0
:104050004012880013DFBF000080FB004012880080
:1040600014DFBF000080FB004012880015DFBF0096
:104070000080FB004012880016DFBF000080FB00BC
:104080004012880080022000C7150700D5A2A800B2
:1040900025F121009542780034F121001442780086
:1040A00043F121009341780052F121001241780040
:1040B00061F121009140780060C6210066D02100A6
:1040C000054878001440980023409800324098003A
:1040D0004140980065004000860F5000F8FF3A000C
:1040E00000000600D5A2A90080022000AE1507003E
:1040F00012DFBF000080FB004012880013DFBF000A
:104100000080FB004012880014DFBF000080FB002D
:104110004012880015DFBF000080FB0040128800BD
:1041200016DFBF000080FB004012880080022000E4
:104130009D150700D5A2A800100020009A150700C1
:10414000D5A2A90041E2A900A7153700889FBE00AB
:104150008A9FBE008C9FBE008E1F780001447800AD
:10416000824478000345780084457800054678004D
:1041700086467800074778008040780080C1B30009
:1041800046FF07008840780090C1B30043FF070056
:1041900089407800A0C1B30040FF07008A40780042
:1041A000B0C1B3003DFF07008B407800C0C1B30031
:1041B0003AFF07008C40780040C2B30037FF070089
:1041C0008D40780050C2B30034FF07008E40780065
:1041D000F0C1B30031FF07004F0778004F06BE0063
:1041E0004F05BE004F04BE0000000600889FBE00C1
:1041F00001447800824478008040780020C0B300F9
:1042000026FF07008840780030C0B30023FF070076
:104210008940780040C0B30020FF07004F04BE0073
:1042200000000600889FBE000144780082447800A8
:1042300080407800B0C0B30018FF070088407800C5
:10424000C0C0B30015FF070089407800D0C0B3009C
:1042500012FF07004F04BE0000000600889FBE004A
:1042600001447800824478008040780080C0B30028
:104270000AFF07008840780090C0B30007FF0700DE
:1042800089407800A0C0B30004FF07004F04BE00BF
:104290000000060021E3A90085A0A9000040060057
:1042A0000C00FA00F27F80002043A9000018800073
:1042B000A0BF9F0010188000B0BF9F002018800092
:1042C000C0BF9F0030188000D0BF9F004018800002
:1042D000E0BF9F0050188000F0BF9F006018800072
:1042E0007018800040632800E0198800E20F510038
:1042F0001400320005003C000200E000080032001B
:10430000E10F51001A003A0009003700E30F510095
:1043100010003200E40F510015003A001100370080
:10432000C802A900C822A80010002000030037001E
:10433000C822A900C842A80020002000F07F880001
:104340000B003700C842A900C862A8003000200056
:10435000FAFF3700C862A900C882A8004000200008
:10436000F6FF3700C882A900C802A800FE2FEF00A0
:1043700010002000F17F80000100DD0001C6270051
:1043800001007000801988009021EF00C0C1B300C7
:104390009161B70021E3A8000000000000000000C8
:1043A0000000000000000000000000002043A80002
:1043B00000000000000000000000000000000000FD
:1043C00000000000000000003D63A80000000000A5
:1043D00000000000000000000000000000000000DD
:1043E0000000000090C1BF0081CFB3000140600019
:1043F0000024A00090E1B7000000000000000000D1
:1044000000000000000000000000000000000000AC
:104410003D23A900820078006C80570044130700F8
:104420000080FA0000000600E07F8000ADE7070092
:1044300021E3A90095A0A9003DE3A9000000EB003D
:10444000800C8800900C8800C802A900C822A9002E
:10445000C842A900C862A900C882A900E1C6070035
:10446000E1143700889FBE000004BE00D914070085
:10447000E87F880021A3A90021C3BF00C1CFB300FA
:104480000140600021E3B70000CEB3002063B70015
:104490002043A90023C3BF007F40600023E3B7008F
:1044A0002343A80022C3BF0031CCB3000140600009
:1044B0008041B30022E3B7002223A8002203A90011
:1044C00025E3A800F0C1B3002563B70000382E0033
:1044D00060198800300020005019880010C627009D
:1044E000801988008001EB004319880095A0A8007E
:1044F00067C164004411DD00AAC0BF00F1C8B30069
:104500000140600002407000AAE0B70040E32000D4
:10451000E019880000E02700F01988003DE3A800BA
:10452000830C8800930C8800C0C1B3009161B70070
:1045300010002000B00C8800B00C80000005B00016
:10454000A00C88008080EB00F27F20000300200098
:1045500008007800D4E70700E07F800009017800B8
:1045600001152A0063E70700CC02A900CC22A900AC
:10457000CC42A900CC62A900CC82A900C802A90043
:10458000C822A900C842A900C862A900C882A9001F
:1045900020002000F07F880021E3A8000000000038
:1045A000000000000000000000000000000000000B
:1045B0002043A800000000000000000000000000F0
:1045C00000000000C802A8003D23A90090C1BF0060
:1045D00081CFB300014060000024A00090E1B7004B
:1045E000E07F800041E707004F04BE0000000600A6
:1045F00074E7A90079EC07000000FE000000060047
:1046000084C4BF004300DE00610060008086FB00C0
:104610000004E00003003200E0FF2F00B03B880000
:104620000100370076A7EF0070A7EF0072A7EF0038
:1046300074A7EF0078A7EF007AA7EF0000CEB300D1
:104640004260B70045C7BF000044A1000046B30068
:1046500045E7B7000004EB000807780088047800FD
:104660006055B8002C00200040A7A8000040FE00C4
:1046700040A7A90046EC07000800E0000200320055
:104680007607A9008804A8007007A9007647A9004A
:1046900000E02700F01988000029B000E019880028
:1046A00025E3A80000382E006019880030002000A3
:1046B0005019880021E3A80020002000401988003C
:1046C0000002EB00010220002023A800C842A8003D
:1046D0003C03A8004567A80000000000000000009F
:1046E0003C03A9002023A900C842A9004567A900EE
:1046F00000188000000242008100E900F2FF3A0049
:10470000830B23000C00E000090032000C06E900D6
:1047100003007800810D230004187800810F5000F9
:10472000FDFF3A00000120000405B8000B0037002F
:10473000098144006280790000005500E0805D003E
:1047400004054000E085480004B179008904E800D0
:10475000F08F540001003A008C0478000201200020
:104760001100090042DDD80080007800B01220005E
:10477000808F500001003E00C112200040ED2F004C
:1047800000804000800F5200020039000007EB005B
:10479000040037000E07E800E30F570001003A005D
:1047A00093FF07007007A8007647A8000800E00004
:1047B000100032004567A80084C4BF000028A30091
:1047C00003003A0084C4BF000038A300FAFF32009F
:1047D0004567A90084C4BF000038A300030032006D
:1047E0000D00E00003003A0081FF07007607A800F3
:1047F0008006EB000800EA00080070004F00DE00B1
:104800006104100098FF37002104200091407800D7
:104810008180FB00C508DE0092028000FF3FFC00A3
:1048200000CEB3004260B700920288000500FC0091
:1048300050052000303B8800A00A2000303B880053
:1048400061E7A800000000000000000061E7AF0081
:10485000FEFF370092028000FF3FFC00C508DD002C
:1048600042C0BF007F4060000140700042E0B700DE
:1048700092028800000006000001BE009401800042
:10488000930188001080BA001201BA0094018800D8
:104890008000780002007800000006000002BE00E0
:1048A00092018000950188001000BA0092018800F2
:1048B000000006000002BE00920180009501880001
:1048C0001080BA00920188000080FB000000060002
:1048D000E8874700889FBE008A9FBE008C9FBE006D
:1048E0008E1F78000005BE00F2B79F0083BF9F00B7
:1048F000405EDE000D0020007FB097006104B8002C
:1049000061004600E0804E00C000DD000000200095
:104910000A0050008B8058008100D1000080D30035
:104920003200200003002000BFAF0700800F5400BA
:10493000818F5C00010036000004BE00080778008B
:1049400032002000110009000284D80080037800A2
:104950000103780090018000E0B79F009C0188006F
:104960000A02BE000FB997008001EB000A00370071
:104970001400BA00004978004800DE001041980099
:104980009480BA0021419800630141008301E8004E
:1049900062024200E0824A00878F5100F4FF390032
:1049A0000600E000060032001400BA00005978004A
:1049B000E10F5300020036004800DE000049780095
:1049C0006FB09700900188003200200003002000A3
:1049D0000800BE00A2AF0700000040008180480030
:1049E0000A0540008B8548000FB897000E00400074
:1049F00080BF9F007FB097000E005000F0B79F006F
:104A0000BBFF3A004F0778004F06BE004F05BE00BF
:104A10004F04BE008F00B100000006000400FA0041
:104A2000881F7800D0BF9F00E1BF9F000001BE003B
:104A3000F03FB20005003200E681570012E020008E
:104A4000210A200020CA2A00731307009801800061
:104A50009301880020042400003B88006110B80006
:104A60000008BB0068FF0700980188004F04780029
:104A70000080FA00000006000400FA00881F780099
:104A8000D0BF9F00E1BF9F000202BE00000178007E
:104A90000008A30005003200E681570012E0200064
:104AA000410B200020CA2A005B13070098018000F8
:104AB0009101880030002400003B880003002000A2
:104AC0006120B8000009BB004028DE000100200082
:104AD0000089BB004CFF0700980188004F04780054
:104AE0000080FA00000006000400FA00E0BF9F000A
:104AF000F1BF9F000001BE00F007B20005003200C8
:104B0000E481570012E02000610C200020CA2A0036
:104B10004113070082F2880093F288004E3EEF00B6
:104B20009001800020F38800930188001000240089
:104B3000003B88000080FA0000000600889FBE004D
:104B400000F82F00F1FF2F0082F2800093F2800026
:104B5000020040008380480078047000E084700008
:104B60000003EB0047E521003700BE004531DD00C2
:104B700008017100030020006102B8000409BB00B5
:104B80004008DE00010020000089BB000603E800A9
:104B9000E40F5300F4FF3A004F04BE00000006008B
:104BA0000002BE0086F2800097F280008601780045
:104BB0007F006300F80F500009003A004B39DD0018
